:020000040800F2
:1000000000800020D5030108CD100108214200081E
:10001000CF100108D1100108D31001080000000022
:10002000000000000000000000000000113B00087C
:10003000D510010800000000A13B0008E53B0008C6
:10004000D7100108D9100108DB100108DD100108E4
:10005000DF100108E11001086110010867100108B4
:100060006D1001087310010879100108E3100108F0
:10007000E5100108E7100108E9100108EB1001087C
:10008000ED100108EF100108F1100108F31001084C
:10009000F5100108F7100108F91001087F10010898
:1000A000FB100108FD100108FF10010801110108F3
:1000B00003110108051101080711010809110108C0
:1000C0000B1101080D1101080F1101081111010890
:1000D00013110108CD1801085D1D01081511010853
:1000E000A31001084D110108171101081911010889
:1000F0001B110108000000000000000000000000CB
:1001000000000000000000005FF808F110B5054C89
:10011000237833B9044B13B10448AFF300800123B3
:10012000237010BD800400200000000050F9010879
:1001300008B5034B1BB103490348AFF3008008BD6A
:10014000000000008404002050F9010808B50348AD
:100150000BF0CAFDBDE8084011F030BEE7AA010867
:1001600011F02CBE10B50446C06910B101210AF08F
:10017000E7FE206910B101210AF0E2FE204610BD21
:10018000F8B50025C0E901120570C0E90335C0E9E2
:100190000555C0E90755456206990446164600F123
:1001A0001C0704F051FC38B9314607480BF09CFDA0
:1001B0002021064803F0A2FF069A3946204604F0A3
:1001C0000BFC2046F8BD00BF05AB010830AB0108B1
:1001D000F8B50025C0E901120570C0E90335C0E992
:1001E0000555C0E90755456206990446164600F1D3
:1001F0001C0704F045FB38B9314607480BF074FD85
:100200002021064803F07AFF069A3946204604F07A
:1002100021FB2046F8BD00BF05AB010830AB01084B
:100220002DE9F04100259DF81860C0E90112057024
:10023000C0E90335C0E90555C0E9075545623146B7
:100240000446174600F11C0804F01AFA38B939467A
:1002500007480BF049FD2021064803F04FFF3246C6
:100260004146204604F0FAF92046BDE8F08100BF7F
:1002700005AB010830AB0108F0B5AFB009F0B2F83A
:100280000146044612A809F0B9FB05F063FC0546D7
:1002900012A90CF05BFB04F111036B632134704B6A
:1002A0002C6308AC6F4A009303216F4B2046FFF785
:1002B00067FF2146284605F0F3FC2046FFF752FF72
:1002C0004FF41653694A00930221694B2046FFF709
:1002D0007FFF2146284605F0E3FC2046FFF742FF5A
:1002E0000823644A00930221634B2046FFF770FF06
:1002F0002146284605F0D4FC2046FFF733FF5F4B2C
:100300005F4A009303215F4B2046FFF739FF2146E8
:10031000284605F0C5FC2046FFF724FF5A4B5B4AF0
:10032000009303215A4B2046FFF72AFF2146284617
:1003300005F0B6FC2046FFF715FF564B564A0093D2
:100340000321564B2046FFF71BFF2146284605F0A8
:10035000A7FC2046FFF706FF514B524A00930321AA
:10036000514B2046FFF70CFF2146284605F098FC2C
:100370002046FFF7F7FE0323012700264B4A009390
:1003800002214B4B2046FFF723FF2146284605F06C
:1003900087FC2046FFF7E6FE464B474A00970221BE
:1003A0002046FFF715FF2146284605F079FC204638
:1003B000FFF7D8FE414B424A394600972046FFF7E7
:1003C0002FFF2146284605F06BFC2046FFF7CAFEAA
:1003D0003C4B3D4A394600962046FFF721FF214617
:1003E000284605F05DFC2046FFF7BCFE374B384A37
:1003F000009602212046FFF7EBFE2146284605F035
:100400004FFC2046FFF7AEFE324B334A00960221E6
:100410002046FFF7DDFE2146284605F041FC204638
:10042000FFF7A0FE28462D4B2D4A2E4905F0FAFA7B
:1004300006212D4B2D4A08932D4BCDE9051209932A
:100440002C4B07960A9305AB93E807008DE807004D
:100450000B9694E80F0005F01BFE2FB0F0BD00BF17
:10046000E7A70108E0A70108CCA70108F9A7010840
:10047000EBA7010815A8010800A8010855DA010832
:100480005DA801081FA8010889A801088EA8010815
:1004900068A80108E4A80108DDA8010894A80108DB
:1004A00051A901084BA90108F2A801087DA901087A
:1004B0005EA9010888A90108CAA90108D0A90108F4
:1004C00001AA010806AA01081FAA01082AAA010810
:1004D0006BAA010877AA0108B2AA01086101000805
:1004E000BDAA0108E1AA0108CD0901080000080819
:1004F000550901084D01000807B5054B02A901F88F
:10050000010D012218680AF085FB03B05DF804FBB9
:100510009C04002007B50B4D0B4E0C4C2B6842F28F
:1005200010720DF10701186801F014FD0128F5D1D2
:100530003378002BF2D09DF8071020460BF0D4FB47
:10054000ECE700BF2C4900200400002071AB01083B
:10055000A0F14103052B02D8373840B27047A0F113
:100560006103052B01D85738F7E73038C0B20928A6
:10057000F3D94FF0FF3070472DE9F04F8DB005F003
:1005800003FB037833B15F480BF0AEFB4D215E48AF
:1005900003F0B4FD002205200121CDE9052001F082
:1005A0005BFB059018B95021584803F0A7FD584B44
:1005B00005AA1A6001240023C822CDE90043554949
:1005C000554802F013F84FF496700AF0B3FC8046D9
:1005D000C8200AF0AFFC064664200AF0ABFC0546D2
:1005E000C8200AF0A7FCCDF82C80DFF848814FF432
:1005F0009671074607A8C8F800000AF004FB00F04F
:10060000CFF921460AF054F800F0ECF9214608F041
:1006100087F842480BF068FB414811F045F900F0BB
:10062000E1F908F09FFBDFF810B1CDF80880DFF8A2
:100630000C91DFF80C81029BC822314618680AF041
:100640001DFB002818DD4FF0FF3A0024721E12F83F
:10065000011F09B3632C2CD80A291DD00D291BD0EA
:100660002029F4D00929F2D00846FFF771FF0028AD
:1006700006DA2C480BF038FB0A2002F031FBDAE7EF
:10068000BAF1FF3F1FBF40EA0A1028554FF0FF3A6A
:10069000013408BF8246DAE7BAF1FF3F03D02248AF
:1006A0000BF022FBE8E7012C01D12048F8E7002CF1
:1006B000E2D058460BF018FB214628460BF07AFB97
:1006C00040460BF011FB00234FF0010A89F800307F
:1006D00000F088F9C823E2B22946CDE9003A3B464A
:1006E00008F004FB039000F07DF908F03BFB104894
:1006F00089F800A00BF0F8FA384603990BF05AFB82
:100700004046CDE776AB010897AB0108ECAB01089A
:100710002C4900202EAC01081505000839AC010851
:10072000F90400088DAC0108B4AC0108E0AC010884
:10073000FFAC01089C040020F3AC01080400002079
:100740006EBC010870470000F8B54FF00047002666
:10075000194CD4E90223BB4208BFB24227D005F0AE
:10076000B9FF04F10805D5E900451449621C45F1BB
:100770000003097806F027FDB94208BFB0420446DD
:100780000D4614D008F02EFE036E60301B689847AB
:10079000A04271EB05030ADB294620460BF024FA40
:1007A000014607480BF0A0FA064B1878F8BD03F095
:1007B000D3FB054BF9E700BF080000202D07002000
:1007C000A8AD0108434800204048002010B5002093
:1007D000002107F01BFA044688B14179042905D0AD
:1007E00080290FD00B480BF07FFA01E000F004FFE6
:1007F000204607F0A5FD082120460AF0A1FB064B84
:10080000187810BD054B02790168186804F03CFDAA
:10081000EEE700BFE6AD01084048002030070020A9
:1008200038B508F0DFFD054608F058FF034C20827C
:10083000284608F05FFF608238BD00BF0800002036
:1008400008B508480BF050FA08F0CCFD036E603094
:100850001B689847044BC3E90201FFF7E1FF034B14
:10086000187808BDD6AD01080800002040480020D7
:1008700038B5114C2368DB0708D405F085F98022D0
:1008800001460E4804F03CFA012323600C4B0B4A4E
:100890001A60FFF7C5FF08F0A5FD05461C200AF009
:1008A0002DFB044605F1740108F000FB054B1C60AC
:1008B000054B187838BD00BFA0040020C8060020F2
:1008C00030070020D80400204048002008B508F078
:1008D00089FDBDE8084008F0BFBD000038B5114BE8
:1008E0001878D8B9104CD4E90023B3F1004F08BFF1
:1008F000002A14D008F076FD036E60301B6898471C
:10090000D4E90023821A61EB030314461D46002339
:10091000064AA242AB41B4BF0120002038BD0120ED
:10092000FCE700BF2C0700204800002043510100D5
:1009300008B50B4B1B685B680BB1012008BD094B68
:100940001B78002BF9D1FFF7C9FF0028F5D1064B22
:10095000186803685B689847003018BF0120EDE70E
:1009600030070020B0040020D80400201FB5612308
:10097000CDE9013101A9039205F0C6FE05B05DF88D
:1009800004FB07B58DF8041001A98DF805208DF83A
:10099000063005F079FF03B05DF804FB08F022BDD6
:1009A00038B50C4C2368DB0712D408F01BFD054654
:1009B00008F018FD05F1480100F15802064809F059
:1009C000A9FD0123054A06490348236015F0F7FDF8
:1009D000014838BDA8040020DC06002000000020EB
:1009E0004507000810B5074C2368DB0708D4FFF75C
:1009F000D7FF00F11C01044807F04CFE01232360DF
:100A0000014810BDAC040020080700202DE9F04F7C
:100A100091B008F0E7FC044608F0BEF9204608F063
:100A2000D1F9FFF729FCFA2002F05AF905F0ACF8E9
:100A3000054604F09BFC284607F0B8F9BA49284659
:100A400004F044FFB94CBA492060284604F03EFF48
:100A5000082804D0092802D0072840F06081002629
:100A6000A060B449284604F03AFF07460146B24860
:100A700018F0D8F8002840F0B9810523E360AF49A9
:100A8000284604F02CFF07460146AD4818F0CAF886
:100A9000002840F0C581452363600E234FF0010814
:100AA000237484F8118084F81280FFF79BFF81463D
:100AB0009E4C04AF0FCC0FC7D4F800C004AF09F1AF
:100AC00010040FCF0FC49F49C4F800C0284604F09B
:100AD00006FF044601469C4818F0A4F8002840F0A0
:100AE000B281C9F808009949284604F0EFFE431E78
:100AF000022B014640F2B48195480BF0F5F801262F
:100B00009449284604F0EBFE934B10AA186000238A
:100B100009A942F8343D0AF0CDFE039919B18F4876
:100B20000BF0E2F801268E49284604F0CFFEB0F51E
:100B3000616F00F29B818B4BC117C3E900018A49A9
:100B4000284604F0C3FEB0F5616F00F29581874B33
:100B5000C117C3E900018649284604F0B7FE431EC9
:100B6000632B014600F28E81824B1870002E40F0FC
:100B70008C81284600F0EEFE05F006F87E4904F070
:100B80008BFE08B1FFF7F8FC7C480BF0ADF808F0DD
:100B900029FC7B4D06462B687A4C13F0010F04D1DB
:100BA00005F098FD012320602B6006F160012068AC
:100BB00005F05CFC2068744905F05AFC664B25681A
:100BC0001A68724909A805F03BFC09A9284605F0F6
:100BD00091FC6F4D6F4A28706F492068FFF7C6FE81
:100BE0006E4A8DF806006E492068FFF7BFFE8DF84B
:100BF0000700206806F01AFD6A4A81466A492068A3
:100C0000FFF7B4FE694A834669492068FFF7AEFEE4
:100C1000684B8246684A6949206807F09BFA684A2F
:100C2000064668492068FFF7A1FE674A8DF805006F
:100C300066492068FFF79AFE2A7880466449206852
:100C400006F0BAFE0746634D20689DF806302A7804
:100C500080F828309DF806109DF80730FFF791FEC8
:100C60004B462A789DF807102068FFF78AFE5A4AFB
:100C70005B46494620681278FFF783FEDFF86891EB
:100C800033462A7859462068FFF77BFE33462A7898
:100C90009DF805102068FFF774FE9DF8053099F85F
:100CA000002031462068FFF76CFE43462A78314623
:100CB0002068FFF766FE494A53464146206812788D
:100CC000FFF75FFE3B462A7841462068FFF759FE52
:100CD0009DF8053099F8002039462068FFF751FE4D
:100CE0002B4A5346394620681278FFF74AFE5B4686
:100CF0002A7851462068FFF744FE206805F07AFF05
:100D000037480AF0F1FF01224FF4C871206805F05E
:100D10000BFF002001F058FD11B0BDE8F08F314805
:100D20000AF0E2FF01269CE6F9A701083000002046
:100D300015A801085DA8010831AE01088EA80108B8
:100D40006FAE0108E0A70108E7A70108CAA90108DA
:100D5000C5AE0108DDA80108D0040020FBAE0108E3
:100D60006BAA0108C8040020B2AA0108B804002038
:100D70007DA90108C0040020F5AF010800B00108FA
:100D8000A4040020D8060020CD0800081DB00108EA
:100D90002D0700207108000866C80108850F0008AB
:100DA00022B00108DD0E00082DB00108410800083E
:100DB00038B0010875110008310900083FB001087A
:100DC000CD07000800C70108490700084CB001081A
:100DD00049C80108404800204448002043480020FA
:100DE00056B001080CAE01080949002039462B48CD
:100DF00017F018FF08B90A2340E63946284817F0CB
:100E000011FF08B90F2339E63946264817F00AFFC3
:100E100008B9142332E624480AF066FF01262EE6BC
:100E20003946224817F0FEFE08B94F2334E639460A
:100E30001F4817F0F7FE08B94E232DE61D480AF0AB
:100E400053FF012629E621461B4817F0EBFE10B997
:100E5000C9F8088047E619480AF046FF464642E6C8
:100E6000174B187017480AF03FFF49E6014616482D
:100E70000AF03AFF012662E6014614480AF034FF00
:100E8000012668E612480AF02FFF12480AF02CFFEC
:100E900040F21B21104803F031F96AE655DA0108E7
:100EA00035AE01089DDA010839AE010874AE0108BB
:100EB00089A8010878AE0108DAA70108A1AE0108E7
:100EC000D4040020E4AE010816AF010841AF0108C8
:100ED0006BAF010893AF0108A6AF010813B5224C10
:100EE00020680368DB69984708F07CFA036E60307D
:100EF0001B6898471D4BC3E900010AF075FE0146C7
:100F00001B480AF0F1FEFFF74BFD012109F0D0FB71
:100F1000FFF768FD012107F003FCFFF741FD154BCA
:100F20001C30D3E90023CDE90023134BD3E9002380
:100F300000F028FC206800F06DFAFFF753FD002157
:100F400007F0EEFBFFF72CFD002109F0B1FB206854
:100F500003685B68984710B90122084B1A70084B68
:100F6000187802B010BD00BFD8040020080000208F
:100F700070B00108B8040020C80400202C0700202D
:100F80004048002013B5FFF74BFC18480AF0ACFEB0
:100F9000FFF706FD012109F08BFBFFF723FD01217F
:100FA00007F0BEFBFFF7FCFC114B124CD3E900230A
:100FB000CDE90023104B1C30D3E9002300F0E2FB05
:100FC000206800F027FAFFF70DFD002107F0A8FBCD
:100FD000FFF7E6FC002109F06BFB20680368DB6982
:100FE0009847064B187802B010BD00BF84B00108C6
:100FF000B8040020D8040020C80400204048002085
:101000002DE9F04FB2F5827FC9B007468946924676
:10101000049303D99721554803F070F840F2051363
:10102000534528BF53464FF0004405930023002644
:101030004FF00108CDE902343B6838465B689847B9
:10104000002800F08E803B68059A1B6906A9384687
:1010500098470528044607D845480AF045FE3B68EE
:1010600038469B699847E7E70DF119009DF818503D
:101070000AF051FFCDE90001E1B28C1F042DE4B26A
:101080002ED80539C9B24B1DDBB2B8F1000F42D0E2
:10109000529A9A4515702DD3062D26D8DDE90023E6
:1010A000484602910AF054FF80460299AAEB0803D1
:1010B0008B421DD3033D012D94BF0125002509EB73
:1010C0000800284498BF09F8084022460DF11E0187
:1010D00016F0C1FE2544EDB2A8445FFA88F80BE093
:1010E000072D2146CFD12346CFE74FF00008DDE79B
:1010F0000025F1E74FF000083B6838469B699847A8
:10110000049B46449E422CD2DDE900344FF0000897
:10111000CDE9023490E7049A8B19934221D8529B6F
:101120001B78AB421DD1DDE90223DDE900BC63453C
:1011300008BF5A4515D1049B9B1B9942DCD8033D3F
:10114000012D98BF4FF0010809EB0600404498BFFD
:1011500009F8064022460DF11E0116F07CFEA0445F
:10116000BBE7304649B0BDE8F08F00BFA6AF01082D
:101170008FAD01082DE9F041514E88B004460D466F
:10118000DE22314604A809F01AFE0023DFF8688148
:101190008DF80E30D8F800305F6887B149480AF002
:1011A000A3FD0DF10F032A463146D8F8000003F0E5
:1011B00001FE9DF80F302660637120711BE0424EE6
:1011C00096F80080B8F1000F18D040480AF08CFD66
:1011D0003F4A404913680968C91A8D4228BF0D4625
:1011E0004FF0050161713C4928BF377019442B4409
:1011F00021602571136008B0BDE8F081FFF76EFB38
:1012000000283FD035480AF06FFD08F0EBF8036E78
:1012100060301B689847324DC5E90001012104A8E0
:1012200009F0F8FD022104A809F0F4FD022104A848
:1012300009F0F0FD2B4B197811B1012183F80080E2
:10124000294E04A809F0E6FDB6F9121004A809F029
:1012500011FE318A04A809F026FED5E9002304A86E
:1012600009F015FE214B04A8197809F0D3FD04A854
:1012700009F0DBFD054604A809F0D9FD012325602E
:1012800063719AE71A480AF02FFD134F0DF10E0310
:10129000184800934FF482722B4639460068FFF7D6
:1012A000AFFE0C4B854218609DF80E3027606371CD
:1012B00083D2074B25711D60012333709BE700BF6C
:1012C000E40400200AAD0108B004002030AD01089C
:1012D000E0040020DC040020C205002054AD010819
:1012E000480000202C07002008000020D404002023
:1012F00071AD0108D804002030070020F7B508F0D0
:1013000071F80F25044640F6C13708F0E7F91D4E85
:10131000B8420CDC014630460AF0E6FC4FF47A7025
:101320000FF0F6FA204608F0D9F9013DF0D1236814
:1013300020469B689847FFF733FB0146204607F09D
:1013400071FD204607F028FD204608F05DF80024D6
:101350000123FA220C49CDE900340C48234601F060
:1013600045F90B480AF0C0FC0A480AF0BDFC01F040
:1013700017FB40F25B21084802F0C0FE204603B094
:10138000F0BD00BFBDB00108F7B001080D0A0008AC
:1013900000B1010813B10108A6AF010810B5044659
:1013A0002C2109F0CDFD204610BD0000FF22014B8D
:1013B0001A7070472D07002010B50446006801F030
:1013C00035F8204610BD000007B5074B8DF8070023
:1013D000186830B1012300220DF10701006800F008
:1013E00015FD03B05DF804FB4407002003463038C8
:1013F000C0B209280DD9A3F14102052A02D8373B12
:10140000D8B27047A3F16102052A01D8573BF7E72C
:10141000FF2070472DE9F04F6E4CD5B04FF4967217
:10142000074609A905A809F0CAFC23685A681B6881
:101430009A4205D168480AF057FC55B0BDE8F08FD4
:10144000FFF7D0FA012107F06BF92368634D5A6862
:101450001E680392039B9E4200F0B6802B7856F8DC
:10146000044B012B03D1032105A809F0D3FC2B78F1
:10147000022B7ED1062105A809F0CCFC584B05A80B
:10148000D3E9002309F003FD217956480AF02CFC2A
:10149000217920680AF08EFC53480AF025FCFFF7FA
:1014A000A1FA804605A8D4F8009094F804A009F0A9
:1014B000C7FC834605A809F0BFFCFF285DD805A836
:1014C00009F0BAFCC0B2494B52461B784946CDE9F7
:1014D00000035B46404607F009FC81460146804612
:1014E00043480AF001FC05A809F0AAFC49460AF0A5
:1014F00061FC3D480AF0F8FB2B78023B012B0ED82B
:1015000005A894F80480D4F800B009F099FCB8F16B
:10151000050F824633D84FF000085FFA88F841463D
:1015200005A809F091FC2B78012B11D12379032B0D
:1015300045D90222216805A8114409F04DFC237900
:1015400005A8052B8ABF23680021597909F062FCA0
:101550003B6805A89C6809F06AFC09A90246384660
:10156000A04710B923480AF0BFFB05A809F061FCA9
:1015700070E7032B82D107217DE7FF20A3E7B9F1B4
:10158000020FC8D94146584607F066F8431EDBB241
:10159000F92BC0D89AF901308046002B05DA0246B3
:1015A000FF21504616F07BFCB7E7C31C9945B2D328
:1015B00002460AF10301504616F058FCADE700213F
:1015C00005A809F070FCBAE7FFF70CFA002107F054
:1015D000A7F832E73807002044B10108D4040020FE
:1015E000080000206BB101086EBC0108C004002097
:1015F0007EB101088DB101082DE9F04FD5B0044648
:1016000004F0C2FA564904F047F928B955480AF0DF
:101610006BFB55B0BDE8F08FFFF7C0F9036E60308B
:101620001B6898474FF49672CDE9020109A905A8F5
:1016300009F0C5FB2679276831464B480AF054FB70
:10164000314638460AF0B6FB48480AF04DFBFFF732
:10165000A7F9012109F02CF8FFF7C4F9012107F0DF
:101660005FF80025DFF81891B54207D26C1C7D5D4C
:10167000E4B2022D0DD83E480AF036FBFFF7B2F96E
:10168000002107F04DF8FFF78BF9002109F010F861
:10169000BFE7321BD2B2954204D9294635480AF039
:1016A00023FBEBE7042105A809F0B4FBDDE90223E5
:1016B00005A809F0ECFBFFF795F9824605A809F0AB
:1016C000BFFB834605A809F0B7FBFF2807EB04081A
:1016D00021D805A809F0B0FBC0B201232A46CDE904
:1016E000000341465B46504607F000FB8246014638
:1016F00021480AF0F9FA514605A809F0A5FB032D87
:101700000BD0A11C0222394405A809F065FB052D68
:1017100008D8002108E0FF20DFE7002105A809F034
:10172000C2FBF6E798F8051005A809F073FB134B08
:1017300005A8D3F80080D8F80030D3F808A009F045
:1017400076FB09A902464046D04710B948460AF040
:10175000CBFA2C4405A8E5B209F06BFB84E700BF87
:1017600001AA0108F6B201084CB301086EBC0108D9
:101770005CB3010891B30108D7B30108D804002075
:10178000E5B301082DE9F74F1D46484B14461A688A
:10179000824612F00102984614D10121444E0846B7
:1017A0003260716000F058FA306018B95021414839
:1017B00002F0A4FC0123404A40493D48C8F80030EB
:1017C00014F0FDFE3E4B1A680AB9394A1A6054EA11
:1017D000050303D0DDE90C23134304D139480AF093
:1017E00083FA01205AE0294620460AF013FA80467F
:1017F000DDE90C010AF00EFA2D4E02464146324850
:101800000AF072FA00220DF10701306800F0A2FB25
:10181000FFF7C4F8026E6030126890474FF47A7B8D
:10182000DAF8002080465269504689462749904799
:10183000DAF800205046DFF8A8A0126A002190478D
:101840000AFB04F20DF10701B2FBFBF2306800F075
:1018500081FB0128374626D11D480AF045FA0C9B2A
:101860000AFB03F6B6FBFBFB5A460DF1070138688D
:1018700000F070FB012814D1FFF790F8036E603080
:101880001B689847B0EB080261EB0903944275EBC3
:101890000303E9DA0F480AF027FA002003B0BDE895
:1018A000F08F0D489BE70D4899E700BF34070020F3
:1018B0003C070020ECAB010800000020B913000831
:1018C0004407002019B4010839B40108C9130008FD
:1018D0006BB4010879B4010898B40108A7B40108F1
:1018E00040420F00F8B504460E46D0E9002180685A
:1018F0008B1A9B100133091AB3EBA10F4FEA830730
:101900000CD83A4462606FF04043216862683068E6
:10191000521A03EBA20341F82300F8BD38460AF03F
:101920007FFA054618B96921094802F0E7FBD4E9B6
:1019300000128A4203D0521A284616F097FA2068FD
:101940000AF058FA25603D44C4E90155DBE700BFC1
:10195000C3B401082DE9F04F0446C5B00C2009F0CE
:10196000CDFA00254D4FC0E90055856038604C49DF
:10197000204603F0B4FF4FF00108834681462C4611
:10198000DFF840A119F8016BB8F1000F0BD12C2E34
:1019900000D066B9A9EB0B0142480AF0A5F928214D
:1019A000504602F0ABFB2C2E2FD0002E54D03046E8
:1019B000FFF71CFDFF280346A9EB0B0209D100909D
:1019C000314639480AF090F94221504602F096FB20
:1019D000009BFF2C08D1354800930AF085F9462179
:1019E000504602F08BFB009BB8F1000F04D01D01A4
:1019F000EDB24FF00008C5E71D43EDB2631C04AA29
:101A000015554FF00108DCB2BCE71CB3284920464D
:101A100009F092FA034640B9009026480AF064F9AA
:101A20003021504602F06AFB009B04A9184622466A
:101A3000019316F010FA3A680820009209F05EFA55
:101A4000019B009A03600471039003A91046FFF7FD
:101A500049FF1EB1002495E7002CD7D13B681648FA
:101A600059681B68154EC91A89100AF03DF93B6880
:101A7000134FD3E9004844450CD054F8045B384672
:101A80000AF032F9286829790AF094F930460AF008
:101A90002BF9F0E745B0BDE8F08F00BF3807002014
:101AA0004BA90108B8B101085AB2010892B2010865
:101AB00051F6010845B20108BAB201086EBC01082E
:101AC000EEB20108F4B1010810B5044602F032F894
:101AD000A46B02F04FF8B4FA84F0400910BD70B561
:101AE0001546026C0446866B42B905689DB980684C
:101AF00001F0C0FBA5600136A66370BD6DB94068FA
:101B000016F0A9F96368226C1344A26863609342DB
:101B100001D3236863600020EDE7C06816F09BF9ED
:101B2000236CE2685B4221681A448A42E2603EBF4D
:101B3000A2689B18E360022DEDD10EB1013EEAE7E9
:101B40003046D8E703461A6C10B4084662B1D9682B
:101B50009C681144A142D96028BF196810BC28BFF5
:101B6000D960D96816F077B910BC704770B50446D3
:101B700001F0E0FF94F8455004F124066DB2002D09
:101B800014DCFF2384F8453001F0F4FF01F0D2FFAC
:101B900094F8445004F110066DB2002D12DCFF23BE
:101BA00084F84430BDE8704001F0E4BF636A002B64
:101BB000E7D0304601F0B0F908B101F02FFA013D4D
:101BC0006DB2DCE72369002BE9D0304601F0A4F9BF
:101BD00008B101F023FA013D6DB2DEE738B50D46DC
:101BE000044620B940F20311194802F087FA01F0C7
:101BF000A1FFD4E90F314B432268D0185B1A13447C
:101C0000A060E3600020FF23A063626084F844309A
:101C100084F8453095B9236963B104F1100001F0EF
:101C20007BF938B14FF080520A4B1A60BFF34F8FE7
:101C3000BFF36F8F01F09EFF012038BD04F110004B
:101C400001F0DEFE04F1240001F0DAFEF2E700BF4D
:101C500003B5010804ED00E0F8B50D461746064649
:101C600020B94FF4BB710D4802F048FA05FB06F0AD
:101C7000503002F099F8044648B155B92060C4E9E3
:101C80000F6501212046FFF7A9FF84F84C7020461C
:101C9000F8BD00F150030360F1E700BF03B5010890
:101CA0002DE9FF47884601921E46044620B940F2BE
:101CB000F1214B4802F022FAB8F1000F06D1236C53
:101CC00023B140F2F221464802F018FA022E07D161
:101CD000E36B012B04D040F2F321414802F00EFAED
:101CE00001F066FA30B9019B23B140F2F6213C487D
:101CF00002F004FA0027B946DFF8E8A001F01AFF65
:101D0000A26BE36B9A4201D3022E19D132464146AF
:101D10002046FFF7E4FE636A1BB104F1240001F0E2
:101D2000FBF838B14FF080522E4B1A60BFF34F8F43
:101D3000BFF36F8F01F01EFF012004B0BDE8F087F4
:101D4000019D1DB901F016FF0020F6E717B902A8A2
:101D500001F022F901F00EFF00F062FE01F0EAFE50
:101D600094F84430FF2B08BF84F8449094F8453031
:101D7000FF2B08BF84F8459001F0FCFE01A902A8E2
:101D800001F016F928BB01F0D5FEA26BE36B9A4275
:101D90000ED101F0EFFE019904F1100001F082F87C
:101DA0002046FFF7E3FE00F0E7FE48B10127A5E774
:101DB00001F0E0FE2046FFF7D9FE00F0DDFEF5E77A
:101DC0004FF08053CAF80030BFF34F8FBFF36F8FCF
:101DD000ECE72046FFF7CAFE00F0CEFEB4E700BFF6
:101DE00003B5010804ED00E010B502460021012012
:101DF000FFF732FF044638B1002383600360C360FD
:101E00001A461946FFF74CFF204610BD2DE9F8434E
:101E1000894690461F46044620B940F2C331274800
:101E200002F06CF9B9F1000F06D1236C23B14FF425
:101E30007171224802F062F9022F07D1E36B012B86
:101E400004D040F2C5311D4802F058F901F04CFFB2
:101E5000EFF311864FF0500383F31188BFF36F8FB8
:101E6000BFF34F8FA26BE36B9A4201D3022F22D1B3
:101E700094F845503A466DB249462046FFF72FFE8A
:101E80006B1C13D1636A0BB901200BE004F1240031
:101E900001F042F80028F7D0B8F1000FF4D001208B
:101EA000C8F8000086F31188BDE8F88301356DB2EB
:101EB00084F84550E8E70020F4E700BF03B50108C7
:101EC00070B50D46044620B94FF48C61204802F0ED
:101ED00015F9236C23B140F264411D4802F00EF95C
:101EE000236833B9A36823B140F26941184802F06E
:101EF00005F901F0F9FEEFF311864FF0500383F37B
:101F00001188BFF36F8FBFF34F8FA26BE36B9342C8
:101F10001CD994F8453001325BB2A2635A1C10D12F
:101F2000636A0BB9012009E004F1240000F0F4FF1A
:101F30000028F7D0002DF5D00120286086F3118805
:101F400070BD01335BB284F84530EBE70020F5E764
:101F500003B501082DE9F04385B00F460192044610
:101F600020B94FF4A061424802F0C8F837B9236C99
:101F700023B140F204513E4802F0C0F801F018F9D4
:101F800030B9019B23B140F20951394802F0B6F84B
:101F90000026B046DFF8DC9001F0CCFDA56BD5B192
:101FA00039462046013DFFF7CDFDA563236963B1A6
:101FB00004F1100000F0B0FF38B14FF080522D4B0B
:101FC0001A60BFF34F8FBFF36F8F01F0D3FD012075
:101FD00005B0BDE8F083019D1DB901F0CBFD0020E7
:101FE000F6E716B902A800F0D7FF01F0C3FD00F034
:101FF00017FD01F09FFD94F84430FF2B08BF84F8D3
:10200000448094F84530FF2B08BF84F8458001F0E8
:10201000B1FD01A902A800F0CBFFF0B92046FFF7FF
:1020200053FDA0B1019904F1240000F03BFF2046CC
:10203000FFF79CFD00F0A0FD38B94FF08053C9F8C0
:102040000030BFF34F8FBFF36F8F0126A4E7204608
:10205000FFF78CFD00F090FDF7E72046FFF786FDC7
:1020600000F08AFD2046FFF72FFD0028EDD0B6E7EF
:1020700003B5010804ED00E02DE9FF41044601919C
:1020800020B940F29151524802F038F8236C23B144
:1020900040F295514E4802F031F801F089F830B91C
:1020A000019B23B140F29A51494802F027F80025DC
:1020B0002F462E46DFF81C8101F03CFDA36BE3B1F7
:1020C000013BA363236813B901F074F9A06023698D
:1020D00063B104F1100000F01FFF38B14FF08052DF
:1020E0003C4B1A60BFF34F8FBFF36F8F01F042FD7F
:1020F0000125284604B0BDE8F081019B4BB925B10C
:1021000040F2E151324801F0F9FF01F033FD0025C2
:10211000EFE717B902A800F03FFF01F02BFD00F038
:102120007FFC01F007FD94F84430FF2B08BF84F8D2
:10213000446094F84530FF2B08BF84F8456001F0F7
:1021400019FD01A902A800F033FF40BB2046FFF7AC
:10215000BBFCF0B123683BB901F0ECFCA06801F0D6
:1021600037F8054601F006FD019904F1240000F05E
:1021700099FE2046FFF7FAFC00F0FEFC38B94FF05C
:102180008053C8F80030BFF34F8FBFF36F8F012724
:1021900092E72046FFF7EAFC00F0EEFCF7E7204666
:1021A000FFF7E4FC00F0E8FC2046FFF78DFC002878
:1021B000EDD0002D9DD001F0BDFC616A19B1236BFB
:1021C0001968C1F10501A06801F0A0F89DE700BF02
:1021D00003B5010804ED00E02DE9F04385B00F469A
:1021E0000192044620B94FF4CD61424801F086FFC8
:1021F00037B9236C23B140F26C613E4801F07EFF99
:1022000000F0D6FF30B9019B23B140F2716139482B
:1022100001F074FF0026B046DFF8DC9001F08AFC84
:10222000A36BD3B139462046E568FFF78BFC636AA0
:10223000E56063B104F1240000F06EFE38B14FF0A8
:1022400080522D4B1A60BFF34F8FBFF36F8F01F099
:1022500091FC012005B0BDE8F083019D1DB901F09E
:1022600089FC0020F6E716B902A800F095FE01F0FF
:1022700081FC00F0D5FB01F05DFC94F84430FF2BAD
:1022800008BF84F8448094F84530FF2B08BF84F8D9
:10229000458001F06FFC01A902A800F089FEF0B9A9
:1022A0002046FFF711FCA0B1019904F1240000F0D1
:1022B000F9FD2046FFF75AFC00F05EFC38B94FF0FC
:1022C0008053C9F80030BFF34F8FBFF36F8F0126E3
:1022D000A4E72046FFF74AFC00F04EFCF7E7204653
:1022E000FFF744FC00F048FC2046FFF7EDFB002818
:1022F000EDD0B6E703B5010804ED00E02DE9F843A1
:1023000089469046054620B940F2FB61204801F01D
:10231000F5FEB9F1000F06D12B6C23B140F2FC6140
:102320001B4801F0EBFE01F0DFFCEFF311874FF0EB
:10233000500383F31188BFF36F8FBFF34F8FAC6BE4
:102340001CB395F84460494676B22846FFF7FAFB7D
:10235000013C731CAC6313D12B690BB901200BE05A
:1023600005F1100000F0D8FD0028F7D0B8F1000FFB
:10237000F4D00120C8F8000087F31188BDE8F88385
:10238000013676B285F84460E8E72046F4E700BFFE
:1023900003B5010810B5044620B940F28A7105481A
:1023A00001F0ACFE01F0C6FBA46B01F0E3FB20469C
:1023B00010BD00BF03B5010838B5054620B940F28D
:1023C000A471064801F09AFE01F0B4FBA86BEC6B17
:1023D000241A01F0CFFB204638BD00BF03B5010829
:1023E000002330B5064A52F8335002EBC3041DB93E
:1023F00042F83310606030BD0133052BF3D1FAE7AA
:1024000084520020002310B5074A02EBC3014C6838
:10241000844204D1002042F83300486010BD0133EB
:10242000052BF2D1FAE700BF8452002010B5044614
:1024300020B94FF4F861054801F060FE2046FFF72F
:10244000E1FF2046BDE8104001F040BD03B50108A2
:1024500070B504460D46164601F06CFB94F8443006
:10246000FF2B04BF002384F8443094F84530FF2B41
:1024700004BF002384F8453001F07CFBA36B2BB92B
:102480003246294604F1240000F026FD2046BDE82E
:102490007040FFF76BBB0000064A13681968064BD3
:1024A00019B94FF0FF321A6070471268D268D268CB
:1024B0005268F8E74C070020FC07002010B50446DE
:1024C00020B940F2F261084801F018FE6269074B3A
:1024D0009A4207D1A06A064B984203D0B0FA80F026
:1024E000400910BD0020FCE74FB501081C08002082
:1024F00004080020F8B51B4B1B4E1C6805463068CD
:102500000F46043001F0ADFA334640B9012031687E
:10251000164EC96A3268884022EA000232606A1C9C
:1025200007D137B1196812480431BDE8F84001F00D
:1025300075BA1A686419546007D30E4A106819688E
:10254000BDE8F840043101F075BA0B4A106819680B
:10255000043101F06FFA094B1A68A24288BF1C606F
:10256000F8BD00BF4408002048070020CC07002029
:102570001C080020500700204C070020FC0700200A
:1025800080B5DFF86480144F144C154E236863B98E
:10259000144B1B68012BF8D94FF08053C8F800305A
:1025A000BFF34F8FBFF36F8FEEE701F0C3FAFB6805
:1025B000DD68281D01F055FA3368013B336023685C
:1025C000013B236001F0D6FA286B01F07FFC28461E
:1025D00001F07CFCDAE700BF30080020BC070020D7
:1025E000B80700205407002004ED00E02DE9F84F63
:1025F0004FEA820A804650460D4699460B9E01F0EE
:10260000D3FB0746002800F0AB805C2001F0CCFB38
:102610000446002800F0A180076325B94FF45871E3
:10262000564801F06BFD5246A521206B15F037FC92
:10263000236BAAF1040A9A442AF0070A6B1E04F1DC
:1026400034020F3513F8011F02F8011B197809B184
:10265000AB42F7D10A9D4FF0000B042D28BF042593
:10266000271DE562C4E9135B384684F843B001F0E6
:10267000D2F9C5F1050504F1180001F0CCF9C4F850
:1026800054B02461A561646284F858B04A4641465A
:10269000504601F025FA206006B1346001F04AFA94
:1026A000374B384E1A68DFF8188101321A603268E9
:1026B000002A58D134601B68012B25D1324801F023
:1026C0009FF9324801F09CF9314801F099F9DFF89F
:1026D000F490304801F094F92F4D304801F090F912
:1026E000484601F08DF9284601F08AF92C4801F09E
:1026F00087F92C4801F084F92B4801F081F92B4B24
:10270000C3F800902A4B1D6001252A4A2A49136804
:10271000086801331360E26A636405FA02F3034355
:1027200014200B60184B394600FB023001F076F99B
:1027300001F020FAD8F8003063B13368DA6AE36A4E
:102740009A4207D24FF080521C4B1A60BFF34F8F52
:10275000BFF36F8F2846BDE8F88F384601F0B6FB0F
:102760004FF0FF35F6E7D8F80030002BCCD13368B6
:10277000DA6AE36A9A4298BF3460C5E74FB5010848
:10278000B8070020480700205407002068070020F1
:102790007C07002090070020E4070020A407002009
:1027A00004080020300800201C0800204C070020EE
:1027B00050070020C8070020CC07002004ED00E0EF
:1027C00018080020D007002070B50446284D01F0FD
:1027D000B1F904B92C68261D304601F042F960B900
:1027E0001421E06A234B41435B5833B9012222494B
:1027F00082400B6823EA02030B60A36A1BB104F159
:10280000180001F02EF91D4A1368013313602B687C
:10281000A34220D131461A4801F000F9194A136841
:102820000133136001F0A6F9174B1B6893B12B68B5
:10283000A3420FD1154B1B6823B140F2B641144897
:1028400001F05CFC4FF08052124B1A60BFF34F8FC7
:10285000BFF36F8F70BD104A206B1368013B13608C
:1028600001F034FB204601F031FBFFF715FED9E7FC
:102870004807002054070020CC070020C80700208C
:1028800030080020BC07002018080020C4070020E2
:102890004FB5010804ED00E0B8070020F8B5054683
:1028A00020B940F24C51174801F028FC164B1B6828
:1028B000AB4220D001F03EF9144B6C691F68144BF9
:1028C0001E6801F057F9BC4217D0B44215D0114B25
:1028D0009C4208D1AB6A83B995F85830012B0CBFE4
:1028E00002200320F8BD0C4B9C4208D0002C0CBFEA
:1028F00004200120F6E70020F4E70220F2E704209C
:10290000F0E700BF4FB50108480700204C07002042
:10291000500700201C0800203008002070B5044635
:1029200020B940F21C71194801F0E8FB184D2B68E2
:10293000A34229D044B301F0FDF82046FFF7BEFDC5
:10294000F0B1261D304601F08CF801231149E26AEE
:1029500008689340034314200B600F4B314600FB83
:10296000023001F05BF82B68E26ADB6A9A4207D317
:102970004FF08052094B1A60BFF34F8FBFF36F8F38
:10298000BDE8704001F0F6B870BD00BF4FB501085A
:1029900048070020CC0700205407002004ED00E089
:1029A00013B50024174B0094019350222346164977
:1029B0001648FFF71BFE012818D100F099FE0128E8
:1029C00014D14FF0500383F31188BFF36F8FBFF31F
:1029D0004F8F4FF0FF320E4B1A600E4B18600E4BAC
:1029E0001C6002B0BDE8104001F024B9013007D1ED
:1029F00040F60401094802B0BDE8104001F07EBB7A
:102A000002B010BDF80700209BB501088125000821
:102A1000FC07002018080020440800204FB50108DA
:102A2000024A136801331360704700BFC4070020D7
:102A3000014B1868704700BF4408002008B501F03A
:102A400053F9014B186808BD44080020014B186871
:102A5000704700BFB80700202DE9F84F3A4B1B68BC
:102A6000002B6AD1394B1C6801341C609CB9384D6D
:102A70002B681B6823B140F66221364801F03EFB0B
:102A8000354B2A68196829601A60344A1368013383
:102A90001360FFF701FD324D4FF0000B2B68314FF3
:102AA000A34211D93A68304BD16A14224A439A584A
:102AB000022A28BF4FF0010B2C4A1268002A0CBFD3
:102AC00058460120BDE8F88FDFF884A0DFF8A49015
:102AD000DAF8002012681AB94FF0FF322A60E1E7F5
:102AE000DAF80020D268D66871688C4201D2296079
:102AF000D8E706F10408404600F0B3FFB16A19B107
:102B000006F1180000F0ADFF01224FF0140CF06A3E
:102B1000D9F8003002FA00F11943134BC9F800103C
:102B20000CFB0030414600F079FF3868F16AC26A58
:102B3000914228BF4FF0010BCAE70D4A4FF0000B3E
:102B4000136801331360B7E7C4070020440800206E
:102B50004C0700204FB50108500700200008002056
:102B6000FC070020480700205407002048080020E8
:102B7000C0070020CC0700202DE9F8432E4C236825
:102B800023B940F668012D4801F0B8FA00F0D2FFF1
:102B90002368013B236024682CB1002400F0EAFF85
:102BA0002046BDE8F883264B1B68002BF5D0254D49
:102BB000254EDFF8A8801FE0EB680127DC6804F1F0
:102BC000040904F1180000F04CFF484600F049FFEA
:102BD0001420E26A316807FA02F30B4300FB02801B
:102BE0004946336000F01AFF184BE26A1B68DB6A43
:102BF0009A4201D3164B1F602B68002BDCD10CB11D
:102C0000FFF74AFC134D2C6844B10127104EFFF723
:102C100023FF00B13760013CF9D12C600C4B1B68DD
:102C2000002BBAD04FF080520B4B1A60BFF34F8F7E
:102C3000BFF36F8F0124B1E7C40700204FB501082F
:102C4000B807002004080020CC0700204807002017
:102C500048080020C007002004ED00E054070020D1
:102C600038B50C46054620B940F2CA41184801F073
:102C700045FA24B940F2CB41154801F03FFA154B13
:102C80001B6823B140F2CC41114801F037FAFFF73D
:102C9000C7FE114B2A68186814192CBF01210021A6
:102CA00082422C600CD961B9FFF766FF38B94FF04A
:102CB00080520A4B1A60BFF34F8FBFF36F8F38BD3E
:102CC00009B9A042F0D20021201AFFF713FCEBE76C
:102CD0004FB50108C40700204408002004ED00E0BF
:102CE00010B5044640B94FF080520D4B1A60BFF347
:102CF0004F8FBFF36F8F10BD0A4B1B6823B14FF48A
:102D0000A461094801F0FAF9FFF78AFE0021204684
:102D1000FFF7F0FBFFF730FF0028E4D0EBE700BF40
:102D200004ED00E0C40700204FB50108224B70B548
:102D30001A68224B12B101221A6070BD204E1A602F
:102D400033681B6B1A68B2F1A53F0BD15A68B2F118
:102D5000A53F07D19A68B2F1A53F03D1DB68B3F173
:102D6000A53F04D030683168343101F097F9154B34
:102D70001C68B4FA84F41423E4B2C4F11F0463435E
:102D8000114DEB5823B940F68831104801F0B6F9DF
:102D9000142202FB04F3E9184868083340682B4406
:102DA000984202FB045408BF4368486008BF4B6068
:102DB0006368DB683360C0E7C40700204808002070
:102DC00048070020CC070020540700204FB5010819
:102DD00070B504462A4E00F0ADFE04B93468251DD6
:102DE000284600F03EFE60B91421E06A254B4143BD
:102DF0005B5833B90122244982400B6823EA02035D
:102E00000B60A36A1BB104F1180000F02AFE2946EA
:102E10001E4800F003FE94F858301D4D012B04BFEE
:102E2000002384F8583000F0A5FE2A682AB100F08B
:102E300081FEFFF731FB00F09DFE3368A34211D104
:102E40002B6883B1134B1B6823B14FF4D96112482F
:102E500001F054F94FF08052104B1A60BFF34F8FBE
:102E6000BFF36F8F70BD094A11680D4A1268914215
:102E700001D13360F6E7BDE87040FFF757BF00BFF0
:102E80004807002054070020CC0700201C08002021
:102E900018080020C40700204FB5010804ED00E029
:102EA000B807002038B50D46044620B940F69F31DA
:102EB000074801F023F9074B20461968183100F044
:102EC000B9FD2846BDE838400121FFF713BB00BF1C
:102ED0004FB501084807002070B50E461446054658
:102EE00020B940F6CA310A4801F008F9094B2846D2
:102EF0001968183100F092FD002C214608BF3046B9
:102F0000BDE8704018BF4FF0FF30FFF7F3BA00BFC5
:102F10004FB501084807002038B5C368DC6824B9FC
:102F200040F6FA31154801F0E9F804F11805284691
:102F300000F097FD124B1B68E3B9251D284600F0F1
:102F400090FD01230F49E26A08689340034314206F
:102F50000B6029460C4B00FB023000F05FFD0B4B71
:102F6000E26A1B68DB6A9A4285BF0120084B002099
:102F7000186038BD29460748EFE700BF4FB5010884
:102F8000C4070020CC070020540700204807002079
:102F90004808002004080020034B1B680360034B13
:102FA0001B684360704700BF0008002044080020F1
:102FB00070B50C46054620B940F66541144801F04D
:102FC0009DF824B940F66641114801F097F800F0E9
:102FD000B1FD104B1A682368591C0FD00E482E689B
:102FE00000686968864201D091420ED9521A934214
:102FF00009D99B1A23602846FFF7CEFF002400F072
:10300000B9FD204670BD002323600124F7E700BF0F
:103010004FB5010844080020000800200122014BA0
:103020001A6070474808002070B50C4616460546E1
:1030300008B91B4A156805F134026260EA6A052B7B
:1030400022612A6B2560E2616A6CA260EA6C6261AF
:103050004FF00002A2611BD011490968A9420BD1AF
:103060002273D6B1296B0A46531A12F8010BA52810
:10307000FAD09B08238470BD032B2373F1D1FFF793
:10308000CFFCAB6A0BB102232373FFF775FDE8E7B2
:103090002846FFF703FC2073E3E72684EBE700BF35
:1030A000480700202DE9F84F0D6881460C469246EE
:1030B0001DB300254FF0240B4B6801F108075B6836
:1030C000BB424B6004BFCB684B604B68D3F80C80AD
:1030D00063680BFB05915B6801229F42636008BF38
:1030E000E36805F1010508BF63606368DE68534665
:1030F0003046FFF799FFB045EAD12846BDE8F88F82
:103100002DE9F84305461746FFF78AFC1F4B1B685D
:103110008B4238D84FF0000824264446DFF88090D0
:1031200009EB080106FB04500122FFF7BBFFA8F1E1
:10313000140818F1640F0444F2D1154B02221968E7
:1031400006FB0450FFF7AEFF124B0444196802223D
:1031500006FB0450FFF7A6FF044404220E4906FBB9
:103160000450FFF79FFF044406FB045003220B4961
:10317000FFF798FF04440FB100233B60FFF7FCFC0E
:103180002046BDE8F8830024F8E700BFB807002018
:103190004C07002050070020300800201C080020A9
:1031A000A4070020014B1868704700BF48070020A3
:1031B000054B1B6833B1054B1B68002B0CBF02206D
:1031C000002070470120704718080020C407002025
:1031D0002DE9F0410446002836D0234AC36A11681D
:1031E0001746C96A8B4237D2142682691F4D002ABE
:1031F000A8BF3A6806FB0353A2BFD26AC2F1050218
:10320000826142699A4221D100F10408404600F0EF
:1032100028FC174B48B9E06A4643AA592AB901214C
:103220001A68814022EA01021A603A681968D26A73
:10323000E262012404FA02F00843186014204146B7
:1032400000FB025000F0EAFB204603E03B68DB6A2B
:10325000C3620120BDE8F0811368C06CDC6AA04243
:103260002CBF00200120F5E748070020540700206C
:10327000CC070020F8B5044608B90020F8BD1F4B64
:103280001B68834204D040F67A711D4800F036FF77
:10329000236D23B940F67B71194800F02FFF236D91
:1032A000E16AE26C013B91422365E6D0002BE4D158
:1032B000251D284600F0D5FB124E134A50B91421A3
:1032C000E76A794373582BB901201368B84023EAA1
:1032D00000031360E36CC3F10501A161E362012403
:1032E000116804FA03F0084310601420294600FB1B
:1032F000036000F093FB2046C0E700BF48070020B2
:103300004FB5010854070020CC070020F8B50D4642
:103310000446002845D0036D23B940F6C971214801
:1033200000F0ECFEE36C9D4238BF1D46E36AAB4201
:1033300037D0236D012B34D11B4B1B68A34204D122
:1033400040F6E471174800F0D9FE1426A269E36A3A
:10335000002AE562A4BFC5F10505A561134D6269A8
:1033600006FB03539A421CD1271D384600F079FB17
:10337000E26A0F4C40B95643AB592BB9012123687F
:10338000914023EA01032360012314202168934024
:103390000B432360394600FB0250BDE8F84000F0C3
:1033A0003DBBF8BD4FB50108480700205407002079
:1033B000CC070020044B1A681AB119680A6D013253
:1033C0000A651868704700BF480700202DE9F041E2
:1033D0001E4C1E4680460F46154600F0ABFB236888
:1033E00093F85830022B14D0012123685A6D22EA39
:1033F00008025A65236883F8581056B13046FFF723
:1034000079F84FF08052124B1A60BFF34F8FBFF321
:103410006F8F00F0AFFB00F08DFB15B123685B6D83
:103420002B602368002293F85830022B09BF012536
:1034300000252368596D04BFB9435965236883F893
:10344000582000F097FB2846BDE8F081480700208F
:1034500004ED00E0F8B50E4617461D46044620B9B7
:1034600041F219212B4800F049FE00F063FB0DB139
:10347000636D2B60022394F8585084F85830EDB2F5
:10348000042F16D8DFE807F00A0307051100636D63
:103490001E43666502E0636D01336365012D11D043
:1034A000012400F067FB2046F8BD022DF1D1002475
:1034B000F7E7636D0133F1D041F24A21154800F07E
:1034C0001DFEEBE7261D304600F0CBFA1420124A11
:1034D000E36A11689D400D431560104A314600FBB8
:1034E000032000F09BFAA36A23B141F25921094855
:1034F00000F004FE0A4BE26A1B68DB6A9A42CFD9ED
:103500004FF08052074B1A60BFF34F8FBFF36F8F9E
:10351000C6E700BF4FB50108CC07002054070020C4
:103520004807002004ED00E02DE9F843DDF8208095
:103530000E4691461D46044620B941F28C2135487D
:1035400000F0DCFD00F0D0FBEFF311874FF05003EB
:1035500083F31188BFF36F8FBFF34F8F0DB1636D8E
:103560002B60022394F8585084F85830EDB2B9F12A
:10357000040F16D8DFE809F00A0307051100636D90
:103580001E43666502E0636D01336365012D11D052
:10359000012087F31188BDE8F883022DF1D10020C6
:1035A000F7E7636D0133F1D041F2CF21194800F004
:1035B000A5FDEBE7A36A23B141F2DA21154800F03B
:1035C0009DFD154B1B6803BB251D284600F049FADD
:1035D00001231249E26A08689340034314200B60F8
:1035E00029460F4B00FB023000F018FA0D4BE26A3F
:1035F0001B68DB6A9A42CBD90123B8F1000F01D0D6
:10360000C8F80030084A1360C2E704F118010748FF
:10361000EAE700BF4FB50108C4070020CC0700202F
:103620005407002048070020480800200408002014
:1036300038B5054608B9084B1D68002400F07AFA31
:1036400095F85830022B04BF85F85840012400F04B
:1036500091FA204638BD00BF48070020F8B50F4C4E
:1036600000F068FA2568ADB90D4F0E4E384600F0EF
:10367000C7F9304600F0C4F90B4B2A461F600B4BCC
:103680000C210A201E60FEF7E7FA206010B10849FD
:10369000FEF7A6FEBDE8F84000F06CBA80080020F6
:1036A00054080020680800204C0800205008002022
:1036B000A0B50108914208B5416000610AD8D21A4C
:1036C00083699A420DD2084B011D186800F0B2F9C7
:1036D000002008BD9A4201D2994202D2011D034B3B
:1036E000F3E70120F5E700BF500800204C08002058
:1036F00007B5FFF7B3FF0C4B1B6843B90B484FF4FA
:10370000897100F0FBFC002003B05DF804FB084B5E
:10371000C822019301230749009307480023FEF7BD
:1037200065FF0028EAD0EFE780080020A5B5010872
:1037300084080020F2B50108553800082DE9F04151
:1037400080462C200D4617461E4600F02DFB0446F1
:1037500088B125B94FF4B671084800F0CFFCFFF7E7
:103760007DFF069BC4F80080C4E9065726626362A9
:10377000201D00F050F92046BDE8F081A5B50108F4
:103780002DE9FF410D4690461F46064620B94FF4ED
:10379000C3710F4800F0B2FC0E4C206878B1052DC3
:1037A000CDE9015803960DDCFFF702FD0023022846
:1037B0000CBF0A9A1A4601A92068FEF771FA04B0F4
:1037C000BDE8F08100233A4601A9FEF71FFBF6E7AA
:1037D000A5B50108800800202DE9F74300271A4D00
:1037E000DFF86C802B681A6832B9184A11681360C8
:1037F000296003B0BDE8F083DB68DC681E6804F173
:103800000409484600F02DF9636A20469847E369A9
:10381000012BE7D1A36933449E4206D26360246141
:103820004946286800F006F9DCE700230097324695
:1038300019462046FFF7A4FF0028D3D140F2723189
:10384000404600F05BFCCDE74C080020500800200B
:10385000A5B501082DE9F04F4FF00108624D89B080
:10386000DFF898B1DBF80020136843B30024D36875
:10387000D3F80090FFF7D4F8FFF7DAF85B4B8246F5
:103880001A681F4690425A4E1CD31860002C4CD028
:10389000584B1B681A68B2FA82F25209A9EB0A0166
:1038A0003068FEF7D5FDFFF767F998B94FF0805201
:1038B000514B1A60BFF34F8FBFF36F8F0AE00124A3
:1038C0009946D7E70393FFF787FF039BC3F800A050
:1038D000FFF752F9002205A93068FEF73BFB0028EC
:1038E000BED0059B002BF5DB079C636913B1201D3F
:1038F00000F0B7F8FFF79CF83B688146984201D288
:10390000FFF76AFF059BC7F80090092BE2D808FA79
:1039100003F313F4047A57D113F0C70F33D19B0686
:10392000D8D5204600F0D2FAD4E7814529D8FFF750
:1039300023F9DBF80030DB68D3F80CB00BF104009E
:1039400000F08FF8DBF81C30012B15D1DBF81810D4
:103950004B46524649445846FFF7ACFE60B10094CE
:1039600023464A4621465846FFF70AFF20B94FF43E
:10397000F471284600F0C2FBDBF824305846984723
:10398000A8E722468AE7A169069B4A4619442046D1
:10399000FFF790FE00289DD0636A20469847E369B0
:1039A000012B97D1A2690699CDF800A00A4453468D
:1039B00051462046FFF7E4FE00288BD140F201314A
:1039C000284600F09BFB85E7069BA36123B94FF4D3
:1039D0004671284600F092FBA1694B464A4649448D
:1039E0002046FFF767FE75E7A5B501087C080020B3
:1039F000800800205008002004ED00E04C08002062
:103A00004FF0FF3200F108034360C0E90223036175
:103A100000230360704700230361704743689A687E
:103A20004B608A609A68516099600368086101334D
:103A3000036070470A6830B5531C0AD103695A689D
:103A40004A6091608B6059600368086101330360CC
:103A500030BD00F108035C6825689542EFD8234625
:103A6000F9E70369D0E901128A60826851605968F8
:103A7000814208BF5A60002202611A68013A1A6046
:103A80001868704706480068006880F3088862B6C6
:103A900061B6BFF34F8FBFF36F8F00DF00BF000031
:103AA00008ED00E0002307B501930B4B1B680133C1
:103AB00003D0CA21094800F021FB4FF0500383F3E3
:103AC0001188BFF36F8FBFF34F8F019B002BFCD08A
:103AD00003B05DF804FB00BF50000020FAB50108F8
:103AE0004FF0807340F8043C054B21F0010140F891
:103AF000081C40F80C3C40F8202C4038704700BFB0
:103B0000A53A0008000000000000000000000000CE
:103B1000074B19680868B0E8F00F80F30988BFF315
:103B20006F8F4FF0000080F311884EF00D0E70473C
:103B3000480700204FF0500383F31188BFF36F8FC5
:103B4000BFF34F8F084A13680133012B136009D16B
:103B5000064B1B6813F0FF0F04D040F275110448A8
:103B600000F0CCBA704700BF5000002004ED00E028
:103B7000FAB5010810B5074C236823B94FF4BE719C
:103B8000054800F0BBFA2368013B23600BB983F3BF
:103B9000118810BD50000020FAB501080000000097
:103BA000EFF30980BFF36F8F0D4B1A6820E9F00F18
:103BB00010602DE908404FF0500080F31188FFF7A6
:103BC000B5F84FF0000080F31188BDE8084019688F
:103BD0000868B0E8F00F80F30988BFF36F8F704773
:103BE0004807002008B54FF0500383F31188BFF356
:103BF0006F8FBFF34F8FFEF72FFF18B14FF080523A
:103C0000024B1A60002383F3118808BD04ED00E025
:103C10000022054B05491A600A6041F26701044A17
:103C2000116007221A60704710E000E018E000E021
:103C300014E000E013B5264B264C1A78D2B201925C
:103C4000FF221A701B78244ADBB28DF803309DF8EE
:103C5000033003F0500313700723002223609DF804
:103C60000310581E090629D402B123602368032BD0
:103C700004D04FF49B71194800F040FA2368144AAD
:103C80001B0203F4E06323600024019BDBB213708A
:103C9000134B1A6842F470021A601A6842F07042BC
:103CA0001A60FFF7B5FF0F4B1C60FFF7EBFEFFF745
:103CB0003DF8FFF7F7FE204602B010BD9DF8033037
:103CC00001225B00DBB28DF803300346C7E700BF7B
:103CD00000E400E08C08002088080020FAB5010804
:103CE00020ED00E05000002008B5EFF305830F2B16
:103CF0000AD90D4A9B5C0D4A12789A4204D940F2C7
:103D0000A5210B4800F0FAF90A4B0B4A1B68126810
:103D100003F4E063934206D9BDE8084040F2B521C0
:103D2000034800F0EBB908BDF0E300E0880800208C
:103D3000FAB501080CED00E08C08002010B50F4B1F
:103D40001A68824218D35C681919884201BF416819
:103D5000184609195960446801198A4207D108496F
:103D600009688A421FBF5168126809194160984268
:103D7000026018BF186010BD1346E1E7A0440020A0
:103D80009008002038B5064B064D1C68246804B91D
:103D900038BD6307FAD07921284600F0AFF9F5E77E
:103DA000A04400205AB601082DE9F8430746FEF763
:103DB00037FE3F493F4D0B680BBB3F4A3F4E500714
:103DC0001DBFD01D20F0070002F570534FF4705353
:103DD0001CBF02461B1A00201344083B23F00703B4
:103DE00070603260C3E90000981A0B60C2E90030CD
:103DF000334B1860334B18604FF000432B602B6837
:103E00001F4252D1002F41D007F1080462071CBFA6
:103E100024F007040834002C47D02A4B1A6898462F
:103E2000A24242D3254B1E687268A24202D2306879
:103E3000002837D10968B14237D01F683168121B9A
:103E4000102A07F10807196010D906EB040919F0C8
:103E5000070F03D0D7211C4800F050F9736848467B
:103E60001B1BC9F804307460FFF768FF14497268BF
:103E7000D8F8003008689B1A8342C8F8003038BF71
:103E80000B602B681343736000233360FEF774FEEE
:103E90007B0704D040F217110B4800F02FF9384689
:103EA000BDE8F88333460646BEE70027EEE700BFCD
:103EB000900800209444002094080020A044002092
:103EC0009C440020984400205AB6010838B50446A6
:103ED00070B3184D50F8041C2A68114204D140F206
:103EE0002B11154800F00AF954F8083C23B14FF49F
:103EF0009671114800F002F954F8043C2A68134204
:103F000016D054F8081C99B923EA020344F8043C7B
:103F1000FEF786FD094A54F8043C1168A4F1080034
:103F20000B441360FFF70AFFBDE83840FEF724BEDC
:103F300038BD00BF944400205AB6010898440020C0
:103F4000014B1868704700BF98440020014B186867
:103F5000704700BF9C4400202DE9F04742488AB0DA
:103F600007F0C2FEFEF772FD2425079007993F482F
:103F700007F0BAFE0798684307F052FF04463C4832
:103F800007F0B2FE94B107990DEB05022046FFF74A
:103F9000B7F80023DFF8F4A0364F07900893089A8B
:103FA000079B9A421DD3204607F024FFFFF7C8FF66
:103FB0000446FFF7CBFF214602462F4807F094FE48
:103FC0002E4B2F4819889A888B1A07F08DFE2D4B9F
:103FD0001B6803B198472C4807F086FE0AB0BDE87D
:103FE000F087089B05FB03431B7B013BDBB2032BE4
:103FF00098BF1AF80320099B88BF3F22642B83BF18
:104000006420B3FBF0F30899002382BF05FB014154
:104010008969B1FBF3F308990898DDF820C0DDF851
:1040200020E0DDF82080DDF8209005FB004005FB56
:104030000949D9F81C6005FB0141CDE9033605FBB0
:1040400008439B69029305FB0E439B68019305FBA4
:104050000C431B8C009303694968384607F044FE03
:10406000089B013308939AE7BCB60108C8B601085B
:10407000D3B6010808B701083AB70108AC520020CE
:1040800059B701082045002038B10108B8B6010829
:10409000014B1860704700BF3C45002073B5124CBF
:1040A000064623780D46114A1BB913780BB172B638
:1040B000FEE70123002113700D48642213F0EFFE88
:1040C0002B4600960B4A6421094814F057FD0A4B11
:1040D0001B6803B198470125054E304607F048FE9E
:1040E00072B62570F9E700BF18450020AC440020E7
:1040F000AE44002090B701083C450020F7B5184CAD
:10410000064623780D46174A1BB913780BB172B6D1
:10411000FEE70123002113701348642213F0BFFE51
:104120002B460096114A64210F4814F027FD104BCE
:104130001B680BB10C4898470E4B1B6803B198479E
:104140000125094E0C4F304607F012FE384607F0A5
:104150000FFE72B6094B257000BF013BFCD1F2E7A0
:1041600019450020AD440020AE440020B8B7010836
:10417000A84400203C450020C7B70108FFFF0F00FE
:10418000F8B5DFF898C003681A4FCCF800304368E0
:10419000194E3B608368194D3360C368184C2B601F
:1041A000036918492360436982690B60164BC06933
:1041B0001A60164A1060DCF8000038683068286819
:1041C00020681C460968124D1968124E1268642254
:1041D0000021284613F063FE2368324664212846F6
:1041E00014F0CCFC284607F0C3FD0B4B00BF013B8D
:1041F000FCD1ECE72C450020344500203845002058
:1042000030450020144500201C4500202445002096
:10421000AE4400207DB70108FFFF0F0028450020B5
:10422000074B1B6803B198471EF0040F0CBFEFF358
:104230000880EFF309808169004A10478141000836
:104240003C45002010B1012106F07ABE704708B14C
:1042500007F0E6BD70478068704740687047436864
:10426000012B08D1D0E90432934204D018780030F1
:1042700018BF01207047002070474B6870B5042BB1
:1042800004460E464FF0000304D0C0E900338360BB
:10429000204670BDD1E90425AD1AC0E90033836022
:1042A0002846FFF7D4FFC4E900000544A560D6E91D
:1042B0000453024629468B4205D00AB10E78167087
:1042C00001310132F7E75B1B18446060E0E74268A8
:1042D0000346022A06D1D3E904031B1A032B01D992
:1042E00007F034BE002070474368032B06D1D0E9A5
:1042F00004329A4208BF0023184670470023FBE7A8
:10430000037870B581680446B3B1284A284807F09D
:10431000EBFC6368022B12D12046FFF7D8FF014661
:10432000244807F0E1FCE1680B78002B3CD02248E0
:10433000BDE8704007F0D8BC204A2148E7E7032BCE
:1043400005D12046FFF7D0FF01461E48E9E7042BC0
:104350000ED100251C4ED4E90431C91A8D4205D274
:10436000595D304607F0C0FC0135F4E71748D8E73F
:10437000012B08D12046FFF772FF1549154B002885
:1043800018BF1946E1E700250F4ED4E904239B1A14
:104390009D4205D2515D304607F0A6FC0135F4E799
:1043A0000D4807F0A1FCBEE70C48C1E7F0A80108E2
:1043B0006BB801087FB80108A1B801086FBC0108FB
:1043C00075B80108FCB9010871AB010889B801088A
:1043D00065B8010860B801088FB801086EBC010813
:1043E000B1F5705F2DE9F84304460F4602D917482E
:1043F00006F066FD066883689B1B994219D9D0F8C0
:1044000004900846FFF723FF05460346A9EB06087C
:10441000B14505D00BB132781A7001360133F7E798
:104420002068FFF70FFF05EB080325603D4463603C
:10443000A56025683DB92846C4E90155FFF702FF8C
:104440002846BDE8F8830120FBE700BFE3B7010879
:104450002DE9F0410368561A904682680446D21A44
:1044600096420D4615D93046FFF7F1FE0746034642
:10447000A84505D02A7803B11A7001350133F7E752
:1044800020683E44FFF7DEFEC4E901662760BDE810
:10449000F0814768481EFF1ABE420ED81A469D1981
:1044A000A91A002904DD10F8011F02F8011BF7E723
:1044B000002EA8BF9B196360E9E73D441F44FA1A28
:1044C000002A04DD10F8012F03F8012BF7E76368D9
:1044D0002E461846B04505D0327800B1027001363C
:1044E0000130F7E7A8EB05084344E4E708B509C83D
:1044F0001B1AC3F57050884202D2104606F0E0FC49
:10450000994238BF1946581805D2B0F5705F28BFD8
:104510004FF4705008BD4FF47050FBE72DE9F8439D
:104520000C46591C204615461F46FFF759FF064604
:1045300080B14FF00003EA1929462046FFF788FFB3
:10454000D4E901539D4208D00DB100232B7063685C
:10455000013363603046BDE8F8831B4A01212046E1
:10456000FFF7C4FF23680746A5EB0309FFF76FFEBB
:1045700010EB090F1CBF002300F8093023688046A8
:104580001A460146954205D009B1107808700132EB
:104590000131F7E7D31A01334344104619466568E1
:1045A000954207D019B192F800C081F800C00132DD
:1045B0000131F5E72D1A1D4420684744FFF742FEFC
:1045C000C4E90085A760C5E71EB801082DE9F041E0
:1045D00005460E4661B1D0E90132D21A8A4209D3AA
:1045E00000221E4403B11A700133B342FAD16B604A
:1045F000BDE8F081114AFFF779FF8046FFF727FEFB
:10460000D5E9001407460A460346944205D00BB18B
:104610001078187001320133F7E70023641A3C4424
:10462000264404B123700134B442FAD12868FFF75C
:1046300009FEC5E900744744AF60D9E752B90108E3
:10464000D0E90032D21A914210B503D9891AFFF786
:10465000BDFF10BD3CBF5B184360FAE770B50C4668
:10466000012120461646FFF7BBFE054628B1012171
:104670002046FFF7E5FF23681E70284670BD000046
:10468000426808B5012A06D1BDE808400A4600F193
:104690001001FFF7E3BF8168024807F025FB002007
:1046A00008BD00BFE1B8010810B50C1A134605D0CB
:1046B00001462246184613F0D9FB0346181910BDCF
:1046C0002DE9F0410446A2EB01081646A3682268D2
:1046D00008469B1A98450F4615D94046FFF7B7FD87
:1046E00005460346BE4205D00BB13A781A70013731
:1046F0000133F7E72068FFF7A5FD25604544C4E9CD
:104700000155BDE8F0816568AD1AA84504D8314669
:10471000FFF7CAFF6060F4E70D442946FFF7C4FFC6
:10472000636829461A468E4205D00AB1087810708F
:1047300001310132F7E7751B1D446560E1E770B593
:104740000E46D2E900313046C91A1446FFF748FE3A
:10475000054630B1D4E900124FF000033046FFF7B0
:10476000AFFF284670BD000070B5D0E9043100F1FC
:1047700010060446C91A3046FFF732FE054640B11E
:10478000D4E90712914206D1A168064807F0ACFAB5
:104790000025284670BD4FF000033046FFF790FF1C
:1047A000F7E700BF38B801082DE9F0418368A2EBB4
:1047B00001081746026804469B1A98450E4615D90B
:1047C0004046FFF744FD05460346B74205D0327820
:1047D00003B11A7001360133F7E72068FFF732FDA5
:1047E00025604544C4E90155BDE8F0814568AD1A2E
:1047F000A84505D839463046FFF756FF6060F3E715
:104800000D4429463046FFF74FFF636829461A4694
:104810008F4205D0087802B1107001310132F7E7FC
:104820007D1B1D446560DFE737B50D4601A81146C5
:1048300007F0A6FB04212846FFF7D2FD044630B15D
:104840004FF0000302AA01A92846FFF7ADFF20465A
:1048500003B030BDFFF7E8BF426808B5022A06D1B1
:10486000BDE808400A4600F11001FFF7DDBF81688E
:10487000024807F039FA002008BD00BF19B9010845
:10488000FFF7EABF2DE9F0410E4600211C4617460E
:104890008AB00DF108082022C0E9001181600546A8
:1048A000404613F0FCFA1E2C94BF22461F223946C4
:1048B000404613F0D0FA7368013B032B14D8DFE8AD
:1048C00003F00230404722462F49384614F0C4F91D
:1048D00028B122462D49384614F0BEF940B90122CC
:1048E00029463046FFF7BAFE28460AB0BDE8F081F7
:1048F00022462749384614F0AFF928B12246254907
:10490000384614F0A9F908B90022E9E700220AA9FB
:1049100041F8242D404614F0C3FA021C18BF0122AE
:10492000DEE700220AA941F8242D404614F0B8FA27
:10493000019B02464345D7D029463046FFF774FF16
:10494000D2E723463A4629463046FFF7E7FDCBE754
:1049500014F00106C8D1640821462846FFF740FD3F
:104960000028C1D021462846FFF76AFEB442BBD0DA
:10497000022107EB460007F01FFB0028B4DB2B6881
:1049800098550136F2E700BF60B80108F3B7010897
:1049900065B80108F8B7010830B51346426885B01C
:1049A000032A044600F110050A460FD0014601A86B
:1049B000FFF768FF204601AA2946FFF7C0FE04461C
:1049C0000198FFF73FFC204605B030BD2946FFF7B0
:1049D000A5FD0446F7E70000F0B5044685B0104693
:1049E00016460F4614F030F962680346032A16D0C3
:1049F0003246214601A8FFF745FFDDE90112914249
:104A00000BD04FF000033846FFF75AFE01250198FE
:104A1000FFF718FC284605B0F0BD0025F7E7441C59
:104A200021463846FFF7DCFC054618B9054807F073
:104A30005BF9EFE74FF00003321931463846FFF7D4
:104A400007FDE7E7FEB701080A4600F11001FFF78E
:104A5000C3BFF8B50D461946284616461F46FFF750
:104A6000BFFC044630B14FF00003F219314628462E
:104A7000FFF79AFE2046F8BD1346426810B5042A97
:104A800006D1BDE810400A4600F11001FFF7E1BF72
:104A90008168024807F028F9002010BDA8B8010875
:104AA0002DE9F0410C4690461D46064640B139B10D
:104AB0000849184606F040FA074618B930602060E9
:104AC000BDE8F0812A46414613F0C5F937602560FC
:104AD000F6E700BF51F6010870B5054610460E46D0
:104AE000144614F0B1F82246034631462846BDE884
:104AF0007040FFF7D5BF000010B50C4631B1044936
:104B000000F004FD231A5842584110BD0846FCE746
:104B10004BBB010810B500B121B9064807F0E4F815
:104B2000002010BD1AB9044AFFF7D6FFF8E70120AC
:104B3000F7E700BF6CB9010879B901082DE9F7431F
:104B400005460E4617469846FFF7E4FFC0B10F49E9
:104B5000222006F0F1F90446A8B13846FFF77BFBA6
:104B600081463846FFF7C0FB14F06EF84346CDE9A6
:104B70000090074A2221204614F000F830602C6093
:104B800003B0BDE8F0833060F9E700BF51F60108DB
:104B9000B3B901082DE9F8430E46984616F8013BD3
:104BA00002F1FF3903704660C0F8089004461546CC
:104BB0003D214A46304613F031F9074668BB4B4663
:104BC000182B28BF1823C4F83001A36204F10C0588
:104BD000A26A3146284613F03EF90022A66AA319BC
:104BE0001A7337B1D4F83021791C04F12C0013F07A
:104BF00032F90022D4F83031234483F82C202EB12E
:104C00002946404600F082FCC4F83401D4E9011280
:104C10000A48BDE8F84307F0DDB8831B023DED1AF2
:104C2000182B1A46A8BF1822B5F5807F28BF4FF46D
:104C30008075A262C4F83051C8E700BFBBB9010853
:104C400030B504460D46084B9DB00093074A084B0B
:104C5000642103A813F092FF03AA29462046FFF718
:104C60003BFF1DB030BD00BFADB90108A5B90108BB
:104C700088B901082DE9F0431646642203F10C04BB
:104C80008FB00746884620461849ADF8042013F037
:104C9000C9FF70B9336B23B1154A322101A813F053
:104CA0006DFF01AA41463846FFF716FF0FB0BDE879
:104CB000F08320460F4913F0B5FF0446A0B9736B8B
:104CC000002BEED00125DFF83490736B01A81B5D3B
:104CD000C5F1320128444A46013413F04FFF102C2D
:104CE00005F10205F1D1DCE7034ADBE7C7B90108AA
:104CF000CCB90108D0B90108D8B9010871AB0108D5
:104D0000016000210273C0E901117047F8B5054642
:104D100017460E4639B332B32049182006F000F981
:104D2000044608B3C0E9006700261D4B00F10807E0
:104D30004361C0E9026606618021384605F0FCFF48
:104D4000D4E90012384606F035F81449082006F078
:104D5000E7F890B16B68C0E9004603B96860AB68DA
:104D600003B15860A860F8BD0E4806F0BDFF0121F0
:104D70003046BDE8F84006F0E3B80B4806F0B4FF53
:104D80000A4A4FF4A9710A4806F0AEFF01212068D3
:104D900006F0D6F818212046EBE700BF51F60108CF
:104DA0008081828377BA01087CBA010898BA010829
:104DB000E1BA010870B54468054604B3266806F1F7
:104DC000080005F0C1FFD6E903239A42C4B216D108
:104DD0006B681BB96A210B48FFF790F968680821D6
:104DE00043686B6006F0ACF86B6803B9AB600121F7
:104DF000306806F0A5F81821304606F0A1F82046E4
:104E000070BD00BF14BA010810B50446006810B1A7
:104E1000012106F095F8204610BD7FB50546FFF745
:104E20001AFA13F011FF0446861C2846FFF715FAFC
:104E3000013803281DD8DFE800F00206080F073408
:104E4000601C04B070BD0D34FAE72846FFF74CFA39
:104E500013F0FAFE3418F3E701A82946FFF70DFA1C
:104E6000DDE9014301A81B1B06EB4304FFF7CCFF60
:104E7000E6E70B34E4E700002DE9F04786B0814611
:104E8000884614461D46FFF745FE68B12046FFF7E9
:104E9000C4FF4049074606F04FF80646C9F800002F
:104EA00028B93D4806F020FF06B0BDE8F08720464F
:104EB000FFF7D3F90138032864D8DFE800F00214C3
:104EC000253D2046FFF7C7F981462046FFF7C7F981
:104ED000324B334A002814BF18461046CDE90090E3
:104EE0002B46304A0AE02046FFF7B5F981462046B6
:104EF000FFF7EDF92B46CDE900902B4A39463046B5
:104F000013F03CFE05463AE0612D20460DD1FFF737
:104F1000A2F905462046FFF7E7F92B46234A009001
:104F20003946304613F02AFEECE7FFF794F9814644
:104F30002046FFF7D9F9D1E72046FFF78CF92B4639
:104F400000901B4A3946304613F018FEDFF868908F
:104F50002146054603A8FFF790F9DDE9034AA2457B
:104F60000AD0AF4214F8013B06D9791B70194A46A2
:104F700013F004FE0235F2E703A8FFF745FFC8F877
:104F8000005091E72046FFF766F92B460090094A4A
:104F9000C6E700BF51F6010877BA010860B80108FA
:104FA00065B80108E7B90108EFB90108F8B90108C7
:104FB000FFB9010805BA010871AB01082DE9F043FA
:104FC0000E4607469046D1B04FF49C72002102A8CD
:104FD0001D46589C12F063FF31463B46424602A8EC
:104FE000FFF7D8FD3678622E00F0E88029D83F2EF2
:104FF0004ED008D82E2E55D09DF80810754806F0D2
:1050000073FE754A52E0532E00F09B80612EF3D15F
:105010000DF1340971484A4605A906F065FE4F981E
:10502000002800F0C480FFF718F9032800F09E80E4
:1050300028466B4A2146FFF74FFD6A4806F054FEAA
:105040002DE0722E42D00ED8642E34D0672ED3D1EC
:1050500005A9654806F048FE33464F9A2146284682
:10506000FFF70AFF1BE0732E4BD0772EC4D15F48A9
:1050700006F03AFE0399002973D05D4813F0D2FD83
:10508000044600286DD15B4806F02EFE214669E0FB
:10509000594806F029FE21462846FFF7D1FD51B0B8
:1050A000BDE8F083554806F01FFE554A21462846C4
:1050B000FFF712FDF3E70399524806F015FE02AB25
:1050C0003A4621462846FFF7D5FDE8E705A94E48B0
:1050D00006F00AFE03994D4813F0A4FD20B93846A6
:1050E00000F02EF94A4AE1E74F993846FFF704FDF0
:1050F00008B1484ADAE74F9808B1FFF735FB722349
:10510000ABE705A944480DAA06F0EEFD4F993846D5
:10511000FFF7F2FC0028ECD14F9810B10DA9FFF772
:1051200093FC73234F9A21462846FFF7A5FE21687A
:105130003A4806F0D9FD2868216806F03BFE384859
:105140007CE705A937480DAA06F0CEFD4F993846F1
:10515000FFF7D2FC0028CCD14F9810B10DA9FFF772
:1051600073FC0121384600F061FE2AE04F98FFF7FA
:10517000BBF813F069FD08F1010606442A493046E0
:1051800005F0DAFE074690B14F98FFF7ADF8274AD1
:1051900003463146CDF80090384613F0EFFC39460F
:1051A0004F98FFF751FC0121384605F0C9FE6123F5
:1051B0004F9A21462846FFF7C1FCB8E71C4806F085
:1051C00093FD1C4806F090FD4FF49B711A48FEF7C2
:1051D00095FF64E74EBC010870BC0108A4BB010840
:1051E000BDBB0108C9BB010815BB010803BC010810
:1051F0002BBC010831BC0108EFBA0108F9BA01085B
:1052000003BB010806BB010826BB0108F0A8010882
:1052100039BB01083CBB010856BB01086FBB010844
:105220006EBC010880BB010851F60108DBBB010818
:10523000E0BB010881BC010898BA01082DE9F041E2
:105240000C4680460D4815461E46069F06F04CFD4E
:1052500004B14DB90A4806F047FD39463046BDE86D
:10526000F041084AFFF738BC069733462A462146E4
:105270004046BDE8F041FFF7A1BE00BFADBC01084C
:10528000C2BC0108D5BC01087FB504460D460068C4
:105290000C49164600F000FB78B100F075FC03AB3A
:1052A00000933246294602ABFFF7C8FFDDE9021240
:1052B0002046FFF72BFD04B070BD034806F014FD37
:1052C000F9E700BF4BBB010858BA010810B10C2127
:1052D00005F036BE704710B1012105F031BE7047B0
:1052E00030B513460D460446AC4207D01BB194E8D6
:1052F000070083E807000C330C34F5E7184630BD8F
:1053000010B5044638B1FAF72DFF2046BDE810402D
:10531000282105F015BE10BD70B50446406AFFF7A0
:10532000D5FFD4E90656AE4204D02846FAF71AFF54
:105330002835F8E7A06908B1FFF7E2FF204670BD05
:10534000F8B5054600242826074FD5E906031B1AA1
:10535000DB107B439C4205D206FB0400FFF704FAF6
:105360000134F2E7F8BD00BFCDCCCCCCF8B5044693
:10537000224806F0B9FC224806F0B6FCD4E9063112
:10538000994218D0C91A1F4EC91071431E4806F021
:10539000ABFC00252827D4E906031B1ADB10734356
:1053A0009D4205D207FB0500FEF7AAFF0135F2E793
:1053B000164806F099FCD4E90931154EC91A89102E
:1053C0007143144806F090FC00250C27D4E909032A
:1053D0001B1A9B1073439D4205D207FB050000F08A
:1053E00087FF0135F2E70C4806F07EFC0B4806F01B
:1053F0007BFCBDE8F8400A4806F076BCC4BD010855
:1054000081CF0108CDCCCCCCCEBD0108E0BD0108D8
:10541000ABAAAAAA19BE01086EBC010829BE0108E0
:105420001EB101082DE9F043002487B00646684606
:10543000CDE90044029405F0A9FA684605F03EFB68
:105440004FF028082F4F304DD6E906239B1ADB106A
:105450007B439C424ED208FB04F302EB0309D35C6E
:10546000002B43D14846FEF7F6FE0146684605F09C
:1054700017FB4846FEF7F1FE042837D8DFE800F0B6
:105480003803101A24004846FEF7E9FE0146684634
:1054900005F0BCFA50BBC2212846FEF72FFE25E0DE
:1054A0004846FEF714FF0146684605F095FAE8B94C
:1054B000C621F1E74846FEF717FF0146684605F0AA
:1054C000EFFA98B9CA21E7E7494603A8FEF7D5FEE7
:1054D000DDE903126846521A05F0BAFA18B9CF216D
:1054E0002846FEF70BFE0398FFF7F5FE0134ABE705
:1054F000D321D1E7684605F009FB029807B0BDE863
:10550000F08300BFCDCCCCCCFCBC01082DE9F0432E
:1055100005460E4600244FF028081A4F8DB0D5E9F5
:1055200006239B1ADB107B439C4224D208FB0429F0
:1055300031461822684613F0A1FB4846FEF78BFE61
:10554000182201460DEB020013F098FB684606F0A6
:1055500058FD684606F067FD06A806F052FD06A84D
:1055600006F061FD182268460DEB020113F074FB92
:1055700018B10134D3E74FF0000948460DB0BDE83B
:10558000F08300BFCDCCCCCC2DE9F04F06460F46C2
:1055900000244FF00C09DFF86C808DB0D6E9095378
:1055A0005B1B9B1008FB03F39C4224D21822394654
:1055B000684613F063FB182209FB04FB0DEB0200A5
:1055C00055F80B1013F05AFB684606F01AFD6846B2
:1055D00006F029FD06A806F014FD06A806F023FD36
:1055E000182268460DEB020105EB0B0A13F034FBA1
:1055F00018B10134D2E74FF0000A50460DB0BDE8B3
:10560000F08F00BFABAAAAAA10B51446FFF77EFF21
:1056100020B12146BDE81040FFF716BA10BD0000CA
:10562000F8B50C46064640F201120021224812F05D
:1056300036FC4FF4807221461F4812F00CFC1E49C4
:105640001E4806F051FB1E491B4813F047FB1C493E
:105650000546002013F042FB294607463046FFF777
:1056600055FFA0B929463046FFF78EFF044600B328
:105670000168144806F038FBA368384698470124AF
:105680002046F8BD3946104806F02EFBF8E73A46AA
:1056900029463046FFF7B8FF04460028F2D00B48F1
:1056A00006F022FB0A4806F01FFB3046FFF75EFEBD
:1056B000E6E729460748E7E7C446002042BE01085E
:1056C00003BA010848BE010871BE01085DBE0108A9
:1056D0006EBC01088ABE010810B54FF48072044602
:1056E0000649043005F0CAFA002805DD2046BDE869
:1056F00010400249FFF794BF10BD00BFC445002011
:1057000038B514461D46FFF701FF28B12A46214649
:10571000BDE83840FFF740B938BD10B51446FFF773
:10572000F5FE20B12146BDE81040FFF795B810BD49
:1057300010B51446FFF7EAFE10B12146FEF7A0FFB0
:10574000002010BD38B514461D46FFF7DFFE28B116
:105750002A462146BDE83840FFF78EB938BD000023
:105760002DE9F04700248CB0074603A8CDE9034497
:10577000059405F00BF9214603A8009405F022FAE0
:105780000146002834D0214603A805F0A4F940F2D0
:10579000E7330446009300263546DFF8F890009B77
:1057A000B34273D9214603A805F0C7F98246002801
:1057B0006CD1182321460DEB030203A805F04EF926
:1057C0000444214603A805F0C6F98046B0B10CAAEE
:1057D000214642F828AD03A805F0DEF8029A0444F9
:1057E00006A93846FFF799FF00B101350136D6E723
:1057F0006A4603A805F076F90446CCE7214603A8DB
:1058000005F0F3F970B10CAA02F8288D214603A81F
:1058100005F0ECF89DF80820044406A93846FFF787
:1058200087FFE1E7214603A805F0B0F9804668B19B
:1058300002AB01AA214603A805F021F9DDE9012305
:10584000044406A93846FFF75BFFCDE7214603A8CD
:1058500005F08EF990B10CAB43F8288D01AA2146D2
:1058600003A8CDF8048005F0E2F89DF80830044460
:10587000019A06A93846FFF765FFB5E7039B48463E
:10588000195D01F0E00106F02FFAAFE728460CB0F1
:10589000BDE8F08753BD010808B5FFF737FE18B122
:1058A000BDE80840FEF7DBBC08BD10B5044608465D
:1058B0001146FFF72BFE014620B9C4E90000A060A5
:1058C000204610BD2046FEF7D8FCF9E708B5FFF7E3
:1058D0001DFE18B1BDE80840FEF7F9BC08BD08B5CB
:1058E000FFF714FE18B1BDE80840FEF7FDBC08BD87
:1058F000037810B5044643B1044806F0F5F90021D9
:10590000204600F093FA0023237010BD3EBD01082D
:10591000002370B5D1E90025AD1A0446C0E9003373
:1059200083600E46284601D006F07AFAC4E90000EA
:105930000544A560D6E90053024629468B4205D0AE
:105940000AB10E78167001310132F7E75B1B18447B
:105950006060204670BD38B504460D460B781030A7
:1059600000F8103C4B68103140F80C3C51F8083CF2
:1059700040F8083C51F8043C40F8043CFFF7C8FFED
:1059800005F11C0104F11C00FFF7C2FF204638BDE1
:105990002DE9F843D0E90054641B9146A2101F4C36
:1059A00006465443B4F5705F0F4602D11C4805F01B
:1059B00087FA002C14BF22460122A418A1EB05058A
:1059C00026D2B4F5705F23D82CB30C20604306F0C8
:1059D00027FA804618EB05031CBF99E8070083E807
:1059E0000700424639463068FFF77AFC716800F1DB
:1059F0000C023846FFF774FC05463068FFF766FC7A
:105A00000C2303FB0484C6E90085B460BDE8F88379
:105A10004FF47054D9E7A046DCE700BFABAAAAAAAE
:105A20001EB801082DE9F043054685B008460C462E
:105A300017461E4613F008F9172803D982212D486E
:105A4000FEF75CFBCDE90147D5E9097803962A4AC0
:105A5000A8EB0706B41054430134B4F5705F02D9C3
:105A6000264805F02DFAEB6ADB1B9B1053439C4242
:105A700015D94FF00C0909FB04F91CB1484606F092
:105A8000CFF90446224641463846FFF729FC686AAA
:105A9000FFF71CFC26446C624C44AE62EC62EA6A7E
:105AA000D5E9090314491B1A9B10121A4B43921093
:105AB0004A430133934206D9114806F015F98C2167
:105AC0000C48FEF71BFBD5E90A3293420AD023B1FA
:105AD00004AA12E9070083E807000C33AB6205B0A3
:105AE000BDE8F08301AA194605F12400FFF750FF35
:105AF000F5E700BFFCBC0108ABAAAAAAE3B70108FE
:105B0000E1BC010838B500250346044603F8045BF0
:105B100029461846142212F0C2F90A4AC4E9065569
:105B20006261C4E90855C4E90A55C4E90C558021ED
:105B300005F069F82046044B044A0549FFF772FF57
:105B4000204638BD444500208D5B0008ADBE0108ED
:105B5000B9BE010810B5084C2368DB0709D4074813
:105B6000FFF7D0FF0123064A06490448236010F0DE
:105B700026FD024810BD00BF40450020C847002058
:105B80000000002019530008FFF7E4BF08B5FFF735
:105B9000E1FFBDE80840FFF7E9BB0022C0E90022B1
:105BA000826010B50C6804600A6042684C6844600A
:105BB0004A6082688C6884608A6010BD70B50E4649
:105BC00005461446B54217D09CB12B7805F110015B
:105BD00023706B6804F110006360AB68A360EB682E
:105BE000E360FFF7DAFF05F11C0104F11C00FFF789
:105BF000D4FF28342835E5E7204670BD2DE9F84369
:105C0000D0E90064A41BE310234C05465C43B4F5C3
:105C1000705F0F46914602D1204805F051F9002CE3
:105C200014BF23460123E418A1EB060623D2B4F5E2
:105C3000705F20D814B32820604306F0F1F8804646
:105C400018EB060002D04946FFF785FE394642466A
:105C50002868FFF7B3FF696800F128023846FFF7AC
:105C6000ADFFD5E900690746B14509D03046FAF7DE
:105C700079FA2836F8E74FF47054DCE7A046DFE7FE
:105C8000286808B1FFF73CFB282303FB0484C5E91F
:105C90000087AC60BDE8F883CDCCCCCC1EB8010841
:105CA0002DE9F047D0E9065704460E46DFF80C818F
:105CB0008AB0AF421BD029466846FFF74CFE6846C3
:105CC000FEF7C9FA81463046FEF7C5FA0146484656
:105CD00006F0D8F930B13046FEF7BDFA014640462D
:105CE00006F002F86846FAF73DFA2835E1E7D4E90C
:105CF00006892E4AA9EB0807FD1055430135B5F575
:105D0000705F02D92A4805F0DBF8236AA3EB080389
:105D1000DB1053439D4220D94FF0280A0AFB05FAB5
:105D20001DB1504606F07CF80546494640462A46D5
:105D3000FFF744FFD4E90689C14505D04046FAF78C
:105D400011FA08F12808F7E7A06908B1FFF7D8FAB7
:105D50002F44A5615544E7612562226AD4E9060310
:105D600012491B1ADB10121A4B43D2104A4301335B
:105D7000934206D90F4805F0B7FF77210E48FEF78A
:105D8000BDF9D4E90703984209D010B13146FFF7B5
:105D9000E2FDE3692833E3610AB0BDE8F08701461C
:105DA000324604F11800FFF729FFF5E7CDCCCCCC43
:105DB000E3B70108A5BD0108FCBC010873BD0108DB
:105DC000002313B502A941F8043D094B0422D3E98D
:105DD0000140084B20445B689847044628B10648B8
:105DE00005F082FF204602B010BD0448F8E700BF6E
:105DF000144800200448002014C1010828C10108EB
:105E000008B5084805F070FFFFF7A4FEFFF798FA01
:105E1000054805F069FFFFF79DFEBDE80840FFF764
:105E2000A5BA00BF45C101085DC1010873B50546AB
:105E30004FF416700C4605F0F3FF064630B92148C2
:105E400005F052FF22212048FEF758F94FF4167250
:105E50000021304612F023F8314628464FF41672DE
:105E6000FFF7E0FA194D014601902CB3184805F0F0
:105E70003BFFD5E901431C44164DEB681BB101996A
:105E80002046083198476B680422104920469847FD
:105E900004226B680DEB0201A01898476B68019A09
:105EA000314604F1080098470B4805F01DFF3046C5
:105EB00005F0A0FF02B070BD084805F015FF6C6842
:105EC000DAE700BF88E20108B6BF010814480020E5
:105ED00006C001080448002040C0010825C0010890
:105EE0002DE9F74FFFF736FE2F4F06462F4805F0F6
:105EF000FBFEB846DFF8D090DFF8D0A0FCF798FDA5
:105F00002B4D38602B68AB462A4C002B37D003F55D
:105F10006A436033984232D223782BB9264805F081
:105F2000E3FE264805F0E0FE012330462370FFF72C
:105F3000D3FB41F2883352464FF0FF310020FDF78A
:105F400045FA0190FCF774FD019BC8F8000023B9E5
:105F5000237813B13046FFF7BFFBDAF80030DA07D9
:105F600044BFD8F800202A609B07C7D50023CBF890
:105F70000030D9F80830002BBED09847BCE7237812
:105F80006BB100213046FFF751FF0D4805F0ACFE24
:105F90000C4805F0A9FED9F8083003B19847002352
:105FA00023702B60C5E700BF2C48002084C0010887
:105FB000284800202048002099C00108BCC00108E2
:105FC000DFC00108F1C00108044800202448002077
:105FD00010B5FFF7BFFD04460021FFF727FF20465D
:105FE000FFF7C4F9BDE81040034800230122022155
:105FF0000068FDF72FBA00BF0048002010B5FFF77A
:10600000A9FD04460021FFF711FF2046BDE810401E
:10601000FFF7ACB92DE9F743194E07468846756876
:106020000AB1B3681D440024DFF8609002A941F86A
:10603000084D0422D9F80030284698473268009964
:106040008A4204D00F4805F04FFE204614E0042297
:10605000D9F800300DEB0201A818984701990A48B9
:1060600005F042FE019A4245EFD8D9F80030394692
:1060700005F108009847019803B0BDE8F08300BF20
:10608000144800204FC001086AC0010804480020DD
:10609000F0B589B002AC84E80F00039B23B940F24D
:1060A00029117D48FEF72AF8029B23B94FF4957118
:1060B0007948FEF723F894E80F00784D784C85E88E
:1060C0000F000EAB93E8070084E8070012B94FF405
:1060D0008063A360236823B940F235116E48FEF750
:1060E0000DF82368013304D140F237116A48FEF7F6
:1060F00005F8FFF72FFD06466A4B6B4A6B49FFF721
:1061000091FC6B4B6B4A6C493046FFF78BFC6B4B39
:106110006B4A6C493046FFF785FC4FF4167005F06A
:106120007FFE074680B9684805F0DEFD674805F048
:10613000DBFD3046FFF704F900233370FFF740FE24
:10614000634805F0D1FD2CE04FF41672002111F0E8
:10615000A6FED4E901032D68042207A91844A84724
:1061600000285ED02268079B9A425AD1594805F010
:10617000BBFD01224FF416713846FFF74BFF044672
:10618000554805F0B1FDFFF71BFE002C45D001235B
:106190003370224639463046FFF7E2FA384605F0BA
:1061A00029FE33783BBB4FF4167005F039FE0446E8
:1061B00030B9454805F098FD7F213748FDF79EFF2F
:1061C0004FF416720021204611F069FE00224FF4B0
:1061D00016712046FFF71EFF074678BB05F00AFE42
:1061E000204605F007FE3D4805F07EFDFFF7B2FCB6
:1061F0000021FFF71BFE3A4BFA2201930123394994
:10620000009339480023FCF7F1F920B94FF4A87145
:106210002148FDF773FF09B0F0BD344805F064FD77
:10622000347000224FF416713846FFF7F3FE04462F
:106230000028AED1384605F0DDFD77E74FF4167043
:1062400005F0EEFD054630B91F4805F04DFD8E21E5
:106250001148FDF753FF4FF416720021284611F044
:106260001EFE4FF4167229463046FFF7DBF808B9D8
:106270002846B3E78742FBD10023E95CE25C914208
:10628000F6D101339F42F8D1284605F0B3FD2046F0
:1062900005F0B0FDAFE700BFB6BF0108044800201D
:1062A00014480020FD5F0008BDBE0108C9BE0108FA
:1062B000015E0008CEBE0108E9BE0108D15F0008FA
:1062C000F1BE010809BF010888E2010870BF01089A
:1062D0005DC101080EBF010832BF010894BF01086B
:1062E00000480020ABBF0108E15E000847BF01087D
:1062F00010B504460168074805F0F6FC616831B145
:106300000B7823B10448BDE8104005F0EDBC03480C
:10631000F9E700BF75C10108A1B801086EBC01080A
:1063200010B50446C06908B105F064FD206908B1E4
:1063300005F060FD606808B105F05CFD204610BD09
:1063400010B504460068FCF771F8204610BD000047
:106350001FB50B46546801780294127801925A686E
:10636000009242681B68024805F0BEFC04B010BDF4
:106370007AC10108CB210148FDF7C0BE98C10108D0
:10638000FE2307B502A901F8043D054B1868002358
:1063900000681A46FBF73AFD03B05DF804FB00BF46
:1063A0003C480020D0B51F467423C0E900310023CB
:1063B000044683600820164604F0A0FDC0E900678B
:1063C000A0602046D0BD00002DE9D043DDE906677E
:1063D00099467223C0E9003100239642836077EB2F
:1063E00009030446904603DA2B210748FDF786FE91
:1063F000102004F083FDC0E90089C0E90267A060B5
:106400002046BDE8D08300BFE2C10108036837B56C
:10641000632B04460D4601D0FFF7ACFF002302AA10
:1064200042F8043DA168284605F044FA019B1BB1DF
:1064300038210248FDF762FE03B030BDE2C1010819
:1064400070B563230025C0E90031044685601A2039
:10645000164604F053FD1A22294611F020FD31465C
:10646000A0602046FFF7D2FF204670BD81647047D0
:10647000C16470472DE9F843D0E9017388460025CF
:106480004FF00C09DB1B0A4E9B105E43ECB2B4428A
:106490000BD209FB04724146506812F0C3FB013570
:1064A0000028F3D12046BDE8F8834FF0FF30FAE72B
:1064B000ABAAAAAA2DE9F843D0E9047388460025BF
:1064C0004FF00C09DB1B0A4E9B105E43ECB2B4424A
:1064D0000BD209FB04724146506812F0A3FB013550
:1064E0000028F3D12046BDE8F8834FF0FF30FAE7EB
:1064F000ABAAAAAA2DE9F0410E4649680446FFF767
:10650000B9FFC0B2FF2803D07C212948FDF7F6FD72
:10651000D4E90123274F9B1A9B107B437E2B03D981
:106520007F212348FDF7EAFDD4E901120C25E0683C
:10653000531A9B10121A7B4392107A4301339342F1
:1065400005FB03F80ED84144A160D4E9013496E874
:106550000700E31A04E9070016489B105843013866
:10656000BDE8F081404605F05BFC054618B969219D
:106570001148FDF7C3FDD4E901C30027A3EB0C03C9
:106580009A100C4B5343002B09DD05EB070E0CEB67
:10659000070207CA013B8EE807000C37F3E76046A5
:1065A00005F028FC65604544C4E90255CDE700BF0D
:1065B000E2C10108ABAAAAAAC3B401081FB56E23A1
:1065C000CDE90131002301A90393FFF793FF05B043
:1065D0005DF804FBFF2270B5002380F828204FF0FF
:1065E00000424FF0FF31C0E90D23C2636FF07F42DC
:1065F000C0E910120522C0E90033C0E91423C0E944
:1066000002330022C0E90433C0E90633C0E908338D
:106610000363C0E9123383654FF000431E4DC0E9A8
:1066200018232A68044612F0010213D101211B4EDF
:10663000084632607160FBF70FFB306018B95021DB
:106640001748FDF75BFD0123164A174913482B60D5
:106650000FF0B5FF154B1A680AB9104A1A601449B1
:106660002046FFF7ABFF134B134918702046FFF786
:10667000A5FF124B124918702046FFF79FFF114BE0
:10668000114918702046FFF799FFFE220F4B187032
:106690000F4B20461A7070BD38480020C0480020BB
:1066A000ECAB010800000020416300083C480020DA
:1066B00024C30108444800202CC30108424800209C
:1066C00034C301084048002039C301084348002072
:1066D0004148002010B5084C2368DB0709D407485F
:1066E000FFF778FF0123064A0649044823600FF0AC
:1066F00066FF024810BD00BF344800205848002003
:1067000000000020216300082DE9F0410E46496891
:106710000446FFF7CFFEC0B2FF2803D087212948E7
:10672000FDF7ECFCD4E90423274F9B1A9B107B4315
:106730007E2B03D98A212348FDF7E0FCD4E904121B
:106740000C25A069531A9B10121A7B4392107A43AE
:106750000133934205FB03F80ED841446161D4E94B
:10676000043496E80700E31A04E9070016489B1072
:1067700058430138BDE8F081404605F051FB05461D
:1067800018B969211148FDF7B9FCD4E904C3002701
:10679000A3EB0C039A100C4B5343002B09DD05EBC4
:1067A000070E0CEB070207CA013B8EE807000C3707
:1067B000F3E7604605F01EFB25614544C4E9055535
:1067C000CDE700BFE2C10108ABAAAAAAC3B4010881
:1067D00038B5D0E901239B1A074A9B105343CDB229
:1067E0009D42044603D3A6210448FDF787FC0C20F4
:1067F000636800FB053038BDABAAAAAAE2C1010854
:1068000038B5CCB2114905460B6813F0010307D126
:106810000F4A70201372012310600E480B60506005
:10682000FF2C10D0D5E904239B1A0B4A9B1053432D
:106830009C4203D3B2210948FDF760FC0C23286970
:1068400003FB040038BD0248FCE700BF30480020CD
:10685000484800202CC20108ABAAAAAAE2C101083C
:1068600010B5D0E90730C9B2D2B2834209D01C7842
:106870008C4204D15C78944201D1987810BD0333E6
:10688000F3E74FF0FF30F9E72DE9F041D0E90423B9
:106890009B1A4F4A9B1053430D4609780446994270
:1068A00003D393214B48FDF729FCD4E901239B1A1C
:1068B000474A9B1053436978994203D39421454832
:1068C000FDF71CFCD4E904239B1A414A9B10534357
:1068D000A978994205D3FE2903D095213D48FDF7BB
:1068E0000DFC6A7829782046FFF7BAFFC3B2FF2B68
:1068F000064629D029782046FFF782FF69780746A7
:106900002046FFF765FF314680462046FFF778FFB7
:10691000414602463846FFF71BFD29782046FFF71F
:106920006FFF697806462046FFF752FFA9780746B1
:106930002046FFF765FF394602463046FFF708FD5F
:106940009C212448FDF7DAFBD4E90723204F9B1A4A
:106950007B437E2B03D99F211E48FDF7CFFBD4E953
:106960000762616A931B7B43521A57430133BB4250
:1069700003EB43080AD8464426622A88236A23F890
:10698000032CAA7803F8012CBDE8F081404605F0FD
:1069900047FA064618B969210F48FDF7AFFBD4E95D
:1069A0000702131A0A4A5A430023002A0ADDC118B3
:1069B000B1F800C0F71826F803C08978013AB97019
:1069C0000333F2E705F016FAE66146446662D3E760
:1069D000ABAAAAAAE2C10108C3B4010813B5FF24F7
:1069E000084A02AB106803F8044D0A4600681946CD
:1069F000FBF7B0FA012814BF20469DF8040002B04E
:106A000010BD00BF3C48002038B5816800681D46B5
:106A1000144605F0E9FA0346201845EBE37138BD4A
:106A200008682DE9F04172281F461FD074280FD046
:106A3000632820D1886804F0FDFF002871F100036D
:106A400004460D460EDADD210D48FDF757FB09E03F
:106A50008B68D3E90045B5F1004F08BF002C01D089
:106A6000A4187D4120462946BDE8F0818868BDE82C
:106A7000F041FFF7C9BF00244FF00045F2E700BF27
:106A8000E2C101082DE9F0410F4606460024FFB29D
:106A9000FFF7B6FED6E90758454511D02B78BB4223
:106AA0000CD169783046FFF793FE0368692B05D156
:106AB00083681B6803B198470134E4B20335EBE700
:106AC0002046BDE8F0812DE9F34180460F460025C0
:106AD000FFF796FED8F81C40D8F820600334033640
:106AE000FFB2A6421BD0234633F8032D9B78ADF8A6
:106AF00004208DF8063014F8033C9F420DD19DF818
:106B000005104046FFF764FE0368692B05D18368D2
:106B10005B6803B198470135EDB20334E1E72846DD
:106B200002B0BDE8F0810000836C73B504460D46E9
:106B3000164623B94FF48C710B48FDF7DFFACDE907
:106B4000006423462A4609490948FBF74FFD0128FE
:106B500007D04FF48F71044802B0BDE87040FDF7D4
:106B6000CDBA02B070BD00BFE2C1010806C3010882
:106B7000A171000838B590F847300446032B0D4644
:106B800004D940F231110648FDF7B8FA94F84730BD
:106B90005A1C84F847201C4484F8425038BD00BF7A
:106BA000E2C1010810B590F84730044623B94FF40C
:106BB0009B710648FDF7A2FA94F84730013BDBB21F
:106BC00084F847301C4494F8420010BDE2C101082B
:106BD000CBB2FE2B10B504460AD0FFF711FE0368B6
:106BE0006D2B05D1017A2046BDE81040FFF708BEA5
:106BF00010BD00002DE9F84304460026114FD4E9EA
:106C000004239B1A9B107B435FFA86F8434516D9F1
:106C100041462046FFF7DCFFD4E90759A9450CD0CF
:106C20002B78434507D169782046FFF7D1FDA97835
:106C30002046FFF7CDFF0335F0E70136DFE7BDE87B
:106C4000F88300BFABAAAAAA38B50546002495F878
:106C50004730A34207DD2B1993F842102846FFF76F
:106C6000CFFD0134F3E738BD00232DE9F74FC0E92C
:106C7000083388461946D8E907594FF000430446BF
:106C8000C0E90613C0E90013C0E90213C0E9041308
:106C9000FF208A469B46D2B284F8200001924D45DF
:106CA000D4E9006720D02B78019A93421AD16978F1
:106CB0004046FFF78DFDDDE90C2301464046FFF716
:106CC000AFFE594508BF50450CD05F4508BF56453B
:106CD00003D0B04271EB070304DA6B78C4E900011A
:106CE00084F820300335DAE7B7F1004F08BF002EF3
:106CF00008D0DDE90C23B21A67EB030316461F46E2
:106D0000C4E90467204603B0BDE8F08FF8B50D462E
:106D10000B4B896906464B434FF47A71B3FBF1F193
:106D2000FFF75CFE0446C7B2B06C03681B68984767
:106D3000FF2FC6E90E010CBF95F820002046F8BDD4
:106D400040420F0038B5C36C04460D461BB9BDE880
:106D50003840FFF7DBBF806C174903685B699847D1
:106D6000A06C0368DB689847D5E9020104F03CFF9A
:106D70000146124804F0B8FFA06C03689968D5E991
:106D800002238847A06C03681B699847E36C984707
:106D9000A06C0368DB689847A06C03681B68984781
:106DA000C4E90E0100212046FFF718FEC0B2FE28FC
:106DB00008BF95F8200038BD8163000811C30108A1
:106DC000F8B5D1E90667B7F1004F08BF002E0546B8
:106DD0000C4608D11AB1BDE8F840FFF797BFBDE8EF
:106DE000F840FFF7AFBF012E77F1000302DA91F808
:106DF0002000F8BD92B121462846FFF787FF94F89E
:106E00002030C0B28342F4D1D5E90E67D4E9002323
:106E1000964277EB0303B8BFFF20EAE7D0E91423DB
:106E2000964277EB0303E6DBFFF78CFFE7E7000012
:106E30002DE9F04F8DB004460D46FFF7E1FC0368E5
:106E40008046702B04D04FF49E716B48FDF756F9C5
:106E5000A06C03681B6898472A46C4E90C01CDE979
:106E60000001214602A8FFF7FFFE29462046FFF752
:106E700009FE9DF828300646FF2B05D120B940F2C7
:106E800047115D48FDF73AF9D4E90C0104F0ACFE76
:106E900001465A4804F028FF3146594804F024FFBF
:106EA0009DF82810FF297ED100224FF00043CDE944
:106EB0000623DDE90223CDE90423DDE90623CDE93C
:106EC0000823A36D13B39847DDE90223D4E9180121
:106ED000B3F1004F08BF002A09D0DDE9062310F105
:106EE0000B0641F10007964277EB03030EDAD4E973
:106EF0000C23161843EB0107CDE90801CDE904671F
:106F000004F088FE01463F4804F0EEFE4FF0000A10
:106F10004FF0004BDFF8F89098F8082002A92046BF
:106F2000FFF74EFFA36D064603B19847F3B2FF2B60
:106F30005AD1DDE90223D4E90E01161A63EB0107E9
:106F400039463046CDE90423CDE90667CDE9086727
:106F500004F060FE0146484604F0C6FEA36D002B17
:106F6000DAD0DDE90223D4E918015B4508BF5245B8
:106F700009D0DDE9062310F10B0641F10007964226
:106F800077EB0303C8DAD4E90E23161843EB0107A5
:106F9000CDE90801CDE9046704F03CFE014619483B
:106FA00004F0A2FEB8E72046FFF712FCD0E9006724
:106FB000DDE9020104F018FE3A4603463146124864
:106FC00004F092FED4E90C23DDE90201801A61EBA2
:106FD00003010F460646CDE9066704F01BFE014695
:106FE0000A4804F081FE64E729462046FFF76BFD5E
:106FF00030460DB0BDE8F08FE2C101083AC2010889
:1070000059C20108B6C2010874C2010898C2010839
:10701000CEC2010870B504460D46FFF7F1FB0368C8
:107020006D2B11D0702B09D0612B14D1836894F88B
:10703000411094F84000BDE87040184729462046AA
:10704000BDE87040FFF7F4BE034840F22B11FDF796
:1070500055F84FF0FF3070BDE2C101082DE9F0474F
:1070600090F828300446FF2B04D14FF4E3714848D0
:10707000FDF744F894F828102046FFF7C1FB94F878
:107080002830DFF8188184F8463094F846102046FE
:10709000FFF7B6FB036805466D2B204694F84610B3
:1070A0000BD1FFF767FD297A204684F84610FFF7D9
:1070B000A7FB2046FFF7C8FDE7E7FFF7ABFFC3B22A
:1070C000FF2B06460BD140F2DB113148FDF716F8D5
:1070D00040F2DB112F4B304A2D4810F069FD02467B
:1070E00094F846102046FFF7BBFBC5B2FF2D09D12F
:1070F00040F2E1112648FDF701F8264B264A40F2FE
:10710000E111E9E794F84610FE2D204621D1FFF762
:1071100049FD074601462046FFF772FB32463946D5
:107120002046FFF79DFBC5B2FF2D0DD1314620460D
:10713000FFF74EFB40F2ED111548FCF7DFFF154B52
:10714000154A40F2ED11C7E72046FFF77DFD3946AD
:10715000DAE7FFF755FB314607462046FFF738FBD5
:10716000294681462046FFF74BFB8246404604F005
:10717000BBFD524649463846FFF7EAF894F84630D8
:1071800084F8416084F8403084F846507DE700BFC1
:10719000E2C1010865B8010841C30108F6C201084F
:1071A00008B5FFF797FAFFF759FFD0B51F46164607
:1071B000FFF70EFB03688468742B01D0FFF7DAF841
:1071C000C4E90067D0BDD0B5044616461F46FFF798
:1071D000FFFA32463B4601462046BDE8D040FFF765
:1071E0001FBC0000836C10B5044623B94FF4267110
:1071F0000248FCF783FFA06C10BD00BFE2C101088C
:10720000FF23054A1370054A1370054A1370054A97
:107210001370054A1370704744480020424800200C
:10722000404800204348002041480020014B187886
:10723000704700BF4048002010B504460068FBF7C7
:10724000F5F8204610BD00002DE9FF4805F0CEFFFF
:107250004FF6FF712E4A2F4C13888B421CBF01330F
:107260001380FFF737FAFFF7BDFF03681B689847E5
:10727000637806460F4603BB274BDB88EBB1274AF2
:10728000D2E900BCBCF1004F08BFBBF1000F0FD02A
:1072900083457CEB010210DA214AB0EB0B0002FBC4
:1072A00003F261EB0C01D317904271EB030304DB93
:1072B0001C4804F019FD012363700023ADF80C3065
:1072C00063782BB101238DF80C30144BC3E90067B0
:1072D0002378154CBBB1012514488DF80D5004F0EE
:1072E00003FD2570124B13481A78134B19780023AD
:1072F00000930068039B06F0BBF830B10F4B187881
:1073000004B0BDE8F0882370ECE70D4BF7E700BF51
:107310000A490020EC480020F848002068000020BE
:107320008051010086C40108F5480020AFC401085F
:10733000EF480020E8480020EE48002040480020A8
:107340004248002008B5164BDB882BB9154804F0DD
:10735000CBFC154B187808BD144BD3E90023B3F1CF
:10736000004F08BF002A01D01148F0E7114B1978EF
:107370000131C9B20129197001D90F48E7E70F4857
:1073800004F0B2FC00230E4A13700E4A13700E4A2A
:1073900013600E4A1370012353700D4BDAE700BFE0
:1073A000F8480020C4C401084048002060000020C4
:1073B000E0C4010820490020FAC4010811C50108F1
:1073C000EF480020EE480020E8480020EC4800206C
:1073D0004348002008B500231A46FAF717FD431E5C
:1073E0005842584108BD000007B50B78012B12D058
:1073F00005D3022B13D00C4804F076FC08E00023E0
:1074000002A941F8043D094B1B681868FFF7E2FF29
:1074100003B05DF804FB02A94FF0FF33F1E7034B23
:1074200004311B68F1E700BF77C50108D848002088
:107430001FB57023CDE90131002301A98DF80C306F
:10744000FFF762F905B05DF804FB00002DE9F04F8D
:107450004A4B85B01A780446002A40F08B800127F9
:1074600047491F70FFF7AAF8464B47491870204656
:10747000FFF7A4F8DFF868A144498AF80000204625
:10748000FFF79CF8DFF85C910A22002389F80000DE
:107490003F4901A8FEF786FF01A92046FFF72AF819
:1074A0003C4E3D4930702046FFF788F83B4B3C4945
:1074B00018702046FFF782F83A4B3B491870204677
:1074C000FFF77CF8394B3A4918702046FFF776F8F9
:1074D000384B394A187039492046F9F747FADFF82E
:1074E00008B1374A8BF8000036492046F9F73EFAD2
:1074F000354905462046FFF79BFF70230193334B28
:10750000804601A9204602938DF80C70FFF7FCF825
:1075100007462F4A2B4612789BF800102046F9F7B1
:1075200030FA43469AF8002029462046F9F729FA0E
:107530003B4699F8002029462046F9F722FA2B46C7
:10754000327841462046F9F71CFA2B463278394604
:107550002046F9F716FA1F4A2B461278294620468C
:10756000F9F70FFA1C4B1D4A1B7812782946204662
:10757000F9F707FA05B0BDE8F08F00BF21490020F8
:10758000CDC60108F0480020D7C60108E2C60108B0
:10759000EEC60108D1480020FBC6010809490020B9
:1075A00009C701080849002015C701080C49002037
:1075B00022C701080D4900204972000830C70108A0
:1075C000D98400083AC701084EC7010861C70108FD
:1075D0004048002043480020414800204448002003
:1075E000F4480020D0480020F248002008B505F0FB
:1075F000DBFD18B1BDE8084005F0F8BD08BD00008E
:1076000030B5044685B00D46FFF720FF6D22064BCE
:1076100001A91B782046CDE901258DF80C30FFF734
:1076200073F805B030BD00BFF24800202DE9F84FD7
:10763000424B434D1A68044612F0010F01BFFF226E
:107640002A7001221A602B78FF2B73D1FFF7FEFE00
:107650003C4A3D492046F9F789F93C4A28703C49A3
:107660002046F9F783F93B4F3B4A38703B492046A7
:10767000F9F77CF93A4E3B4930702046FFF7C0FFDE
:10768000394982462046FFF7D3FE384983462046D3
:10769000FFF7CEFE8146364A3B781278297820469D
:1076A000F9F76FF9334ADFF8E080337812782978F8
:1076B0002046F9F766F9337898F8002039782046A3
:1076C000F9F75FF92B7898F8002031782046F9F720
:1076D00058F9294A5B46127839782046F9F751F96A
:1076E00026493B780A7820465946F9F74AF9244A50
:1076F0004B46127839782046F9F743F91F493B7811
:107700000A7820464946F9F73CF91A4A5346127856
:1077100031782046F9F735F9337898F8002051464A
:107720002046F9F72EF9174A2B781278317820463F
:10773000F9F727F92878BDE8F88F00BFCC4800207A
:1077400023490020E97E000861C80108ED7900089E
:107750006BC80108F14800204573000875C801088E
:10776000F34800207FC801088BC8010899C80108A8
:10777000F048002043480020F4480020D148002071
:1077800042480020404800204448002038B50446C4
:107790000D46FFF75BFE034A29462046F9F7E6F857
:1077A00038BD00BF6D7C0008344B2DE9F04F1A89BD
:1077B0000023044689B0CDE9002303910023002271
:1077C0002F4905A8FEF700FE05A92046FEF792FE08
:1077D0002C4982462046FFF72BFE2B498346204644
:1077E000FFF7D4FF294A804629492046F9F7BEF819
:1077F000284A054628492046F9F7B8F80646274F93
:10780000DFF8A8903B7899F8002029462046F9F740
:10781000B8F8234A5B46294620461278F9F7B1F8B2
:10782000204A4346294620461278F9F7AAF83346FB
:10783000524659462046F9F7A4F833465246414687
:107840002046F9F79EF8184A3B78414620461278C0
:10785000F9F797F83B7899F8002031462046F9F778
:1078600090F86D230593039B05A9204606938DF898
:107870001C50FEF749FF09B0BDE8F08FF848002022
:10788000A8C80108B5C80108C5C8010809800008D2
:10789000D6C801082D720008E5C80108414800203B
:1078A0000C4900200D4900200949002040480020D3
:1078B0002DE9F04F044687B008460E4615469A4615
:1078C00011F0C2F900F106090746484603F032FB01
:1078D0004946334607F107092F4A804611F04EF911
:1078E000484603F027FB0837494633462B4A834670
:1078F00011F044F9384603F01DFB33463946284A57
:10790000814611F03BF9274A41462046F9F72EF807
:10791000594680462046FFF78BFD49468346204660
:10792000FFF734FF8146204A5B46127841462046E5
:10793000F9F727F81D4A4B46127841462046F9F7D9
:1079400020F81B4F1B4A3B78127849462046013DE0
:10795000F9F717F805EB0A030193019B9D420ED03E
:1079600015F801AF3B78524659462046F9F709F819
:107970003B78524649462046F9F703F8EDE76D2378
:1079800003A92046CDE903368DF81480FEF7BCFE2E
:1079900007B0BDE8F08F00BF46C801084EC8010817
:1079A00057C801082D8000080C4900200D4900200F
:1079B000414800200949002013B502AC04F8042D09
:1079C00001232246FFF774FF02B010BD70B50D46CB
:1079D0000446FEF77FFE044922462B46BDE8704070
:1079E0000978FFF7E2BB00BFD1480020F7B5644C2F
:1079F0002668A6B9082003F081FA05460660012032
:107A0000324668600421FAF727F9286018B9502136
:107A10005C48FCF773FB5C48256005F0FDFB5B4DA3
:107A20005B4F29685B480131296004F05DF905F07E
:107A3000DDFB3B781BB901233B7005F003FC002301
:107A400002A941F8043D2368534A1868FAF782FAFC
:107A5000012807D0514804F047F94FF4D971504834
:107A6000FCF74CFB019E731C5DD14E4804F03CF9C1
:107A70002B68042B0FD9FEF787F803785BB14A48CF
:107A800004F032F94FF47A70FBF72AF940F2BD1195
:107A90004348FCF733FB2B681E22013BDBB21E2B55
:107AA00028BF1E230020A3F120040025387002FA0D
:107AB00004F74FF4E144C3F1200122FA01F10F432E
:107AC00002FA03F6BD4208BFB44225D3002F08BF17
:107AD000B6F5616F22D2B6F5167F77F1000320DA92
:107AE0003C2E77F10003ACBF11460A21002004F0C0
:107AF0007BFA341847EBE0752946204604F08AF8F3
:107B000001462A4804F0F0F820462946FFF75EFFB8
:107B1000274B187803B0F0BD26462F464FF4167158
:107B2000E4E73C21E2E74EB13146224804F0DCF8BC
:107B300001980021FFF74AFF1F4BEAE71F482E601C
:107B400004F0D2F805F00CFBFEF7C4FDFFF74AFB8A
:107B500003681B6898471A4BC3E9000123686BB19F
:107B6000304605F059FB256835B12868FAF75EFC08
:107B70000821284603F0E4F900232360114BC8E7ED
:107B8000D8480020ECAB0108E97300081C4900202C
:107B90001849002066C30108A086010079C30108C6
:107BA00093C30108E7C30108FEC301084BC40108E1
:107BB0004248002061C40108F448002076C401084E
:107BC0005800002044480020054B1870054B1A70DF
:107BD0000022054B1960054B1A705A70704700BFA0
:107BE000EF480020EE480020E8480020EC48002044
:107BF000027901684079FFF7E7BF08B505F030FC6E
:107C0000C0B2DE2828BFDE2008BD00004FF47A7322
:107C100037B5002403FB00F2074802A9056841F8C4
:107C2000044DB2FBF3F22868FAF794F9012814BF67
:107C30002046019803B030BDD44800204FF47A7339
:107C400037B5002403FB00F2074802A9056841F894
:107C5000044DB2FBF3F22868FAF7BEFA012814BF0C
:107C60002046019803B030BDD44800202DE9F04FE4
:107C700097B0FEF72FFD4FF00009064690F846B08A
:107C8000FFF7B4FCDFF8C8A0DFF8C880B06C02AD25
:107C900003680CAC1B6898475A46CDE90001314691
:107CA0000CA8FEF7E1FF0FCC0FC50FCC0FC5DDE927
:107CB0000C012368B1F1004F08BF00282B70DDE9EB
:107CC000104516D11C4804F00FF8002501271B4C65
:107CD0004FF47A73A4FB030103FB0511FFF7AEFF1A
:107CE00010B30122164B5A72164B187817B0BDE824
:107CF000F08F03F079FF29460746204603F08AFFFC
:107D000039460246504603F0EFFFA04579EB0503E4
:107D100008DA0021094803F07DFF01460A4803F014
:107D2000E3FFD2E70027D3E71FB1084803F0DCFFE9
:107D3000ACE79DF82800D9E7FFC501088051010094
:107D4000DC4800200949002039C6010852C6010854
:107D500017C601088551010010B500200021FFF76A
:107D60006DFF10B1084B187810BD084C2368984778
:107D700020B9074B1B780BB9064BF4E7637A0BB1BC
:107D8000054BF0E7054BEEE709490020DC480020F1
:107D90000E4900204048002044480020434800206D
:107DA000022818BF002005F0DDBC0000F8B53B4BF1
:107DB00005461E78002E6FD101271F7004F0D2FEF9
:107DC00037492846FDF782FDC31F052B354C42D8A5
:107DD00020710E23344928466371FDF780FD334935
:107DE000074610F01FFF00283AD1E06030492846CE
:107DF000FDF752FD2F4960702846FDF767FDB0F58D
:107E00007A7F3AD8E0802C492846FDF75FFD42F2A0
:107E10001073984236D8208128492846FDF73CFD4A
:107E20002749A0702846FDF751FDB0F57A7F2ED284
:107E3000608124492846FDF72FFDE07036B12248C5
:107E400003F052FF71212148FCF758F9E068BDE8C2
:107E5000F840FFF7A5BF1E4803F046FF3E46B8E7CF
:107E60001C49384610F0DEFE10B90223E360BDE77E
:107E7000194803F039FF0126B8E7184803F034FF2A
:107E80000126C0E7164803F02FFF0126C4E7154876
:107E900003F02AFF0126CCE7F8BD00BF22490020ED
:107EA00075C70108F84800208EC7010831C80108CD
:107EB000B1C70108B5C70108DCC701084BBB010801
:107EC00004C801082EC8010833C8010893C301087B
:107ED00078C70108A6E0010895C70108BEC70108D8
:107EE000E5C701080FC8010870B5234BC0B21B7865
:107EF000984206D1FDF748FEFDF7FAFC1F4B1878B3
:107F000070BD1F4DFDF740FEFFF750FF95F90500CE
:107F100007F016F805F04AFB287906F0DFFF05F0B8
:107F200039FB687805F018FC164B1A681C4612F0ED
:107F3000010213D10421144E084632607160F9F732
:107F40008BFE306018B950211048FCF7D7F8012398
:107F50000F4A10490C4823600EF031FB0E4B1A6893
:107F60000AB9094A1A600D4805F002FCEB780BB11A
:107F70000B4BC4E70B4BC2E7F348002044480020FA
:107F8000F8480020C848002010490020ECAB010848
:107F90000000002039720008D44800205D840008E9
:107FA000F048002043480020034B93F83230022B66
:107FB0000CBF022000207047C000002008B5FFF76A
:107FC000F3FF30B905F0F0F818B9BDE8084005F046
:107FD000C7B8FFF7E9FF022806D105F0E5F818B1A8
:107FE000BDE8084005F002B908BD000008B5FFF77C
:107FF000DBFF02280CBF024B024B187808BD00BF04
:108000000D4900200C490020054B1B8913B9054B75
:1080100018787047044B5B7A002BF8D1FFF7E6BF66
:10802000F848002040480020DC480020FFF7DEBF71
:1080300001232DE9F348394C002000216372FFF73A
:10804000FDFD10B1364B18781AE02368984718B92F
:10805000344B1B78002B3CD005F090FB012871F1CC
:10806000000306460F460EDB2F4803F03DFEFEF7E9
:1080700031FB32463B46217AFFF797F8FFF7B6FF10
:1080800002B0BDE8F08823689847054688B12748C4
:1080900003F02AFE002364680093ADF80430FFF774
:1080A000ACFD01466846A0476846FFF7A1FD204B9E
:1080B000C9E71C4B1B7863B11E4803F015FE1E4B2D
:1080C0001B88022B28D82A4629462846FFF77CFD24
:1080D000EDE71A4D6B89EBB1EB78DBB1FEF7FAFAFD
:1080E000FFF780F803681B6898476B89144A154DA1
:1080F0005A43D5E90067861B61EB0707D317B242E5
:10810000BB4107DA104803F0EFFD40F269310F4838
:10811000FBF7F4FF002363720D4B94E7DC4800206B
:10812000094900200E490020A5C50108B6C501086F
:1081300008490020C8C501080A490020F848002065
:108140008051010058000020DFC5010893C30108D9
:10815000404800202DE9F04F0446574D87B0C5E94F
:108160000023019100230A22544903A8FEF71AF9BB
:1081700003A92046FEF7BEF9514A814628725149AB
:108180002046F8F7F3FB504A054650492046F8F7D9
:10819000EDFB4F4907462046FFF732FA4D498DF86F
:1081A00002002046FFF744F94B498DF803002046B2
:1081B000FFF7ECFA494982462046FFF7F5FA834675
:1081C000474EDFF83881337898F80020394620464A
:1081D000F8F7D7FB434A3378394620461278F8F748
:1081E000D0FB414A5B46394620461278F8F7C9FB76
:1081F0003E492B460A7820463946F8F7C2FB394AF1
:108200002B46594620461278F8F7BBFB337898F88E
:10821000002059462046F8F7B4FB337898F8002040
:1082200029462046F8F7ADFB2E4A337829462046EA
:108230001278F8F7A6FB2E4A9DF802302946204610
:108240001278F8F79EFB29492B460A7820469DF8BC
:108250000210F8F796FB274A9DF80330294620467E
:108260001278F8F78EFB2B464A469DF803102046FD
:10827000F8F787FB204A5346294620461278F8F73C
:1082800080FB2B464A4651462046F8F77AFB337866
:1082900098F8002051462046F8F773FB6D230393AE
:1082A000019B03A9204604938DF81470FEF72CFA65
:1082B00007B0BDE8F08F00BFDC480020F4C801081B
:1082C0003180000804C90108597D000812C901085D
:1082D0001FC90108D7C60108E2C601082BC9010859
:1082E00041480020404800204348002044480020E6
:1082F000084900200C4900200D49002009490020B0
:10830000F8B51D4600234171BDF8181004460360FE
:10831000C180174602B115B923712046F8BD07493F
:10832000284602F009FE064610B920712660F4E7DF
:108330002A4639460FF08FFD2571F7E751F60108FF
:1083400010B50446006808B102F0F8FD204610BDE3
:108350007FB5364E0446326822B94FF4F87134487E
:10836000FBF7CCFE002C5ED00022324B1A80D4E901
:108370001C23134320D0304B1D68FAF759FB0146EC
:108380002E48A847D4E91C0103F02EFC226F0146B9
:108390002B4803F0A9FCD4E91C232A49C1E9002396
:1083A0002949C1E90023FEF795F9FEF71BFF036891
:1083B0005968D4E91C238847FEF78CF9FEF712FFB1
:1083C00003681B689847214B214AC3E90001237ABF
:1083D000C3F3C0031370637F2BB3237F1BB31D490B
:1083E000082002F09DFD054630B16289237F617F40
:1083F0000092A26EFFF784FF0395A5B100233068B9
:108400001A4603A90068F9F74BFC01280BD0124863
:1084100003F06AFC039C34B12046FFF791FF08216A
:10842000204602F08DFD04B070BD00BFD44800208E
:1084300093C301080A490020C000002068C6010853
:1084400075C6010860000020680000205800002068
:108450000E49002051F60108A2C6010810B50446D5
:10846000FFF776FF24B12046BDE8104007F0D2B8F0
:1084700010BD000038B542F2107004F0D3FE04467F
:10848000124803F031FCECB12578022D16D160685A
:108490000021FFF79BFAD4F89800FFF759FF237AE1
:1084A0002BB10B4803F020FC00220A4B1A70204627
:1084B00005F00CFE032D06D1284638BD032DEAD168
:1084C0000020E5E70125FFF779FDF5E72CC5010858
:1084D0004AC50108F5480020002310B5144C84F863
:1084E000363004F061FE08B104F080FEFFF7C2FFF1
:1084F000032815D8DFE800F005020A080D4803F04C
:10850000F3FB0D4B187810BD0C4BFBE7FFF74CFD50
:10851000022809BF01230A4B84F83630094BF1E7E2
:10852000094840F2DA21FBF7E9FD4FF0FF30EAE7B6
:10853000C00000205DC501084448002043480020D9
:10854000F4480020D048002093C30108FF230021F5
:108550000D4A13700D4A13700D4A13700D4A1370B3
:108560000D4A13700D4A13700D4A13700D4A1370A3
:108570000D4A13700D4A13700D4A13700D4AC2E96B
:1085800000111372704700BFF2480020F14800202C
:10859000F348002009490020084900200D49002027
:1085A0000C490020F0480020F4480020D04800206A
:1085B000D1480020DC48002010B504460068F9F7D7
:1085C00035FF204610BD00002DE9F843054616464C
:1085D0000446DFF838900C4F00EB01084445A4EB4B
:1085E00005020FD046B13AB1B2FBF6F306FB1323F6
:1085F00013B9484603F078FB14F8011B384603F022
:1086000073FBEBE7BDE8F88371AB01083FE00108BD
:1086100013B50B4B02AC04F8010D1868002321467A
:108620001A460068F9F7F2FB064B186828B10023D8
:1086300021461A460068F9F7E9FB02B010BD00BFF9
:10864000284900202C490020C0F3C70342071CBF63
:108650000133DBB218467047052910B501D8002058
:1086600012E04378013B032BF9D8DFE803F00E0E4C
:1086700002020024043003F04AFC44B1FFF7E4FF97
:1086800080B2FA28EBD8C0B210BD0124F2E7400056
:10869000F6E700001B4B70B5036000234FF4165241
:1086A000C0E9023103714E230821C0E904230A23E3
:1086B000C0E9061301210E23134D04462A6880F8F1
:1086C00020300A4080F8211080F8221013D14FF496
:1086D00080700E4E32607060F9F7BEFA306018B9E3
:1086E00050210B48FBF70AFD01230A4A0A490748B3
:1086F0002B600DF064FF094B1A680AB9034A1A602F
:10870000204670BD000100022449002030490020AD
:10871000ECAB010800000020B985000828490020C2
:108720000246C068036819B11B6802F110011847BE
:108730005B6818472DE9F3471C469DF8285006460C
:108740008DF807108DF806200DF1070101224FF674
:10875000FF7002F0F7FB01220DF1060102F0F2FBBF
:108760002A46214602F0EEFB81464FEA202A9DF878
:108770000620C7B29DF807101B4803F0B5FA29463A
:108780001A4803F0B1FA294601222046FFF71CFFE0
:10879000174803F0A9FA52464B463946154803F0EC
:1087A000A3FAF0689DF807100368013C9B6898479E
:1087B000F0689DF8061003685FFA8AF89B6898478E
:1087C0002544F068A54203689B6803D014F8011F94
:1087D0009847F6E739469847F068414603689B6832
:1087E000984702B0BDE8F08796C90108C1C90108E1
:1087F0006EBC0108DCC901080B4670B505460A11BC
:10880000D1B2092A03F00F03C068D4BF3031373129
:10881000092B94BF03F1300403F1370403689B680C
:108820009847E8682146BDE8704003689B68184790
:108830002DE9F047064690461C4689469DF8207073
:108840001144C9B21A1BD2B2974204D913F8012BB2
:108850001144C9B2F6E749424246CDB21D484946E5
:1088600003F042FA39461C4803F03EFA0122394629
:108870002046FFF7A9FE194803F036FA29461848A2
:1088800003F032FAF0683A210368013C9B6898478C
:1088900049463046FFF7B0FF41463046FFF7ACFF90
:1088A0002744BC4205D014F8011F3046FFF7A4FF4F
:1088B000F7E729463046FFF79FFFF0680D21036870
:1088C0009B689847F0680A21BDE8F04703689B68F9
:1088D000184700BF96C90108C1C901086EBC01084C
:1088E000F7C9010830B485689DF808401DB1012D15
:1088F00005D030BC7047029430BCFFF71BBF029418
:1089000030BCFFF795BF00002DE9F04F85B09046D1
:108910006A4600AF7B600388464C0733DB08A2EB56
:10892000C3039D4605468A466E46A3462368002239
:1089300007F10F011868F9F70DFB0128F6D0E86878
:108940003D49036800245B699847FAF771F84FF4D2
:108950007A7300F57A79DBF800001A4607F10F0107
:1089600000683B60F9F7F6FA01280AD1621C92B25E
:10897000F97B012A31551DD029883B6891421BD8CB
:1089800014463CB3317851451AD1E8680021036898
:108990005B6998472146294803F0A6F90022214641
:1089A0003046FFF711FE264803F09EF9032C1FD82E
:1089B000244815E04FF47A731446CCE70022FBE715
:1089C000214803F091F9FAF733F8A9EB0003B3F566
:1089D0007A7FF3D9E868002103685B6998471B48F0
:1089E00003F082F9002420461437BD46BDE8F08F1D
:1089F000331913F8012C13F8025C023C05EB022535
:108A00003146A2B24FF6FF7002F09CFAADB2854239
:108A1000014604D02A460E4803F066F9E2E77B6877
:108A2000E4B29C4228BF1C463146224640460FF025
:108A300012FAD8E7284900201186000806CA010862
:108A40006EBC010869CA010824CA010852CA01089B
:108A5000A2CA01082DE9F04F85B016466A4698462D
:108A6000438800AF0733DB08A2EBC3039D466C4C81
:108A7000824689466D46A3462368002207F10F010E
:108A80001868F9F767FA0128F6D0DAF80C0065499A
:108A900003685B6998470023DBF8000041F28832E5
:108AA00007F10F0100687B60F9F754FA01287B6831
:108AB00026D1FA7B5C1CA4B202F07F02012CFA736F
:108AC000EA5408D92B1913F8022C0D2A03D113F8F4
:108AD000013C0A2B03D0BAF80230A3420ED8DAF8D0
:108AE0000C00002103685B6998475CB94E4803F0AD
:108AF000FBF820461437BD46BDE8F08F2346CBE790
:108B00001C46ECE7082C10D8484803F0EDF8214645
:108B1000474803F0E9F8284601222146FFF754FDB3
:108B2000444803F0E1F80024E3E72B783A2B08D11E
:108B30002B1913F8022C0D2A03D113F8013C0A2B30
:108B400001D03D48E1E72946E31E9BB211F8012F11
:108B5000A2F13000162802D83A3A062A01D837483E
:108B6000D3E74A1B92B29342F0D8DA0705D53448CE
:108B700003F0BAF821463348CBE728462C46C3F326
:108B80004703621BD2B2934223D94178A1F130024C
:108B9000D2B2092A07D9A1F14102052A8EBF0022CB
:108BA000A1F13702D2B290F802C01201ACF130014B
:108BB000C9B20929D2B207D9ACF1410105298EBF4A
:108BC0000021ACF13701C9B20A4304F8012B02308D
:108BD000D7E700221146581ED4B2844202F10102A6
:108BE00003DA2C5D2144C9B2F6E749422A5CC9B2D6
:108BF000914203D0144803F077F894E72A784A4565
:108C000002D00A461148F6E7013BDCB2444528BFD2
:108C100044462946224630460FF01DF969E700BF59
:108C2000284900201186000852CA0108E5CA010837
:108C300006CA01086EBC01081ECB01083ACB010828
:108C400084CB0108B3CB0108D2CB010815CC0108B5
:108C50002DE9F0411F46104B04461B680D46164691
:108C600023B94FF4F5710D48FBF748FAA3681BB11F
:108C7000012B09D0BDE8F0813B463246294620460B
:108C8000BDE8F041FFF740BE3B463246294620464C
:108C9000BDE8F041FFF7DEBE2849002049C90108C0
:108CA0002DE9F34704460D4690469946C0689DF865
:108CB00028A0036801211B6A0B9E9DF8307098471D
:108CC00042464B4629462046CDF800A0FFF70AFE53
:108CD000E068002103681B6A98473B4632462946F4
:108CE000204602B0BDE8F047FFF7B2BF2DE9F04FD4
:108CF00082460C469046002687B01D46931EDBB286
:108D00009DF840709DF84490DFF854B00593B1454C
:108D100021DD01364A463146584602F0E5FF059B03
:108D2000627800932178CDE90157A31C5046FFF7E4
:108D3000B7FF0028EBD007B0BDE8F08FB8F1010F06
:108D40000BD9237803202B70637863F07F036B705B
:108D50000B23AB70EFE7022FF0D80020EBE700BF4A
:108D600036C9010810B50446C068002103681B6AB3
:108D70009847E06802490368BDE810405B691847FE
:108D800011860008034A0260002202710274C0E9E1
:108D90000222704754CC010870B50646084802F01C
:108DA000A3FF002406F108053379A34206DD55F838
:108DB000040B013403689B689847F5E770BD00BF5A
:108DC00068CC010870B50646002400F10805337927
:108DD000A34206DD55F8040B01340368DB689847AD
:108DE000F5E770BD38B5047900F1080500EB84049F
:108DF0000834AC4205D054F8040D03685B69984709
:108E0000F7E738BD70B50646002400F10805337950
:108E1000A34206DD55F8040B013403681B6998472B
:108E2000F5E770BD38B503790446012B0D4603D92B
:108E30005B210748FBF762F96968064802F054FFB6
:108E400023795A1C0233227144F8235038BD00BFE5
:108E500080CC0108C3CC010870B504460D460368F8
:108E60000121DB6898472368294620461B699847FB
:108E700023682046BDE87040DB6800211847806900
:108E800070474069704738B5036804461B699847C6
:108E90000546236820469B699847284638BD836865
:108EA000C0E90333002383617047000038B5002513
:108EB000094B0446C0E900310B68C0E90355C0E91D
:108EC00005551B6808469847A5606061C4E90355CD
:108ED000A561204638BD00BF34CD0108D0E903327A
:108EE000934291BFD01A40698018C01A70470000A1
:108EF00038B505460C46FFF7F1FF884203D213212F
:108F00000648FBF7FBF8E9686A69AB68214413443B
:108F10009942E96024BF891AE96038BDDACC0108BA
:108F200008B50146FFF7DAFF4B69181A08BD0000C3
:108F30002DE9F04702EB030899464369044698453A
:108F40000E46174603D93C211C48FBF7D7F8636946
:108F5000A56860681D4423690121ED1A03681B6937
:108F60009847A84560680DD80368E1685D68324697
:108F70003B464944A84760680021BDE8F0470368C4
:108F80001B6918470368A945D3F804800FD2E1682C
:108F9000A5EB09052B4632464944C0476068A168E5
:108FA00003687219D3F804807B1BC047E3E7A1680C
:108FB0003B4649443246491BF7E700BFDACC01087B
:108FC00007B5042200230DEB0201FFF7B1FF019862
:108FD00003B05DF804FBF8B5064617460D4679B1B7
:108FE00084695CB1FFF7ECFF87423C4628BF04462A
:108FF0000423224629463046FFF79AFF2046F8BD53
:109000000C46FBE783690BB1FFF7DABF18467047E0
:1090100038B5836904466BB1FFF7D2FF05460421DA
:109020002046FFF765FF29462046FFF761FFA36949
:10903000013BA36138BD000038B5436905468B424A
:109040000C4603D25F210748FBF758F829696A6983
:10905000AB68214413449942296124BF891A2961CC
:1090600038BD00BFDACC01082DE9F04116461D4A93
:10907000044613680F4633441360FFF751FFB042B4
:1090800003D22B211848FBF739F86369A56860689B
:109090001D4423690121ED1A03681B699847606824
:1090A000AE4203680FD89D683A4633462169A84707
:1090B0006068002103681B69984731462046BDE877
:1090C000F041FFF7B9BFD3F808803A462B46216933
:1090D000C04760687A190368A168D3F80880731BD9
:1090E000C047E5E738490020DACC010807B502ABF4
:1090F00043F8041D04221946FFF7B6FF03B05DF8DC
:1091000004FB70B5144605460E46FFF709FF231D04
:1091100098420DD321462846FFF7E8FF2246314604
:109120002846FFF7A1FFAB690133AB61204670BD54
:109130000024FBE738B50A4C05460121204607F01C
:109140008DFE002320461A46012107F0C5FD85F05B
:1091500001022046BDE83840012107F08BBE00BF68
:109160000000024008B50120FFF7E4FFBDE8084019
:10917000032008F033BE0846FFF7DCBF10B50446F5
:10918000024B036002F086FF204610BD5CCD010853
:1091900010B50446054B503040F8503C044B40F8A5
:1091A000083CFFF7EBFF204610BD00BF50D101087F
:1091B000DCD3010810B50446FFF7E0FF2046082184
:1091C00001F0BEFE204610BD10B50446FFF7E0FFDB
:1091D0002046782101F0B4FE204610BD024B01214B
:1091E000186803681B68184748490020021C18BF0C
:1091F00001220321014807F03DBE00BF00040240E8
:1092000010B50C46F9F7D4FF022808D14FF47A7054
:109210004443B4FBF0F0BDE81040F9F761BD2046CF
:10922000BDE8104007F074BB0321014807F02BBED6
:109230000004024010B5094C094802F055FD2046D3
:109240000B2107F00BFE002320461A460B2107F0E6
:1092500043FDBDE8104007F041BB00BF00000240E5
:10926000ECD0010808B5022007F09CFA07F0FEFADE
:1092700000F076FC07F024FB00F062FE08F088F8AE
:109280000C48FAF705FF4FF4E13008F003FC0A4BF5
:109290001A680AB9094A1A60094B1A680AB9074AD2
:1092A0001A60084802F020FDBDE80840064802F0B8
:1092B0001BBD00BF65910008284A00203519010830
:1092C0002C4A0020CCCD0108E4CD01082DE9F3475C
:1092D000044626464FF01B09FFF754FD284B04F1C6
:1092E000210846F8113B1022002130460EF0D7FD30
:1092F0004A46002140460EF0D2FD00252146214B72
:10930000C4E90F5504F1480041F8443F01F07EF8EC
:109310001D4B1E4FA3651E4B84F85C5023661D4BEE
:10932000C4E91A5563661C4B84F8705063671B4888
:1093300002F0DAFC3B68DFF870A00193DAF8003045
:10934000174D00932B68174A494640460FF016FC0C
:109350002968304602F006FEDAF8001004F1150024
:1093600002F000FE396804F1190002F0FBFD2968E3
:1093700004F11D0002F0F6FD204602B0BDE8F087C2
:1093800050D1010844D20108E0D201086400F81F5E
:1093900038D30108FCD201087CD2010820D1010891
:1093A0005000F81F35D101085400F81F10B5094CC2
:1093B000FFF758FF2368DB0709D40748FFF786FF4C
:1093C0000123064A0649044823600DF0F8F80248D4
:1093D00010BD00BF404900204C4900200000002083
:1093E0009191000838B5064D064C2B6813F0010F1B
:1093F00004D1FFF7DBFF012320602B60206838BD1C
:1094000044490020C44900204FF4FA71FFF724BDFD
:1094100008B50B21054807F03BFD28B1BDE8084021
:109420000B21024807F048BD08BD00BF0000024004
:1094300008B519B1BDE80840FFF7FCBE044802F0CA
:1094400053FCBDE8084002220B21024807F082BC11
:1094500008D1010800000240F8B50446384804F17C
:10946000440502F041FC2846002100F091FD002156
:10947000284600F0A3FD334D2046FFF7B3FC03F070
:109480006FFE20460021FFF7D3FF0BF0A7FE0CF084
:10949000CBF901220C21284607F05CFC08F0A8F863
:1094A00004F1480000F094FF23682046DB6804F1D3
:1094B000640600219847244F0021304600F082FEC8
:1094C00007F058FD214802F00FFC08F0BFF907F043
:1094D000F7F9384601220D2107F03CFC01223846FD
:1094E0000E2107F037FC0021084608F02DF804F1A2
:1094F000580000F0F7FD0121304600F063FE4FF404
:10950000E13008F0C7FA124802F0EEFB28460C21C1
:1095100007F0A4FC002328461A460C2107F0DCFBC8
:109520000120002108F088F80CF090F90BF07CFD88
:1095300008F05CF82046BDE8F840FFF763BC00BFC8
:10954000BAD001080004024000000240DED0010849
:10955000C0B6010838B50546FFF75AFF044628B1E2
:1095600000212846FFF764FF07F0B8F907F084F8F8
:1095700005460CB1FFF75EFE284638BD70B50C46B7
:109580000646154920460EF009F920B9002120466B
:109590000EF0E6F870B1114920460DF043FF0EF0D1
:1095A00007F901460E4802F09FFB40F27F110D487B
:1095B000FAF7A4FD3046FFF72BFF054648B93046C1
:1095C000FFF7C8FF014620460EF0E8F808B1FFF7A4
:1095D00031FE284670BD00BF3333534000007A444B
:1095E000FACD010829CE010870B52D4AD6B013680E
:1095F0000546DB0705D42B4900F164030B6001230A
:10960000136029492846FFF7B9FF0646274802F0AC
:109610006BFB002105F1440000F0D0FC244C254BED
:10962000E360254B2361254BA360254B6360254BED
:109630002360254B6361254BA361254BE36104F156
:1096400010030FCB8DE80F0094E80F000CF028FBFF
:10965000002305A8EB632B640CF0AEFA9DF81430E0
:1096600005F13C04012B14D1DDF8153005A8EB639E
:10967000DDF819302B640CF06FFA164802F034FB59
:109680000821204602F096FBBDF91611124802F09F
:109690002BFB31462846FFF7CBFE56B070BD00BF0E
:1096A0003C490020484900200000404065CD0108A9
:1096B000385300201109010899080108DD910008BC
:1096C00029920008ED910008E9BC0008353B00082C
:1096D000753B000886CD0108ACCD010808B5FFF741
:1096E00039FF03490DF09EFE0EF088F880B208BDE8
:1096F00000007A4470B507490546FFF73FFF06466C
:109700000CF0F2F9044631462846FFF791FE204658
:1097100070BD00BF000040407FB5F82300F1580540
:1097200004AC0646284604F8013D00F0E1FC0223A3
:10973000214600930122A123284600F0DDFC4FF4CE
:1097400000430822009306F16801A123044628463D
:1097500000F0FCFC0440E4B2284600F0CBFC2046BC
:1097600004B070BD30B58BB0044608F065FB01460F
:10977000594802F0B9FA594802F0B6FA204600F00A
:1097800095FB04F1580500F0C7FA00F071FA54484F
:10979000544902F0A9FA284600F0A4FC38B952480E
:1097A00002F0A2FA4FF49D715048FAF7A7FC07F0B7
:1097B00095F82046FFF7B0FF20B940F23F114B4823
:1097C000FAF79CFC94F86F0094F86A30049094F8CF
:1097D0006E0094F86920039094F86D0094F8681076
:1097E000029094F86C00019094F86B00009040484F
:1097F00002F07AFA284600F03DFA284600F09EFA78
:1098000004F1440584F8700004F1740000F01CFCBD
:109810000021284600F0BCFB012000F005FE0021DD
:10982000284600F0CBFB012000F01CFE2046FFF78D
:10983000DBFE00F0CFFA2F4802F056FA4FF4FA7030
:109840000EF0CAFA054600283ED12B4802F04CFA29
:109850002A4802F049FA2A4802F046FA294802F05A
:1098600043FA294802F040FA284802F03DFA284815
:1098700002F03AFA274802F037FA274802F034FAA1
:10988000264A2749274802F02FFA2749274802F09D
:109890002BFA274802F028FA04F12101254802F0AA
:1098A00023FA1E49244802F01FFA07A807F008FD12
:1098B00007A802F06FF90146204802F015FA104897
:1098C00002F012FA0BB030BD1D4802F00DFA284626
:1098D0000EF08AFABCE700BF71CE010887CE0108FE
:1098E0009ECE0108A0860100B9CE010829CE01084C
:1098F000CFCE010804CF010837CF01086DBC0108A5
:1099000075CF0108A6CF0108B5CF0108D7CF010850
:10991000FACF01081ED001086EBC0108ADB90108DC
:1099200088B9010841D0010851D0010858D0010878
:1099300063D0010883D001088ED00108A8D00108A7
:109940006BCF01082DE9FF4100F15805284600F0D2
:10995000CFFB04240226284F013C14F0FF0432D030
:10996000A123012239460096284600F0C5FB4FF49A
:109970000043804600930422A12302A9284600F058
:10998000E5FBB8F1000FE7D00028E5D09DF80830DE
:10999000442B1FD19DF809306E2B1BD10DF10A000D
:1099A00002F0B5FA013084B221460DF109008DF8BC
:1099B000086002F0E0FA002303220093A02302A92A
:1099C000284600F099FB284600F094FB204604B09E
:1099D000BDE8F0814FF488430024ADF808306E23D1
:1099E00000210DF10B008DF80A3002F0C4FA00944A
:1099F000A0230522E3E700BF64CD010838B50C467B
:109A00001131054603F068FA214651F8683F2846AF
:109A10002B604B686B6038BD024B186803685B684D
:109A2000184700BFD4490020024B186803689B68A0
:109A3000184700BFD44900202DE9FF4100231546F7
:109A40001370022206460D4F04AC386804F8011D5D
:109A500003680092D3F80C80012233462146C047A8
:109A600048B14FF4004238682946036800921C69E7
:109A700001223346A04704B0BDE8F081D44900205C
:109A800030B585B08DF80D200022074B8DF80C10F5
:109A90001C6803A923680092DD6802220346204661
:109AA000A84705B030BD00BFD449002037B54FF4FA
:109AB0000045064B1C68236800951D6913460A463D
:109AC00001462046A84703B030BD00BFD049002062
:109AD00037B50025054B1C6823680095DD681346E3
:109AE0000A4601462046A84703B030BDD0490020B1
:109AF00037B50225054B1C6823680095DD681346C1
:109B00000A4601462046A84703B030BDD049002090
:109B1000024B186803681B68184700BFD049002033
:109B2000024B186803685B68184700BFD0490020E3
:109B3000024B186803689B68184700BFD049002093
:109B40004FF47A735843B0FBF3F0F9F7C9B810B586
:109B50000446FFF747FC2146BDE81040FFF7F2BE80
:109B600010B5424C0BF08CFB20460222002107F07E
:109B7000F1F801222046114607F0ECF820460122B8
:109B8000022107F0E7F820460222032107F0E2F85D
:109B900020460022042107F0DDF820460222082199
:109BA00007F0D8F820460122092107F0D3F8204613
:109BB00001220A2107F0CEF8204602220B2107F0ED
:109BC000C9F806F07DFE002320461A460C2107F056
:109BD00083F8204600220C2107F04CF92046002291
:109BE00004F580640F2107F0B5F82046012200211A
:109BF00007F0B0F820460022022107F0ABF820461B
:109C00000022032107F0A6F820460222062107F0D1
:109C1000A1F820460022082107F09CF820460022E7
:109C2000092107F097F8204601220C2107F092F84D
:109C3000204602220D2107F08DF8204602220E2137
:109C400007F088F8204602220F2107F083F800234E
:109C500004F5806420461A460D2107F03DF82046A1
:109C6000BDE8104000220D2107F004B900000240B9
:109C700007F08EBB1D4B00B51A6889B0D2075FBFD5
:109C80001B4A106001221A601A4B1B4A04931B4B9B
:109C900005931B4B03931B4B02931B4B079308AB82
:109CA00043F8082D93E803008DE8030002AB0FCBC7
:109CB0000BF0AAFE90B1154802F016F800221448E5
:109CC000114607F047F80F2302220021104806F042
:109CD000E1FE09B05DF804EB0BF030BE69210D48E0
:109CE00009B05DF804EBFAF709BA00BFCC490020CF
:109CF000D4490020199A0008419B0008299A0008BD
:109D0000399A0008819A0008E9BC0008E2D10108EC
:109D100000000240F3D10108002307B5ADF804307C
:109D200001238DF8063001980BF006FA06F0C8FD05
:109D300003B05DF804EB0BF051BA0000194B10B5FD
:109D40001A688CB0D2075FBF174A106001221A60F0
:109D5000164B0793164B0593164B0693164B089319
:109D6000164B0993164B0A93164B0B930CAB13E946
:109D700007008DE8070005AB0FCB0BF02BFB04466B
:109D800001220F21104806F0E5FF3CB10F4801F019
:109D9000ABFF0BF0FDFA20460CB010BD0C4801F0F3
:109DA000A3FFF8E7C8490020D0490020AD9A000879
:109DB000D19A0008F19A0008119B0008219B000825
:109DC000319B0008E9BC00080000024064D1010892
:109DD00097D101082DE9F0479EB002F0C9FCDFF8E9
:109DE000C890284C284E294F16AD50B9CDE91944DA
:109DF000CDE91776CDF85890009495E80F0002F061
:109E0000BDFC234B4FF0000A1793224B4FF0010883
:109E10001693214B09A91893204B28461993204BE0
:109E2000CDE91C76CDE91A340423CDE9093A8DF841
:109E3000298009F0A3FC09F095FC0EF037FE51468D
:109E400010220CA80EF02BF8164BCDE910441593F8
:109E500003238DF836800B9302AC0BAD0FCDCDE90B
:109E60001376CDF848900FC42B68236014AB93E8A9
:109E700003008DE8030010AB0FCB03F06FF81EB0AA
:109E8000BDE8F087E9BC0008F5BD000821BE000868
:109E90006151010829500108394F0108D14E0108CC
:109EA000E54E01084F9B00087D1301082DE9F0479E
:109EB000044606F0E1FB1E4905460DF0B3FA0DF02D
:109EC00077FC01461B4801F00FFF4FF08041284608
:109ED0000DF046FC48B30025DFF86090DFF85080B5
:109EE000154E06F0C9FB494607460DF04DFCA8B9D2
:109EF000414638460DF096FA0DF05AFC01463046C0
:109F000001F0F2FE236885F001052046DB68294652
:109F100098474FF47A7006F0FBFCE2E7236820468E
:109F2000BDE8F047DB6800211847BDE8F08700BFB7
:109F300000007A44B5D10108C7D1010800002040D3
:109F400008B50D49012007F079F80C490B2007F0FE
:109F500075F80B490A2007F071F80A49042007F048
:109F60006DF80949072007F069F8BDE8084007497E
:109F7000052007F063B800BF614A0108A54D01083C
:109F8000154C0108C54E0108194E0108A14E0108E3
:109F9000002310B50C461A460D21074806F09CFE1A
:109FA00014B1012C00D010BD2246BDE810400D2197
:109FB000014806F05FBF00BF00080240002310B553
:109FC0000C461A460C21074806F086FE14B1012CF7
:109FD00000D010BD2246BDE810400C21014806F01B
:109FE00049BF00BF000002400BF044BB08461146C9
:109FF0001A460BF0DDBB084611461A460BF05ABB59
:10A00000084611461A460BF08FBB00000C2110B118
:10A01000024806F023BF014806F026BF00040240B4
:10A0200010B561B1FFF7DEF904460BF0F7FA01460F
:10A030002046FFF7A3FABDE810400BF007BCBDE8CF
:10A0400010400BF0F1BB000070B588B0FFF7CAF903
:10A050001D490546FFF792FA0C2106461B4806F0FB
:10A06000FDFE00230C211A46184806F035FE00219B
:10A07000012007F0E1FA102200210DEB02000DF0A3
:10A080000EFF134B02AC0293124B0693124B039339
:10A0900008AB13E903008DE8030094E80F000BF010
:10A0A000EDFB60B10BF0E6FA01460C4801F01CFE36
:10A0B0003146284608B0BDE87040FFF7B9B90848F6
:10A0C00001F012FEF4E700BF00004040000402402F
:10A0D0000DA0000811090108ED1601084CD2010875
:10A0E00062D20108014806F033BF00BFA08601001C
:10A0F00006F0FEBE06F018BF2DE9F041069F1E4691
:10A1000007F00303032B80460C46154603D12F218D
:10A110000D48F9F7F3FF2046BC07324629460AD519
:10A1200006F050FF10B10120BDE8F08101230020AE
:10A1300088F80430F8E7FB0702D506F051FFF1E795
:10A1400006F032FFEEE700BF90D201082DE9F041A2
:10A15000069C0D46E107804616461F4603D54C2156
:10A160000D48F9F7CBFFA20703D54F210A48F9F7AD
:10A17000C5FF23043A46314628460AD506F03EFF7D
:10A1800010B10120BDE8F0810123002088F80430DF
:10A19000F8E706F0FBFEF3E790D2010808B50321CB
:10A1A000034806F070FE003018BF012008BD00BF54
:10A1B000000402400A460248032106F05BBE00BFCD
:10A1C0000004024008B581B1012303211A460A4860
:10A1D00006F082FD0321084806F040FEBDE8084075
:10A1E00003220548114606F057BD0122BDE808408C
:10A1F0000321014806F0AEBD0004024007F0BEB8DE
:10A200001FB501A801F088FC01A807F097F905B077
:10A210005DF804FB07F000B907F018B9084606F02E
:10A220008FBFDFB50023CDE90133ADF80C3001233A
:10A230008DF807308DF808306FF01D038DF8093068
:10A240000723044601A88DF80A3001F08AFC236830
:10A2500006461B6820460F469847864277EB010367
:10A26000B4BF0120002004B0D0BD00002DE9F043B0
:10A2700085B014461D4607F081F880468946261AA7
:10A2800022462B4601A865EB010701F045FC40463C
:10A29000494601F0A9FC29468046204601F0A4FC6D
:10A2A00039460446304601F0B5FC22460346414695
:10A2B000064801F019FD01A806F0F2FF18B130467A
:10A2C000394602F089FA05B0BDE8F08308D30108E9
:10A2D000704770477FB500F10806054630460C46CA
:10A2E00001F002FF60BB334801F0FEFCA27C617C00
:10A2F000314801F0F9FC637C3BB1686800210368D8
:10A300001B689847022000F08FF8A37C3BB1686877
:10A31000002103685B689847022000F0A3F8616899
:10A320004E2918D04F2916D0452914D0162123487C
:10A33000F9F7E4FE1721224B224A20480DF038FCA1
:10A340006421304601F0BCFE0028CFD143211B48D8
:10A35000F9F7D4FECAE7A268082A0BD0092A09D067
:10A36000072A07D024211548F9F7C8FE144B164ACE
:10A370002521E2E7E3680A2B10D009DC052B0ED07B
:10A3800034210E48F9F7BAFE0D4B104A3521D4E7B7
:10A390000F2B04D0142BF3D1022300E00123A07C67
:10A3A0000290607C0190207C0090206807F0ACFB5C
:10A3B00004B070BD54D30108B5D301086DD30108B2
:10A3C00065B80108FCD3010860D401082CD4010849
:10A3D00010B5044607F06AFB04F10800BDE8104020
:10A3E00001F085BE084607F077BC38B50C468D18DD
:10A3F000AC4204D014F8010B07F06EFCF8E738BD4E
:10A4000007F07ABB084607F097BC000010B5044679
:10A41000044BC0E900310121083001F073FE2046F1
:10A4200010BD00BFDCD30108042817D8DFE800F016
:10A430000309100E1200002303211A46084806F0F3
:10A440004BBC00220321064806F084BC0222F9E737
:10A450000122F7E70321024806F0A2BC704700BFC3
:10A4600000000240042817D8DFE800F00309100EAE
:10A470001200002302211A46084806F02DBC0022D3
:10A480000221064806F066BC0222F9E70122F7E73E
:10A490000221024806F084BC704700BF0000024061
:10A4A000406803681B681847406803685B68184782
:10A4B000406803689B68184740680368DB68184772
:10A4C000406803681B691847406803685B69184760
:10A4D00070470000436910B504469BB983698BB986
:10A4E0008168094801F000FCA168084801F0FCFB04
:10A4F00041F28830F8F7F4FBBDE810403121044800
:10A50000F9F7FCBD10BD00BF43D5010861D50108B6
:10A5100078D50108C0E903120346002210B5074CA4
:10A52000C0E905224460064C8460064C0460064C79
:10A53000C0E90741586280F8282010BDB9D501084C
:10A54000BFD50108CCD50108ECD50108436970B529
:10A5500005460C4633B3012913D002291CD000292B
:10A5600052D10A46184601210BF021FF2246022152
:10A5700068690BF01CFFE868BDE8704003681B6960
:10A5800018470A4618460BF012FF22466869022156
:10A59000BDE870400BF00BBF0E21BDE870401846BF
:10A5A0000BF066BE806948B301290CD0022914D093
:10A5B00051BB0A4601210BF0F0FF22460221A86997
:10A5C0000BF0EBFFD7E70A460BF0E7FF224602212C
:10A5D000A869BDE870400BF0E0BF1A4601210BF0FE
:10A5E000DCFF01222146A8690BF0D7FF01220421DC
:10A5F000A8690BF0D2FF01220821E9E76921BDE833
:10A6000070400248F9F77ABD70BD00BF78D50108E7
:10A610008068FFF79BBF000038B504460C2000F0AF
:10A620006DFC054621690BF0FFFD656128460BF0C6
:10A63000ABFE38B342F26252A168144801F054FBF9
:10A64000002384F828300C2000F058FC05462169CE
:10A650000BF0C0FEA56128460BF006FFA0B14FF439
:10A660001552A168094801F03FFBF021A0690BF0E9
:10A670008AFF012384F828302046BDE838400221B3
:10A68000FFF764BF6061DEE7A061F5E798D40108D9
:10A690000221FFF75BBF034640690A4610B104215F
:10A6A0000BF085BE986910B104210BF076BF70479E
:10A6B0002DE9F04790F8284006460F46002C3CD084
:10A6C000FEF790FE0546002F51D0FFF707F80F2444
:10A6D00040F64759DFF8B08048450EDC0146404659
:10A6E00001F002FB2B684FF47A711B6928469847EA
:10A6F0002846FEF7F3FF013CEED1B168204801F097
:10A70000F3FA00213046FFF7C6FF1E24DFF87CA0D5
:10A71000DFF87C802846FEF71DFF81460CF012FA18
:10A7200015A3D3E900230CF0F5FC48B12B6840F2E7
:10A73000DC511B69284698473C462046BDE8F08717
:10A74000514648460CF06EFE0DF032F8B1680246F4
:10A75000404601F0C9FA2B6864211B6928469847D6
:10A76000013CD7D101213046FFF795FFE5E7B168FD
:10A77000044801F0B9FAF5E7666666666666064063
:10A78000F1D401082DD50108B9D4010800007A449C
:10A7900006D50108F0B508B90020F0BD00274668CD
:10A7A0004D1CB5421760F7D803685C185B5C03F07A
:10A7B0001F03A3F1180103298FBF38460D49C9189B
:10A7C00011F8180C0544AE42E6D304280DD8DFE892
:10A7D00000F00403070C0C00637813600130DCE721
:10A7E000B4F801305BBA9BB2F7E7D4F801301BBA7A
:10A7F000F3E700BF10D60108F7B51F4643681646B9
:10A800004A1C9A4205460C4617D803685B5C03F065
:10A81000C003402B11D196B101AAFFF7BBFF50B185
:10A82000019A04446B68A118994206D8296810441B
:10A830000C4434603A6003B0F0BD0020FBE73046C2
:10A84000F9E72DE9F7439946436817464A1C9A42AF
:10A8500080460D4624D803685B5C03F0C003402BA0
:10A860001ED1FFB101AAFFF795FF0446A0B1019EDA
:10A8700009F10109B14513D30544D8F80430721920
:10A880009A420DD8D8F800103246294438460DF0C7
:10A89000E2FA00233444BB55204603B0BDE8F08300
:10A8A0000024F9E73C46F7E7F0B5002931D0172A34
:10A8B0001CD8D3B2A3F11804032C8CBF0024164C6F
:10A8C0008D689CBFE41814F8184C6F1C4E6804EB9C
:10A8D000070CB4451DD20E6818438F6070550020D8
:10A8E0000130231A5D1C0BD1601CF0BDFF2A05D975
:10A8F000B2F5803F2CBF1A231923DBE71823D9E7D1
:10A900008E680D68DB00771C22FA03F38F60AB556D
:10A91000E6E70020E9E700BF10D60108172BF8B5DD
:10A920000D4616461C4612D8DBB2A3F11802032AC4
:10A930008FBF0022144A9B1813F8182CAB68013201
:10A94000234413446A6893420BD30020F8BDFF2BC5
:10A9500005D9B3F5803F34BF19231A23E5E718233F
:10A96000E3E722462946FFF79FFF07460028ECD081
:10A970002868AB68314618440DF06DFAAA68E019F2
:10A980002244AA60E2E700BF10D6010818B10023F4
:10A99000C0E9001283607047436873B514464A1CCF
:10A9A0009A4206460D4602D9002002B070BD0368E7
:10A9B0005B5C13F0C00FF7D1002CF5D001AAFFF7B4
:10A9C000E9FE0028F0D03268019B525D12F0E00FE2
:10A9D00018BFDB432360E8E70A1EABBF0146014610
:10A9E0000020D243B8BF2020FFF75EBF03685B5C46
:10A9F00003F0E001E02907D132B1A3F1F5014B42A8
:10AA00004B4113700120704700207047836810B5D8
:10AA100044685A1CA24208D2002914BFF524F42429
:10AA2000016882600120CC5410BD0020FCE7F0B426
:10AA300046684F1CB74208D805686C5C04F0E00417
:10AA4000402C02D1F0BCFFF7D7BE0020F0BC70470D
:10AA500013460A4601464020FFF760BFF0B446683F
:10AA60004F1CB74208D805686C5C04F0E004602C09
:10AA700002D1F0BCFFF7E5BE0020F0BC7047F0B497
:10AA800046684F1CB74208D805686C5C04F0E004C7
:10AA9000602C02D1F0BCFFF7AFBE0020F0BC7047C5
:10AAA00070B5054608460C460EF0CEF82246034621
:10AAB0002946BDE870406020FFF730BF83684168D9
:10AAC0005A1C8A423FBF8260BF220168012034BF06
:10AAD000CA54002070470368585CA0F1BF03584275
:10AAE0005841704713B5036814465B5C03F0E003FC
:10AAF000A02B07D142B101AAFFF74CFE019B2360B6
:10AB000002B010BD0020FBE71046F9E783684168FA
:10AB10005A1C8A423FBF8260FF220168012034BF75
:10AB2000CA540020704730B18068013888428CBF19
:10AB30000020012070470120704708B50246FFF74A
:10AB4000F2FF30B91268505CA0F1FF03584258413F
:10AB500008BD0120FCE743688B4207D903685B5CB2
:10AB600013F0C00F0CBF0120002070470020704779
:10AB700043688B4208D90368585C00F0E000A0F1FC
:10AB800040035842584170470020704743688B4249
:10AB900008D90368585C00F0E000A0F16003584257
:10ABA000584170470020704743688B4208D90368BA
:10ABB000585C00F0E000A0F1A003584258417047F3
:10ABC0000020704710B50446FFF7EEFF50B16368F0
:10ABD0008B4208D92368585C00F01F00A0F11F03C6
:10ABE0005842584110BD0020FCE743688B4208D909
:10ABF0000368585C0C30C0B201288CBF00200120D3
:10AC00007047002070470023C0E9013303690160E9
:10AC1000C360704703468068F0B51D68013090FB43
:10AC2000F5F405FB14005C68A04224D0002696428F
:10AC3000304601D11046F0BD8F5DD3E902452F5556
:10AC40009C681D68671C97FBF5F405FB14745F682E
:10AC50009C60BC4204F1010402BF94FBF5F705FBC4
:10AC600017475F6094FBF5F705FB17445D68AC423E
:10AC7000E1D00136DBE70020DDE70000F8B503682E
:10AC80000446002B0D46164603DC3E212948F9F701
:10AC900035FA3246002128460DF001F9D4E9017059
:10ACA000B8420CD00021236801EB070C9CFBF3F2A7
:10ACB00003FB12C2904205D10020884204D14FF01C
:10ACC000FF3031E00131EFE7C21992FBF3FE03FBE5
:10ACD0001E2ED4F80CC01CF80EE0BEF10A0F26D1CF
:10ACE00028B3013A92FBF3F103FB1122002106F194
:10ACF000FF3E71450ED2E7686368FB5C6B54676882
:10AD00002668013797FBF6F306FB1377013188427B
:10AD10006760EEDA1CF802300D2B4FF0000304D10F
:10AD2000054405F8013C0138F8BD2B54FCE701301F
:10AD3000C3E700BF14D601084B1C017343738B1C7F
:10AD400003318373C17370472DE9F041074688468C
:10AD50001E4615461AB952211548F9F7CFF9D7E919
:10AD60000143A34221D2E41ADEB1A3B9A5420ED316
:10AD70003B7B3370BB6839682246194440460DF06E
:10AD80006AF8BB682344BB602046BDE8F0817B7B4A
:10AD900033702C46EEE7A54201D3FB7BE9E7BB7B92
:10ADA000F6E7AC4228BF2C46E4E70024ECE700BFFE
:10ADB00064D601080023C0E900128360704710B513
:10ADC00004460846C4E900120021A16021730DF079
:10ADD00066F8204610BD000038B51546D0E90123BD
:10ADE00004465819904202D9257B55B1D51A2068DE
:10ADF0002A4618440DF02FF8A3681D44A5600125CC
:10AE000003E017210248F9F779F9284638BD00BF59
:10AE1000A8D6010807B502AB03F8011D01221946A7
:10AE2000FFF7DAFF03B05DF804FB00687047806845
:10AE30007047002383607047D0E90120101A7047E3
:10AE4000026880681044704738B5D0E901230D4688
:10AE500059189142044602D9017B21B1D51AA16843
:10AE60002944A16038BD45210148F9F747F9F6E7C3
:10AE7000A8D6010813B5044689B201A801F07BF8F1
:10AE8000022201A92046FFF7A7FF02B010BD13B5AB
:10AE90000446684601F05CF8052269462046FFF743
:10AEA0009BFF02B010BD13B5044601A801F063F882
:10AEB000022201A92046FFF78FFF02B010BD00005B
:10AEC00008B50146044800F00FFFBDE808400C211A
:10AED0000248F9F713B900BFE8D6010806D7010800
:10AEE00008B5044800F000FFBDE808401E210248F4
:10AEF000F9F704B971D701089ED7010810B500F021
:10AF00008FFF044630B9044800F0EEFE27210348C5
:10AF1000F9F7F4F8204610BD5FD701089ED7010865
:10AF200000F07EBF10B9024800F0DEBE00F062BF44
:10AF30004AD70108FFF7E2BF00F072BFFFF7F2BF88
:10AF4000FFF7F0BF10B5074C0A44914200D110BD85
:10AF500011F8013B4340DBB234F8133083EA102090
:10AF6000F3E700BFE2D70108F8B50E46054680B109
:10AF70004F1C384600F054FF044640B13A460021C9
:10AF80000CF08DFF3246294620460CF064FF204627
:10AF9000F8BD0446FBE738B50D46044628B10DF070
:10AFA00053FE23462044834201D1002038BD13F8CC
:10AFB000012BAA42F7D10120F8E737B504460D4628
:10AFC0000CF022FE002201A9026020460DF068FF6D
:10AFD00004460CF019FE0368222B08D0019B1B7855
:10AFE0002BB9002C03DB20462B6003B030BD0123BE
:10AFF00000202B60F9E700002DE9F04F05464FF0E7
:10B00000010B002687B0CDE9031206F10903122BCC
:10B010008CBF0320022000F003FF0090E8B132460D
:10B0200036490DF0DFFD039B53F82690EDB900245F
:10B03000009800F0DFFEBBF1000F02D1284600F0BF
:10B04000D9FE84B1049B0136B34225464FF0000B74
:10B05000DBD1204607B0BDE8F08FBBF1000F02D175
:10B06000284600F0C7FE0024F3E7254B4FF0000808
:10B07000B9F1000F08BF994648460DF0E5FD019073
:10B0800000980DF0E1FD0290284649460DF00BFEB8
:10B09000B8B928460DF0D8FDDDE9012301309B1A2F
:10B0A00008FB030000F0BCFE04460028BFD00346A6
:10B0B0002F4618F1FF3809D2394618460DF0BCFD6D
:10B0C000B6E7019B08F101081844DEE74946384617
:10B0D00005930DF0E8FD059BA0EB070A52463946A3
:10B0E00018460DF0CBFD009950440DF0A5FD019AD6
:10B0F000029B9244C3185744DBE700BFB8B901086C
:10B100006FBC010830B580B10346021F00F118047E
:10B1100052F8045F8D4208D0A242F9D11C301A4681
:10B1200014680433013401D1116030BD8342F6D17B
:10B13000FBE770B5044680B1064600EB8105AE42E0
:10B1400004D12046BDE8704000F054BE56F8040B10
:10B150000028F4D000F04EFEF1E770BD2DE9F74F66
:10B1600089460092002838D00027C45D8CBB054674
:10B170008346264600EB070AD34538D104B1013691
:10B18000002E6FD00137384600F04AFE8346002873
:10B1900066D03A4600210CF082FEB00000F040FE7E
:10B1A0000446002860D04FF000084146AA4532D13D
:10B1B00031B15846FFF7D8FE002855D044F8280092
:10B1C000584600F017FE009B1E60204603B0BDE805
:10B1D000F08F0137B7F5807FC7D10024264620467F
:10B1E00000243146FFF7A5FF009B1C60EDE79BF8AC
:10B1F00000304B4505D10CB1002401360BF1010B99
:10B20000BAE70CF0DBFD9BF80030184443781B07CD
:10B2100058BF0134F2E72B784B4513D181B1584622
:10B22000FFF7A2FE00B308F1010344F82800002153
:10B230003A46584601930CF032FE019B0021984695
:10B240000135B3E701910CF0B9FD2B780199184451
:10B25000407810F0080F04BF0BF801300131EFE720
:10B260000446BCE73446B0E7584600F0C3FDB6E7F5
:10B270002DE9F743002506460820884691461F46DB
:10B28000009500F0CDFD0446002868D0C0E90055C7
:10B2900030460DF0D9FC01280FD133782A2B0CD180
:10B2A00009F1FF33C4F80080636022684A4502D286
:10B2B00063684B4543D32B4B0EE02D213046FFF7FF
:10B2C0006AFE0546C0B902A941F8040D3046FFF7F1
:10B2D00074FE019B63B1244B3B6000992846FFF745
:10B2E00028FF002C37D0204600F084FD002432E0F7
:10B2F000C4E900001D46D8E76A462D213046FFF715
:10B300002DFF009B0546013B012B01D9174BE3E7BD
:10B31000002302AE46F8043D31460068FFF74DFEBB
:10B320002060019B0BB1124BD6E731466868FFF7EE
:10B3300044FE6060019B002BB7D00E4BCCE742452A
:10B3400001D3434501D20C4BC6E700992846FFF7CD
:10B35000F0FE00233B60204603B0BDE8F0830546C5
:10B36000BBE700BFBEDA010838DA010857DA010886
:10B3700080DA01089FDA0108DEDA010838B590B1F9
:10B38000451E15F8014F0CB9204638BD0CF016FDCE
:10B3900023462044427802F00302022A08BFA4F1A7
:10B3A00020032B70EDE70120EFE708B520B34A1C1E
:10B3B00022D0062920D8DFE801F0040D1013161959
:10B3C0001C00002303600CF04DFE0840431C584253
:10B3D000584108BD00234360F5E700238360F2E78E
:10B3E00000238361EFE70123C360ECE700230361DF
:10B3F000E9E700234361E6E70120EAE770B5064686
:10B400000D1F01F1180455F8041F4B1C03D1A54270
:10B41000F9D1002070BD3046FFF7C7FF0028F6D0F5
:10B42000F8E708234A4291FBF3F302F0070201F028
:10B43000070158BF51420122DBB2C9B202FA01F141
:10B44000C25C1143C154704708234A4291FBF3F395
:10B4500002F0070201F0070158BF51420122DBB29E
:10B46000C9B28A40C15C21EA0201C1547047082375
:10B4700091FBF3F3DBB2C05C4B4203F0070301F036
:10B48000070158BF5942C9B2084100F00100704796
:10B490002DE9F047089E8A4690461D46DDF8289023
:10B4A000074610B11446A24507D875B901220024F9
:10B4B0000B9B1A602046BDE8F08721463846FFF70F
:10B4C000D6FF002861D10134EDE7099B023B042B34
:10B4D00004D8DFE803F0282C2C3034006B680133EB
:10B4E0006B6028460CF0BEFD013108BFB0F1FF3F94
:10B4F000DCD031462846FFF758FF0028D6D12FB3BD
:10B50000044621463846FFF7B2FF002841D10134F6
:10B51000A245F6D10446013E042E19D8DFE806F014
:10B520002B2D2F313300AB680133AB60D9E7EB68CB
:10B530000133EB60D5E72B6901332B61D1E76B69F0
:10B5400001336B61CDE7002DE5D1AFE73C46E2E783
:10B550002C6028460CF086FD013108BFB0F1FF3F9A
:10B56000A4D0B9F1000FA1D049462846FFF746FF05
:10B5700000289FD09AE76C60EBE7AC60E9E7AC612C
:10B58000E7E7EC60E5E72C61E3E7A045DBD1444663
:10B5900090E7A045BFD1FAE700232DE9F04F06461A
:10B5A0008BB01C200C469046099300F039FC0546F0
:10B5B000002800F0E4801C2000F032FC0746002840
:10B5C00000F0DD804FF0FF31021F2B1F05F1180046
:10B5D00043F8041F984242F8041FF9D100230121C7
:10B5E000D4F800A00DF12409CDE90031CDE90279AC
:10B5F0003C21234652463046FFF74AFF099900296D
:10B600006ED1824502D12846FFF77CFD02234FF020
:10B61000010AD4F804B0CDE900A3CDE902592346CC
:10B620005A463C2106F10800FFF732FF099B002B28
:10B6300056D183454CD151462846FFF763FD03237D
:10B640004FF0020AD4F808B0CDE900A3CDE90259C1
:10B6500023465A46182106F11000FFF719FF099BEF
:10B66000002B3DD1834546D151462846FFF74AFD80
:10B6700040F26F1BA3690593E368049306F114037A
:10B680000693DDF810A006F11303079351460698C0
:10B69000FFF7EDFE28B105990798FFF7E8FE0028AF
:10B6A00036D1BBF1010B33D0E36820460133E360B0
:10B6B0000CF0D8FC013108BFB0F1FF3F24D0A369E2
:10B6C00029462046D4F80CA00593FFF797FEDDE746
:10B6D000424621463046FFF75FFF09900028AED072
:10B6E000284600F087FB17B1384600F083FB099825
:10B6F0000BB0BDE8F08F424621463046FFF74CFFC5
:10B7000009900028ECD1B3E701234FF0000A099318
:10B71000099B002BE4D1049B534520D104212846EA
:10B72000FFF7F0FC05230622D4F810A0CDE9003283
:10B73000CDE90259234652460C2106F11800FFF7C5
:10B74000A7FE099B002BCBD18245C9D06369A3EB2F
:10B750000803042B0CD94FF0FF330993C0E742468E
:10B7600021463046FFF718FF09900028B8D1D9E7E5
:10B77000424621463046FFF70FFF0990B0E74FF0F1
:10B78000FF330993002DB2D00027A9E72DE9F04F30
:10B79000002487B0924606AA894642F80C4D2C2117
:10B7A0009846109DFFF7DAFC074688B93E4B2B60A0
:10B7B00003993846FFF7BDFC07B0BDE8F08FD0F81D
:10B7C00000B072685A451CD2304600F013FB0134B9
:10B7D000039BA342ECD957F824602F213046FFF792
:10B7E000DAFBA8B92B46304642465146FFF740FDEA
:10B7F0002B680646002BE2D00028D9D000F0FAFAD8
:10B80000D6E759464846FFF70CFE0BF1010BD8E787
:10B8100000232F21304604AA0493FFF79FFC0499CC
:10B8200006464B1E012B04D9204B2B60FFF781FCF1
:10B83000BEE742462B4651460068FFF719FD2A68CD
:10B8400083462AB108B100F0D5FA04993046EDE7F5
:10B850002D213068FFF79FFB18B908F1FF32CBF8B4
:10B860000420002306A941F8043D7068FFF7A5FBFA
:10B87000059A00901AB10E4A58462A60E3E7DBF8B1
:10B880000020DBF80410914205D230460499FFF7FE
:10B8900050FC584699E7114648460192FFF7C1FD12
:10B8A000DDE900321A44ECE703DB010815DB01088F
:10B8B0003ADB01082DE9FF4100230E4603931446AD
:10B8C00002B902AC236048B90546564B2360039980
:10B8D0002846FFF72EFC04B0BDE8F08103AA202122
:10B8E000FFF73CFC039B0546062B02D04E4B236022
:10B8F000EDE71A22002130460CF0D1FA0094002224
:10B900003C2331462868FFF741FF2268002ADED138
:10B9100000943C2306F108016868FFF737FF2268AE
:10B92000002AD4D10094182306F11001A868FFF76B
:10B930002DFF2368002BCAD16869FFF71FFD07227E
:10B940003A496869FFF758FB80460DF07DF90128F8
:10B9500006F1130706D198F800303F2B04BF2A23C5
:10B9600088F8003000220823394640460094FFF74B
:10B970000DFF404600F03EFA2268002AA7D10721B9
:10B980003846FFF774FD30B111463846FFF749FDE0
:10B990000721FFF759FDEF6806F1140838460DF04E
:10B9A00053F9012804D13B783F2B04BF2A233B7075
:10B9B00020230022414638460094FFF7E7FE00218D
:10B9C0004046FFF741FD2368002B80D12F693846A0
:10B9D000FFF7D4FC00287FF47AAF38460D221449D3
:10B9E000FFF70AFB074600283FF471AF18360094B2
:10B9F0000D2301223146FFF7C9FE384600F0FAF95F
:10BA0000012421463046FFF732FD30B1611E304639
:10BA1000FFF707FD2146FFF717FD01340D2CF0D18C
:10BA200055E700BFE2D90108FAD9010870000020EB
:10BA30008C000020F0B58DB0CDE90023054628B973
:10BA40004FF0FF304FF0FF310DB0F0BD2422002148
:10BA500003A80CF024FA03A968460CF0FFF804468A
:10BA60000028EDD00CF0FEFA4A1C08BFB0F1FF3FF1
:10BA700006460F46E4D0626921462846FFF78CFD52
:10BA80000028DDD120460CF0EDFA4B1C08BFB0F1C8
:10BA9000FF3FD5D08F4208BF864203D020460CF02E
:10BAA000E1FAD1E723682046013323600CF0DAFA8B
:10BAB000013108BFB0F1FF3FC2D06269214628467C
:10BAC000FFF76AFD0028E9D0BAE770B53C258AB0D7
:10BAD000DDE90E64019496FBF5F405FB1464029411
:10BAE000182493FBF4F505FB1433CDE90330481E0D
:10BAF0000C2190FBF1F301FB13010023CDE9073387
:10BB00009DF84030A2F26C7201A80591069209934B
:10BB10000CF0A8FA0AB070BDF7B5044602A860E9B7
:10BB200002230CF089F80269037A551C426990F8E7
:10BB300004C0077B02F26C71067EC2690068A370C4
:10BB40000033207018BF01232046013284F801C061
:10BB5000E7702571A4F80510E6712272637203B0D4
:10BB6000F0BD30B5457A85B0C4788378B0F805204B
:10BB70000179029505780195407800902046FFF7FD
:10BB8000A4FF05B030BD904271EB0303B4BF0120A8
:10BB900000207047032210B5104986B00B7801339E
:10BBA00093FBF2F202EB42029B1A0D4A0B7052F821
:10BBB00023400278B0F80530049242781A210392AB
:10BBC00082780292C2780192027920460092054A58
:10BBD0000CF0D4FF204606B010BD00BF264A00205E
:10BBE000E4DB0108A9DB0108B1F1004F08BF002820
:10BBF0001FB502460B4608D001A8FFF78DFF01A82C
:10BC0000FFF7C8FF05B05DF804FB0148FAE700BF85
:10BC1000DBDB01082DE9FF4703220D462B490028F5
:10BC20000B78044603F1010393FBF2F202EB4202AC
:10BC3000A3EB0203264A0B7052F8236075F1000350
:10BC40003EDA4FF0010A444265EB4505214A0023E4
:10BC5000204629460BF0F2FD1E4A074600232046E7
:10BC600029460BF0EBFD104619464FF461620023A4
:10BC70000BF0E4FD4FF46162804600232046294624
:10BC80000BF0DCFD104619463C2200230BF0D6FDDC
:10BC90003C2281460023204629460BF0CFFDCDF8FB
:10BCA0000080CDE901923B46BAF1000F0BD00A4A61
:10BCB0001A2130460CF062FF304604B0BDE8F08730
:10BCC0004FF0000AC2E7054AF2E700BF264A00200B
:10BCD000E4DB010880510100C7DB0108C8DB010873
:10BCE0000FB404B0704700000FB437B51B4C256883
:10BCF00055B9032229460120F5F7AEFF2B462A4607
:10BD000029462060F5F7CCFF154D2A68013A033229
:10BD10001ED864212068F6F7AFF98022002111486F
:10BD20000CF0BDF807AB069A80210E4801930DF088
:10BD300027FB7F2803DD0C490C480CF07DFF2B68A6
:10BD400008489847002320681A461946F5F7A8FFC7
:10BD500003B0BDE8304004B0704700BFB04A0020D7
:10BD6000284A0020304A00205AD70108AB4A002058
:10BD70000FB410B50D4CA2B02268013A033210D8AE
:10BD800025AB249A802102A801930DF0F9FA7F28AF
:10BD900004DD07490DF183000CF04EFF236802A873
:10BDA000984722B0BDE8104004B070472C4A0020EC
:10BDB0005AD7010870B50446054E4518AC4200D16B
:10BDC00070BD14F8011B3046FFF78EFFF6E700BF89
:10BDD000F0DB010838B50C461546FFF785FF204615
:10BDE0002946FFF7E7FFBDE838400148FFF77CBF71
:10BDF0006EBC010810B5044670B1F7F7C3FF2046CA
:10BE0000F8F764F8F7F796FEBDE81040034A938808
:10BE100001339380F7F7AEBE10BD00BFAC520020D7
:10BE200070B5214C8AB0226806460132632A22602E
:10BE30001E4D0BDDF7F7B6F90523002201A9F7F730
:10BE4000F3F8F6F7F5FD002328602360F6F7F0FD20
:10BE50002B6803F57A73984204D9F6F7E9FD0023BD
:10BE600028602360124A134C13781BB92360636067
:10BE700001231370F7F786FF3046F7F795FF054665
:10BE800068B1324600210CF00AF8F7F753FE238818
:10BE900001332380F7F76EFE28460AB070BD638831
:10BEA00001336380F8E700BFB84A0020BC4A002095
:10BEB000B44A0020AC5200202DE9F04B00240027AA
:10BEC000467805784FEA066848EA04024FEA1629E0
:10BED00090F80280067949EA050342EA060B4FEA28
:10BEE00008464BEA0602C67843EA070C4FEA1847B1
:10BEF0004CEA07034FEA16694FEA062848EA0200AF
:10BF000049EA0301BDE8F08B006800BA7047008879
:10BF100040BA80B270472DE90048FFF7CDFF0022FC
:10BF20008C4601F08003134314BF61F0FF016146AA
:10BF3000BDE8008800687047837842781B04007869
:10BF400043EA02231843704700887047FFF7F2BFA7
:10BF50000370130E4370130C8370130AC3700271C5
:10BF6000052070470B0E03700B0C43700B0A837097
:10BF7000C170042070470B0A0370417002207047A3
:10BF80000B0A017043700B0C090E8370C170042002
:10BF90007047A0F14103052B02D83738C0B2704773
:10BFA000A0F16103052B01D85738F7E73038C0B24C
:10BFB0000A2828BFFF2070470022013910B501442C
:10BFC000441E8C4204D014F8010F08B1002A01DA93
:10BFD000104610BDFFF7DDFF0F2802D840EA02121D
:10BFE000EFE74FF0FF32F3E738B505460C460CF0AB
:10BFF00081FD611B013190FBF1F303FB110028442B
:10C0000038BD38B5451E15F8014F04B938BD0BF0E1
:10C01000D5FE23462044427802F00302012A08BFDD
:10C0200020332B70EFE72DE9F04106460CF00CFEB3
:10C0300030B3002734180BF0C1FE14F8013C35462C
:10C0400018444378621E19070DD42F463B78A4EBA1
:10C05000050801355BB908F1010239463046BDE8F3
:10C06000F0410BF003BF04F8017C1446E3E70BF04A
:10C07000A5FE15F8013C184443781B07E5D4EAE710
:10C08000BDE8F08108B50CF0CDFDB0FA80F04009B4
:10C0900008BD000010B50446034B03604068F6F786
:10C0A000C5F9204610BD00BF44DC010810B50446A8
:10C0B000FFF7F0FF20460821FEF742FF204610BDA3
:10C0C00038B5436804460D461BB90E210548F8F7FC
:10C0D00015F829466068F5F7CFFF431E58425841CE
:10C0E00038BD00BFF6DB01084068F6F753B908B564
:10C0F000002340681A461946F5F7D2FD431E584200
:10C10000584108BD38B50D4600210B4B044641602F
:10C11000036003220120F5F79FFD606018B95721E5
:10C120000648F7F7EBFF2DB1002360681A46194661
:10C13000F5F7B6FD204638BD5CCD0108F6DB0108F9
:10C14000014BDB68184700BFC04A00200120704740
:10C1500001B1096818B1806A431A584258417047C2
:10C160002DE9F041DFF84C80D8F80430984710F5FD
:10C1700061760446D8F800000D4641F1000700F052
:10C1800082FB08B9BDE8F081016879B1D1E90823E3
:10C19000944275EB030301DAC1E90845D1E90623AE
:10C1A000964277EB030301DAC1E9066700F062FB10
:10C1B000E7E700BFC04A002038B50C4B05461868B9
:10C1C00000F061FB10B90023184638BD4FF47A74B3
:10C1D00003686C431A68A242F6D000F04BFB0028BB
:10C1E000F1D003681A689442F6E700BFC04A002005
:10C1F00010B5044618B9ED210748F7F77FFF074B44
:10C200005B689847D4E90623904271EB0304B4BFFE
:10C21000101A002010BD00BF84DC0108C04A0020B5
:10C220002DE9F8498846044610B10369012B04D171
:10C230004FF481711648F7F761FFD4E906BC5BEA59
:10C240000C0323D0D4E90867BBEB06006CEB0701B5
:10C250000BF0AAF80546206901380BF08BF801466F
:10C2600028460BF093F9054640460BF083F8294623
:10C270000BF0D8F829460AF0CBFF0BF0BFFA3218C2
:10C2800047F1000310461946C4E90601BDE8F889E4
:10C2900084DC010841F65832A0F55223A3F6183386
:10C2A000934224D8A0F55423A3F1F902622A1ED99F
:10C2B0006FF454729A18C62A19D9A3F21353302B6B
:10C2C00015D9104B984214D903F6B833984212D9B5
:10C2D00003F51673984210D903F5167398420ED9D8
:10C2E00003F5E173984294BF0520062070470020B3
:10C2F00070470120704702207047032070470420D8
:10C30000704700BFE8320D00F8B5054620B94FF47C
:10C3100087712348F7F7F2FE224E306800F0B3FA37
:10C3200000283CD0002D3AD003681A79AA4232D1B5
:10C330001F7B00F09FFA28BB8FB3062D03D9402145
:10C340001748F7F7DBFE184B53F835402CBB40F28B
:10C3500019111348F7F7D2FE306800F094FA064638
:10C36000E8B17C4337683B79AB4204D1214638467B
:10C37000FFF756FF3C61304600F07CFA0646002885
:10C38000F0D10CE003681A79AA42D2D11B7B002BB2
:10C39000CFD00137CDE70027CBE7012CDCD1F8BDAA
:10C3A00084DC0108C04A00204CDC010810B5084CB0
:10C3B000236863B1FFF7D4FE206800F06DFA30B156
:10C3C000206800F060FA00F055FA0028FBD110BD9B
:10C3D000C04A0020F8B5114C0646227E0F4622B90D
:10C3E00040F27F110E48F7F789FE206810B900254A
:10C3F0002846F8BD0B4B002E08BF1E4600F043FA3E
:10C4000004460028F3D0256839462846B04700285E
:10C41000EED1204600F02EFAF2E700BFC04A00201D
:10C4200084DC01084DC100082DE9F04F3A4C91B071
:10C43000237E83468946924623B940F2AF1137489E
:10C44000F7F75CFE236823B90024204611B0BDE84D
:10C45000F08FFFF785FE324B2068B9F1000F08BF5F
:10C46000994600F010FA80460028EDD00468237B3E
:10C47000DBB94FF0FF3600240027404600F0FAF900
:10C480008046F8B9BAF1000F01D0CAF80060002E5A
:10C49000DBD1012FD9D9791E3046FFF7A5FD10ABAE
:10C4A00003EB800050F8404CCFE7A3685B45E0DB2E
:10C4B00000212046C8470028DBD02046FFF798FE21
:10C4C0000646D9E7D8F800502B7B002BD5D0AB68B7
:10C4D0005B45D2DB00212846C8470028CDD028463E
:10C4E000FFF786FE38B90F2F9FBF10AB03EB870312
:10C4F00043F8405C01376CB186420AD8BDD1D4E91B
:10C500000823D5E90801FFF73EFB002818BF2C4699
:10C51000B3E706462C46B0E7C04A002084DC010899
:10C520004DC1000800000000F8B50D46044620B9D2
:10C5300040F20F211A48F7F7E1FD236923B94FF4C0
:10C5400004711748F7F7DAFD164B5B6898470F46FA
:10C5500006462069C4E908670AF00CFF29460AF07C
:10C5600061FF29460AF054FE0AF0ECFA0AA3D3E967
:10C5700000230AF069FC0AF027F80AF0D5FD32180A
:10C5800047F1000319461046C4E90601BDE8F8402A
:10C59000FFF70CBFAFF300800000000080842E4145
:10C5A00084DC0108C04A002008B5FFF773FE0030A4
:10C5B00018BF012008BD00000A4B10B51B7E0446C1
:10C5C00023B940F24A210848F7F798FD44B1237B8C
:10C5D00033B1002320792373BDE81040FFF794BEE8
:10C5E00010BD00BFC04A002084DC01080A4B10B512
:10C5F0001B7E044623B940F256210848F7F77EFD1A
:10C6000044B1237B33B9012320792373BDE8104063
:10C61000FFF77ABE10BD00BFC04A002084DC0108CD
:10C62000F8B5144E0546337E23B940F26221124814
:10C63000F7F764FD306808B90020F8BD002DFBD085
:10C6400000F021F904460028F6D023689D420CD161
:10C650002F792846FFF774FD2146306800F02AF94B
:10C660003846FFF751FE0120E7E7204600F002F9C7
:10C67000E8E700BFC04A002084DC01082DE9F84348
:10C680002A4D07462B7E8846914623B940F2272142
:10C690002748F7F733FD3846FFF786FF18B900241F
:10C6A0002046BDE8F8833846FFF786FD08B1FFF75E
:10C6B000B7FF2B7E1BB976211D48F7F71FFDAB682E
:10C6C0003020984704460028E9D0302200210BF0A2
:10C6D000E6FB3846FFF7DEFD0646207118B9EB6829
:10C6E00020469847DBE7062803D940211048F7F792
:10C6F00005FD104B214603EBC60253F83630526855
:10C7000023614FF47A73A2605F4300220023C4E9DF
:10C71000062301232760C4E90A892373286800F0EF
:10C7200093F82079FFF7F0FDBAE700BFC04A002078
:10C7300084DC01084CDC010838B50A4C0546227E31
:10C7400022B940F29E210848F7F7D8FC23682BB1A4
:10C75000064C29462046FFF73DFE00B938BDFFF7DD
:10C76000EFFCF6E7C04A002084DC010851C1000854
:10C77000014B187E704700BFC04A002084B070B5DE
:10C7800004AC84E80F00104C237ECBB9251D04AE09
:10C790000FCE0FC533682B600BB90C4B6361236957
:10C7A0000BB90A4B2361E3680BB1A3681BB9084BB3
:10C7B000E360084BA36000F039F801232060237682
:10C7C000BDE8704004B07047C04A0020E1BC0008DA
:10C7D000E97D0108D97D0108134B2DE9F048044695
:10C7E00018680D4600F04FF818B9BDE8F048FFF79B
:10C7F000B7BC0368ABB1D3E908BC5BEA0C0205D057
:10C800001BEB04064CEB0507C3E90867D3E906BC3C
:10C810005BEA0C0205D01BEB04064CEB0507C3E9F1
:10C82000066700F027F8DFE7C04A002010B50820AF
:10C83000FFF7F6FA0446F6F7F3F80023C4E90034EC
:10C84000F6F79AF9204610BD70B505460C200E4645
:10C85000FFF7E6FA044660B10660F6F7E1F8002358
:10C8600063606B68A3601C6004346C60F6F784F945
:10C87000012070BD10B50446F6F7D2F86468F6F7EB
:10C880007BF9204610BD10B50446F6F7C9F82468B8
:10C89000F6F772F9204610BD10B50446F6F7C0F859
:10C8A000236800241BB9F6F767F9204610BD013450
:10C8B0005B68F7E738B50C460546F6F7B1F8D4E9FA
:10C8C00001324BB19A60A2681360F6F755F9204621
:10C8D000BDE83840FFF78EBA6A60F4E770B50446E9
:10C8E000044E451814F8011B3046FFF7FDF9AC4221
:10C8F000F8D170BD71AB010870B515460022C0E9D2
:10C9000001150270C0E90332C0E90522C0E907221F
:10C910004262DDE90412044600F11C06F8F7ACF8A7
:10C9200038B929460748FFF7DFF92B210648F7F702
:10C93000E5FBDDE9042331462046F8F78AF8204676
:10C9400070BD00BF05AB010830AB0108F0B5012692
:10C95000044608270D468DB0694B6A4A3146009659
:10C9600002A8F3F75DFC02A92046F9F799F902A89D
:10C97000F3F7F8FB644BCDE900571A4604210DEBA1
:10C980000700FFF7B9FF0DEB07012046F9F788F91B
:10C990000DEB0700F3F7E6FBEB195C4A01970093F8
:10C9A00004215B4B0DEB0700FFF7A6FF0DEB070122
:10C9B0002046F9F775F90DEB07001027F3F7D2FBC6
:10C9C000EB190093534B04211A46019702A8FFF775
:10C9D00093FF02A92046F9F763F9203502A8F3F77F
:10C9E000C1FB4D4B4D4A00950421019702A8FFF76A
:10C9F00083FF02A92046F9F753F902A8F3F7B2FB27
:10CA00000C23474A00930221464B02A8F3F7E0FBB0
:10CA100002A92046F9F744F902A8F3F7A3FB424B19
:10CA2000424A3146009602A8F3F7FAFB02A92046D3
:10CA3000F9F736F902A8F3F795FB032200230392D6
:10CA40003B4D3C4A3C4902A88DF808300495CDE99D
:10CA50000523CDE90733CDE909330B93F7F7F4FF4D
:10CA600038B929463548FFF73FF920213448F7F710
:10CA700045FB0025304A09A902A8F7F7ADFF02A936
:10CA80002046F9F70DF902A8F3F76CFB2D4B2E4A5F
:10CA90000095022102A8F3F79BFB02A92046F9F7B3
:10CAA000FFF802A8F3F75EFB284B294A0095022104
:10CAB00002A8F3F78DFB02A92046F9F7F1F802A8C6
:10CAC000F3F750FB0121234B234A009102A8F3F70F
:10CAD000A7FB02A92046F9F7E3F802A8F3F742FB07
:10CAE0001E4B1F4A0095022102A8F3F771FB02A911
:10CAF0002046F9F7D5F802A8F3F734FB0DB0F0BDE6
:10CB0000D6DC01082EC80108E9DC01085AE001085A
:10CB100041E00108F7DC010862E001088CE001084F
:10CB200075C70108FEDC010857DD0108B1C701081F
:10CB30008EC7010893E0010831C8010805AB010860
:10CB400030AB0108A8E00108B5C70108E6E001081C
:10CB5000DCC7010821E101084BBB01083DE10108E8
:10CB600004C8010830B504468DB001467A4A6846CB
:10CB7000F8F79BFE794A214603A8F8F796FE784A13
:10CB8000214606A8F8F791FE76492046F8F784FE7C
:10CB900005467548FFF7A8F80123039A02F1100132
:10CBA000914205D011F8010D002818BF0023F7E7C6
:10CBB000002B53D06D48FFF797F85DB36C48FFF733
:10CBC00093F86C4A214609A8F8F76FFE6A48FFF708
:10CBD0008BF808210098FFF781FE6848FFF784F87A
:10CBE00008210998FFF77AFE6548FFF77DF81021C4
:10CBF0000698FFF773FE6348FFF776F80998069AE0
:10CC0000009900F071FE09A8F8F7FEF85E48FFF7FA
:10CC10006BF861E05D48FFF767F85D48FFF764F87F
:10CC20000699009800F0BEFD5A48FFF75DF8042110
:10CC300000980844FFF752FE5748FFF755F81021B7
:10CC40005648FFF74BFE5648FFF74EF8102155485F
:10CC5000FFF744FE4B48FFF747F8D7E71022069846
:10CC60000BF0EAF85049514B002808BF19465048CC
:10CC7000FFF73AF8002D3DD03D48FFF735F83D4A23
:10CC8000214609A8F8F711FE4A48FFF72DF80821B8
:10CC90000098FFF723FE4848FFF726F80821099877
:10CCA000FFF71CFE4548FFF71FF810210398FFF718
:10CCB00015FE4348FFF718F810210698FFF70EFEFF
:10CCC0003048FFF711F80998039B069A009900F085
:10CCD00023FE09A8F8F798F82A48FFF705F806A8F0
:10CCE000F8F792F803A8F8F78FF86846F8F78CF889
:10CCF0000DB030BD2548FEF7F7FF3248FEF7F4FFD0
:10CD0000039A0699009800F091FD2248FEF7ECFF87
:10CD1000042100980844FFF7E1FD2B48FEF7E4FFEB
:10CD200010211E48FFF7DAFD2848FEF7DDFF10212D
:10CD30002748FFF7D3FD2748FEF7D6FF10212648E6
:10CD4000FFF7CCFD2548FEF7CFFF16481021FFF76F
:10CD5000C5FD0C485BE700BFE9DC01088CE0010879
:10CD6000F7DC01082EC8010889DD0108A0DD0108F3
:10CD7000BBDD01085AE00108C1DD0108D2DD010870
:10CD8000E4DD01086EBC01088CDE010804DE010848
:10CD900009DE01083BDE01084DDE010868010020C4
:10CDA00079DE0108980100206FBC010872DD0108DE
:10CDB000ABDE0108C8DE0108DADE0108EDDE01089D
:10CDC0000DDF010856DF010890DF0108FCDF0108D4
:10CDD0007801002013E00108880100202AE0010802
:10CDE00010B5084CD4F82C211AB964210648F7F77D
:10CDF00085F9D4F82C010023BDE81040032220213E
:10CE0000F6F728BBC00000209DE20108F0B51F46E0
:10CE10001446C7B005460E46F122002109A80BF0C2
:10CE20003EF809AA1021384602F08AF920460BF094
:10CE30000BFF07461022002101A80BF030F8102F3D
:10CE40003A46214628BF102201A80BF004F809AA8F
:10CE500005A901A802F0EEF9324605A928460AF014
:10CE6000FAFF47B0F0BD000038B50C4C0C4D94F8FB
:10CE70003230022B0ED1082394F8FF20D4F8001191
:10CE8000012002F013F96B6B00209847042384F80B
:10CE9000303038BDEB6A98470123F8E7C000002026
:10CEA00084F1010810B5044601F0D0F820B92046FD
:10CEB000BDE8104001F0A0B810BD0000054B93F88C
:10CEC000212022B993F8350080F00100704700203E
:10CED000704700BFC0000020F0B570279DB0064627
:10CEE0000D463A46002168460AF0D9FF08212B4634
:10CEF0000DEB010004AC0B4AFFF788FF2B462046E0
:10CF0000094A102108ADFFF781FF94E80F0085E87A
:10CF10000F003A46694630460AF09DFF30461DB084
:10CF2000F0BD00BF8EE2010896E2010808B5054891
:10CF3000FEF7DAFE044A92F80431013382F8043134
:10CF400008BD00BF32E20108C00000200022024BF1
:10CF500083F80421704700BFC000002084B070B582
:10CF60008AB00EAC84E80F00744C4FF49C722546D6
:10CF7000002120460EAE0AF092FF0FCE0FC596E8B4
:10CF8000030014AE85E803000FCE04F118050FC5A9
:10CF900033682B600E9B0BB9694B23600F9B0BB959
:10CFA000674B2360109B23B940F271116548F7F776
:10CFB000A5F8129B23B940F275116248F7F79EF865
:10CFC000119B23B940F279115E48F7F797F8139B4C
:10CFD00023B940F27D115B48F7F790F8A3690BB9CC
:10CFE0000323A361E3690BB90A23E36194F82330B7
:10CFF00013B9012384F8233001F0EEFD94F82430B6
:10D0000013B9012384F8243001F0DEFDA36A0BB9C3
:10D010004D4BA36201F0CCFD06F0F0F9C4F82801F5
:10D020000138033004D963684848984700207DE000
:10D03000032200210120F4F70FFEC4F8300120B9CB
:10D040004FF4D3713F48F7F759F800220421E06903
:10D05000F4F702FE606420B94FF4D5713948F7F750
:10D060004DF800220421E069F4F7F6FDA06420B930
:10D0700040F2AD113348F7F741F8002204210120B6
:10D08000F4F7EAFDE06420B94FF4D8712D48F7F7C2
:10D0900035F84FF48163A4F80A31002384F8363060
:10D0A000012384F80E31FFF763FB05AD68B9A3686F
:10D0B00022690593236807920893E26863680692E1
:10D0C000009395E80F00FFF759FB01F0ABFD2368D3
:10D0D0001F4E0793636806F1A00208932369049624
:10D0E0000693E368DC3605930AAB43F81C2D93E8FE
:10D0F00003008DE8030095E80F0002F023FA019683
:10D10000A3694FF4CD720093124901231248F5F739
:10D110006DFA012805460ED1002303220421D4F81C
:10D120002C01F6F797F9284684F834500AB0BDE888
:10D13000704004B070476368084876E7C00000207C
:10D14000E1BC00089DE2010808E6D3338CE1010848
:10D1500010010020BFE10108BDD20008C7E10108AD
:10D1600010B50F4CD4F82C3123B940F2DD110D4825
:10D17000F6F7C4FF002303220421D4F82C01F6F7AC
:10D1800069F942F21071D4F83001F4F775FF002309
:10D19000D4F830011A46BDE810401946F4F780BDB6
:10D1A000C00000209DE2010838B50E4DD5F83031A1
:10D1B00023B94FF4F7710C48F6F7A0FF0021D5F81A
:10D1C0003001F4F759FF0128044608D10023D5F8AF
:10D1D00030011A461946F4F763FD204638BD002099
:10D1E000FCE700BFC00000209DE2010810B5FFF77A
:10D1F000DBFF68B1074C0023D4F82C01032208217F
:10D20000F6F728F9D4F82C01BDE81040F5F786BBF5
:10D2100010BD00BFC0000020014BD863704700BFA5
:10D22000C0000020002307B502A941F8043D044BCB
:10D230000246D86CF4F78EFE019803B05DF804FB4B
:10D24000C000002038B5FFF7AFFF194D044620B1EC
:10D250006B6818489847002038BD686CF5F79AF855
:10D26000EB698342F7D32146204602F09BF905463D
:10D270000028F0D0047000F0ADFE044618B928462E
:10D2800002F0C8F9E7E70C4A13680133136063B989
:10D290001368013313606360012363700323204626
:10D2A0002370FFF7FFFD6068D6E71368F3E700BF60
:10D2B000C0000020F7E10108DC4A00202DE9F84316
:10D2C0000123604C604F614E84F830300A235E4A7F
:10D2D0004FF0FF310020F6F779F801286AD138685D
:10D2E00043071AD5337833B105F0ECFF002006F080
:10D2F0003DF800233370F6F71DFCF6F73BFC0223E4
:10D3000084F830300023D4F830011A461946F4F777
:10D31000C7FC0020F5F75CFDD8E710F0080521D028
:10D3200033787BB941F2883005F0F8FF18B9A021B5
:10D330004748F6F7E3FE474806F018F80123337034
:10D34000FFF792FD0020F6F773F94FF4FA61D4F875
:10D350003001F4F791FE0028B8D1A7213C48F6F738
:10D36000CDFEB3E710F0200043D03378FBB194F842
:10D370003030042B1BD1DFF8E4802A464146D4F834
:10D380002801F4F729FF0128814610D198F80030D0
:10D39000072B22D1284600F01DFE40B10522C0E92E
:10D3A0000155056180F801900270FFF77BFD0020B8
:10D3B000F6F73EF93378002B88D000F05FFE054683
:10D3C000002883D0032384F830300378052B35D828
:10D3D000DFE803F01219192A2A312A464146D4F807
:10D3E0002801F4F7B7FD0128E1D1404605F0C4FF5C
:10D3F000DDE7F6F71DF969E7D6211548F6F77EFE59
:10D40000FFF732FD62E7FFF759FD38B9284600F013
:10D41000A7FA60B1284600F0EFFDF1E72846FFF7D4
:10D4200041FDFFF70FFFEBE701F0FAF9F1E72846BE
:10D43000FFF738FDE4E700F09DFDEBE76368064881
:10D440009847E7E7C0000020F04A0020E04A0020AB
:10D450009DE20108E1CD00086CE10108E44A0020EA
:10D46000024B93F8FC0001F097BD00BFC000002004
:10D47000F0B585B007460C461546ADF80430FFF709
:10D4800093FE404E28B173683F489847002005B08E
:10D49000F0BD706CF4F77EFFF3698342F6D3FFF7BB
:10D4A000DFFF8442F2D8002D47D1002CEED1214677
:10D4B000384602F077F804460028E7D09DF805309A
:10D4C000002B3DD004230370FFF730FD9DF804309E
:10D4D0003BB10D2304A901F8043D0122204600F0D0
:10D4E0000BFF96F8312096F83230934203D196F82C
:10D4F0003330934217D02023022A18BF00228DF820
:10D500000C3094F8783003A90BBF43F0040343F0C8
:10D5100001038DF80D208DF80D20204684F8783019
:10D52000022200F0E9FE6577204600F053FD054633
:10D5300048B9204602F06EF8A8E7E02DA6D8B6E775
:10D5400002230370C2E70023104A8360136801338B
:10D55000136093B91368013313606B600A9B28460C
:10D560002B6101236B702B7000F058FD38B92846F1
:10D5700000F042FD7368064887E71368EDE76868C6
:10D5800085E700BFC0000020F7E10108DC4A002069
:10D5900066E20108082808BF0120034B83F8230036
:10D5A00083F8FC00704700BFC0000020024B83F8E6
:10D5B000240083F8FD007047C000002008B5FEF786
:10D5C000A3FC014B586508BDC0000020034630B5E0
:10D5D000054C00F11005224618685968083303C24B
:10D5E000AB421446F7D130BD88010020034630B568
:10D5F000054C00F11005224618685968083303C22B
:10D60000AB421446F7D130BD78010020034630B557
:10D61000054C00F11005224618685968083303C20A
:10D62000AB421446F7D130BD68010020034630B547
:10D63000054C00F11005224618685968083303C2EA
:10D64000AB421446F7D130BD9801002010B5044616
:10D65000FFF7BCFF2046FFF7C9FF2046BDE810409A
:10D66000FFF7D4BF30B51025C3B0224CF122002102
:10D6700005A80AF014FC2A46002101A80AF00FFCB4
:10D6800094F8673005AA8DF8053094F8663029467D
:10D690008DF8063094F8653004F178008DF8073085
:10D6A00094F864308DF8083094F863308DF80930C0
:10D6B00094F862308DF80A3094F861308DF80B30B0
:10D6C00094F860308DF80C3001F03AFD052305AA7E
:10D6D00004F1980101A88DF8043001F0ABFD062398
:10D6E00005AA04F1880101A88DF8043001F0A2FD1B
:10D6F00043B030BDC00000200246024B00685168B4
:10D7000003C37047180100200246024B00685168AD
:10D7100003C3704720010020034630B5054C00F1DB
:10D720001005224618685968083303C2AB421446F4
:10D73000F7D130BD28010020034630B5054C00F17B
:10D740001005224618685968083303C2AB421446D4
:10D75000F7D130BD38010020014B83F8220070471B
:10D76000C0000020014B83F831007047C00000204A
:10D77000014B1864704700BFC000002013B500249F
:10D78000064B02AA42F8044D054993F8FD00FEF746
:10D790004BFE2146019802B010BD00BFC000002022
:10D7A00051D9000830B50430C7B00D46FFF706FF69
:10D7B0001C4B0DF1050203F10C0153F8040B8B42D5
:10D7C00042F8040BF9D11B880124138000238DF843
:10D7D0001330022309AA102128468DF8043001F0E5
:10D7E000AFFC09AA05A901A801F024FD05A8FFF7CF
:10D7F0001DFF09AA102128468DF8044001F0A0FC65
:10D8000009AA05A901A801F015FD05A8FFF71EFF4B
:10D810001022054B83F8214083F8202083F8502004
:10D8200047B030BD23E20108C000002030B504300D
:10D83000C7B00C461546FFF7C1FE294B0DF1050296
:10D8400003F10C0153F8040B8B4242F8040BF9D19D
:10D850001B882046138000238DF8133002230124F7
:10D8600009AA10218DF8043001F06AFC09AA05A963
:10D8700001A801F0DFFC05A8FFF7D8FE09AA1021D6
:10D8800028468DF8044001F05BFC09AA05A901A80F
:10D8900001F0D0FC05A8FFF799FE032309AA05A90A
:10D8A00001A88DF8043001F0C5FC05A8FFF79EFE25
:10D8B000042309AA0DEB030005A98DF8043001F03B
:10D8C000B9FC05A8FFF7A2FE1122064B83F8214000
:10D8D00083F8202083F8502083F8084147B030BDFA
:10D8E00023E20108C000002038B50D461446FFF7BA
:10D8F00003FF2846FFF708FF2046FFF70DFF2046ED
:10D90000FFF71AFF0022034B83F82120102283F82F
:10D91000202038BDC000002070B50E4615461C46BC
:10D92000FFF7EAFE3046FFF7EFFE2846FFF7F4FE6A
:10D930002046FFF701FFBDE870400022034B83F84B
:10D940002120112283F82020FFF78CBEC000002088
:10D9500028B1836A012B01D1007B704700207047FA
:10D960002DE9F04F054689B010B10378012B03D0A3
:10D970001C218348F6F7C2FB6B691BB91D21804847
:10D98000F6F7BCFB6B691B78042B05D0022B03D088
:10D990001E217B48F6F7B2FB00267A4C08AA94F8C1
:10D9A000FF3094F8FD800293D4F8003142F80C6DFA
:10D9B0007549404694F8FCB094F8FEA00393FEF736
:10D9C00033FD074638B9284600F0BCFB012738462E
:10D9D00009B0BDE8F08F059B8BB1FEF7E7FC059918
:10D9E000042904D9284600F0E5FB0027EFE7674843
:10D9F00041434FF47A70B1FBF0F0F5F771F9AB6881
:10DA00000133012BAB600FD1D4F8F03068690133DA
:10DA1000C4F8F03094F80931013384F8093100F08A
:10DA200025FC686900F088FC636D6E697360D4F84A
:10DA3000F030738194F80531002B61D0002384F815
:10DA40000531337A43F00403337294F8FC303846DE
:10DA500086F87C3001F028F986F87D0094F80E21D4
:10DA60004FF47A7312F00F0208BF012200265A43C6
:10DA700007AB019306AB0093394602F57A736869E8
:10DA8000069600F061F9074600289CD0F4F7D0FF15
:10DA9000E860069870B1314600F000FCFFF756FAD6
:10DAA000069B1B78052B04BF012384F80531002356
:10DAB00084F80731069800F0B5FBDDE9060100F0B7
:10DAC0005FFE069BFBB11B7A13F004032FD0B9460F
:10DAD00094F80C31AB606A691278022A02D194F88A
:10DAE0000C21AA6000F0E2FA064610BB8C21244803
:10DAF000F6F704FB264B274A8D2121480AF058F8F7
:10DB0000A6F87A30A1E79946ECE73146686898476D
:10DB10006420F5F7E5F8304600F0D8FA94F80C31B7
:10DB2000AA689A42BFF453AF032333705DE7994666
:10DB3000D1E78022696918300AF08DF900229DF83A
:10DB400008300699F373039BC6F89810297872720F
:10DB5000336194F83530C6F8802033752B6986F828
:10DB60000CB086F80D8086F80EA03270717086F8C1
:10DB70000890002BC9D1304600F0C2FACEE700BFB2
:10DB8000F3E20108C000002051D9000840420F0014
:10DB900038E30108E5E201082DE9F04385B00646C7
:10DBA0000C468DF80F202BB101220DF10F01002042
:10DBB00005F050FFF4F73CFF1C4B1D4DDFF878805B
:10DBC0009DF80F1007469B6A2046984741F288321D
:10DBD0002946D8F82801F4F7BDF928B32B78012B92
:10DBE0001DD12846AC6805F0C7FB4FF47A70A4EB52
:10DBF000070909FB000009F0BDFB01463046FEF7AE
:10DC000093FC9DF80F10CDE90049D8F800503B4631
:10DC100032680848A847204605B0BDE8F08328468A
:10DC200005F0AAFB0024F6E70446F4E784F10108B6
:10DC3000F44A0020E4E30108C00000202DE9F84F79
:10DC4000394E9846736B0546894614464FF47A7AE6
:10DC50009847DFF8DCB0354F0AFB05F202F59C323D
:10DC60008032B2FBFAF23249D7F82801F4F772F9A0
:10DC700020B9336B98474FF0FF302FE09BF800300E
:10DC8000072B07D1584605F077FB4FF47A6505F06E
:10DC900065FEE1E7032B366B22D1DBF804502879CF
:10DCA0002968844228BF0446484622460AF0D3F831
:10DCB0003F6895F90830B5F90620A9881D48B8478E
:10DCC000B8F1000F05D0EB88A8F800302B7A88F85F
:10DCD0000230174805F050FBB0472046BDE8F88FEA
:10DCE000042B0BD1124805F047FBB0473C68F4F712
:10DCF0009FFE01461048A0470020EFE7052B0AD100
:10DD00000B4805F039FBB0473C68F4F791FE01463B
:10DD10000A48A047AFE7EC210948F6F7EFF90448B5
:10DD200005F02AFBB047A6E784F10108C0000020F7
:10DD3000004B002049E3010873E301088BE301086D
:10DD4000A1E30108000000002DE9F04FC9B00F4623
:10DD5000914608A9FF2282469846539E01F074FC22
:10DD6000029018B9002049B0BDE8F08F7C4C3A68A9
:10DD700094F8FC1094F8FE5008468D429ABF4D1B53
:10DD8000EDB20025D4F800B00592049101F0B0F88E
:10DD9000039094F8FD0001F0C1F8DDE90412039B43
:10DDA00000907048D8473A682846D4F800B00392EB
:10DDB00001F09EF8039A034629466B48D84794F829
:10DDC000FF10D4F800210846D4F800B00492039163
:10DDD00001F08EF8DDE9031203466448D8470121BB
:10DDE000504600F05BFA94F8FD3094F8FC20396856
:10DDF000002001F05BF90023029A08A93846FFF7DA
:10DE0000CBFE04460028ADD09AF8783013F0050F09
:10DE10000BD013F0040F0CBF00220222504B93F8DA
:10DE20003210914218BF83F83220FF22002108A847
:10DE30000AF035F82A4608233968012001F036F93E
:10DE4000A9F1140008F05CFE41A3D3E9002308F017
:10DE5000D1FE09F069F9054609F2AB2008F050FE41
:10DE60003DA3D3E9002308F0C5FE09F05DF907469C
:10DE7000A8F1140008F044FE35A3D3E9002308F00C
:10DE8000B9FE09F051F9A0F1140ABA4594BFC5EBE7
:10DE90000A0AC5EB070A4FF47A7707FB05F18146BA
:10DEA000B1FBF7F107A80794F4F7DAFEFF22334637
:10DEB00008A95046FFF7C2FE421C05463FF452AF88
:10DEC0000028274917DD0F68F4F7B2FD2346024604
:10DED00029462748B8470EB10123F3700023529A10
:10DEE0009D42136005DDE9B208A801F01FFF529BB7
:10DEF0001860012037E791F8FF200823D1F80011BE
:10DF0000012001F0D3F807FB09F107A8B1FBF7F1F5
:10DF10000794F4F7A5FE08F2AB2008F0F1FD0EA37C
:10DF2000D3E9002308F066FE09F0FEF83346FF222D
:10DF300008A9A0EB0900FFF781FE431C05463FF44A
:10DF400011AF0028CADD002EC8D00223C5E700BFEC
:10DF50000AD7A3703D0AEF3FA4703D0AD7A3F03F54
:10DF6000C00000205BE401088DE40108B3E401086F
:10DF7000D9E4010870B5C2B001ABFF2202A94FF489
:10DF80007A60FFF75BFE061E1EDD114DF1B26A6D71
:10DF900002A801F09BFC0446B0B10378052B01D028
:10DFA000032B0DD10021204600F078F9204600F027
:10DFB00039F92046019900F0E3FB2B6C204613B998
:10DFC00001F028FB00E09847304642B070BD00BF2A
:10DFD000C000002038B5074B0546DB68182098477D
:10DFE000044620B11422002109F059FF6561204642
:10DFF00038BD00BFC000002010B5044650B14069D4
:10E0000001F008FB00236361034B2046BDE810408C
:10E010001B69184710BD00BFC0000020037807B57A
:10E02000052B4FF0000302A941F8040D06481A46DB
:10E030000CBF806C406CF3F733FE431E58425841CE
:10E0400003B05DF804FB00BFC000002007B50378F3
:10E0500002A941F8040D0848052B4FF000024FF0CB
:10E0600001030CBF806C406CF3F71AFE431E58424C
:10E07000584103B05DF804FBC000002037B5002212
:10E0800002AC094D44F8042D2146A86CF3F762FF59
:10E09000019B33B995F836201AB92146686CF3F71D
:10E0A00059FF019803B030BDC0000020064B10B5E9
:10E0B000DB68A0209847044618B1A022002109F08F
:10E0C000EEFE204610BD00BFC000002070B5044623
:10E0D00090B1D0F88000094D08B12B699847D4F869
:10E0E000980020B101F096FA0023C4F898302B690B
:10E0F0002046BDE87040184770BD00BFC00000203A
:10E100001FB50E4C0190E06CF4F756F9024638B991
:10E1100003A9E06CF3F71EFF10B10398FFF7D6FFD9
:10E12000002301A91A46E06CF3F7BAFD20B940F2CA
:10E1300081110348F5F7E2FF04B010BDC0000020D4
:10E14000A1E30108F8B50423437003780546032BC7
:10E150000ABF144B0469DC6BFFF7A8FF0646B0B991
:10E160004FF4C8711048F5F7C9FF104B104A40F240
:10E1700091110D4809F01CFD31466868A0473046F2
:10E18000FFF7A4FFFA20F4F7ABFD3846F8BD0127EE
:10E190002B7807704370002CEED1FFF7B1FF2046BB
:10E1A000F4E700BFC0000020A1E3010841E301083B
:10E1B00017E40108F8B503780646032B08BF154B92
:10E1C0000F460CBFDC6B0469FFF770FF0546B0B962
:10E1D00040F2A9111048F5F791FF104B104A4FF487
:10E1E000D5710D4809F0E4FC29467068A04728461F
:10E1F000FFF76CFFFA20F4F773FD0120F8BD02234E
:10E200000370337847604370002CEDD1FFF778FF3F
:10E210002046F3E7C0000020A1E3010841E3010824
:10E2200033E4010808B5104A10B1002382F809311F
:10E2300092F82230BBB192F8093192F80A118B4260
:10E2400011D95B1A92F80B1193FBF1F201FB123317
:10E250004BB900F0C9FC30B900F0D4FC18B9BDE8E6
:10E26000084000F0DFBC08BDC00000200A4B93F856
:10E2700022207AB1027A42F00102027293F8092157
:10E2800093F80A319A4205D9037A43F002030372E4
:10E29000FEF74CBE704700BFC00000207047000072
:10E2A000064A1378FD2BDFBF00780549C8540133B7
:10E2B000DABF012013700020704700BF0D4C002012
:10E2C0000E4B002038B10078032803D0431F58427A
:10E2D0005841704701207047052307B502A800F890
:10E2E000013DFFF7DDFF0348FFF7DAFF03B05DF8FC
:10E2F00004FB00BF0C4B0020037A70B51B09D61835
:10E3000004460F2E00F10C001546184409DC09F0F4
:10E31000A2FD0120237A05EB131565F30713237281
:10E3200070BDC3F10F0209F096FD237A002043F07F
:10E33000F0032372F4E7000037B5114C054622784C
:10E3400022B11049FFF7D8FF002323700E4C94F838
:10E3500007213AB1082302A901F8043D0122284609
:10E36000FFF7CAFF94F8083143B140F2011302A944
:10E3700021F8043D02222846FFF7BEFF03B030BD5E
:10E380000D4C00200E4B0020C00000200122044B49
:10E3900000F00F0083F80E0183F80721704700BFDB
:10E3A000C0000020000000002DE9F04F17461E4677
:10E3B0004FF000088BB0CDE901019DF85050C04CE2
:10E3C000A84502D30BB0BDE8F08F16F8083006EB75
:10E3D000080A013B1F2B00F2CE81DFE813F020007A
:10E3E000CC012C006601DC00C0001E01600166014A
:10E3F0004701CC017901940092019501CC01CC0137
:10E40000CC01CC01CC01CC01CC01CC01CC01CC01A4
:10E41000CC01CC01CC01CC01CC01CC01B701A5EBE6
:10E420000803DBB2012B4FF0000920D084F80891DB
:10E430004FF002091BE04FF00009A5EB080B5FFA53
:10E440008BFB8DF81C9009F104035B4503DA1AF885
:10E450000930032B0DD0B9F1000F08D003230AA80F
:10E4600000F8083DFFF71CFF07A8FFF719FFC1449C
:10E470008AE00AEB09014B7809F102001A095044BD
:10E4800003F00F03059104920393FDF75DFD0599D9
:10E49000049A097909F10509062AC1F3021C5FFAF9
:10E4A00089F901F00F01039B21D90F2A05D19DF8AD
:10E4B0001C2042F002028DF81C205A1E062A19D98F
:10E4C0000F2B05D19DF81C3043F004038DF81C3050
:10E4D00009B184F80C11BCF1000F0ED100F06EFCF4
:10E4E0009DF81C3043F001038DF81C30ABE784F835
:10E4F000FC20DCE784F8FD30E4E7BCF1060FA2D194
:10E500004FF6FF70EAE7A5EB0803DBB2052B40F2FC
:10E510002F810AF10100FDF70DFD9AF90530002168
:10E52000002B18DB62A3D3E9002312184B4191465C
:10E530009A46002394F80E2119EB02004AEB0301DE
:10E54000022F02D1013041F10001019BC3E91C01FE
:10E550004FF006098BE758A3D3E90023E5E706232C
:10E560000AA800F80C3DFFF79BFE029B0DF128095D
:10E5700003F01F0309F8083D5248FFF791FE484693
:10E58000FFF78EFE08F101095FFA89F9C8453FF4EB
:10E5900019AFC84614E7A5EB0803DBB2042B40F221
:10E5A000E780DAF80120DFF824910892D2B2C2F3B2
:10E5B000021384F8FE3099F80030C2F30302052AF2
:10E5C00043F0040394BF43F002036FF341030DF1E2
:10E5D000210098BF84F8FF2089F800304FF0640ACA
:10E5E000FDF7AAFC0AFB00FA504605F0B9F978B12C
:10E5F00099F80030C4F800A143F00103012289F822
:10E600000030314B1A70FFF767FE4FF005092EE717
:10E6100099F8003060F30003F0E7A5EB0803DBB2E4
:10E62000052B40F2A580534653F8010F9AF80310CA
:10E630001A799AF80430090241EA03419AF8023043
:10E640000890194364239AF8010059438DF8242057
:10E6500000F04CFB07238DF818000AA800F80C3DC9
:10E66000FFF71EFE06A8FFF71BFE71E7A5EB0803E8
:10E67000DBB2042B7CD96421DAF80100030A594388
:10E68000C0B200F065FB0A238DF81C000AA800F850
:10E69000083DFFF705FE07A8FFF702FEB5E79AF869
:10E6A000010000F00F00FFF771FE08F102096BE7AF
:10E6B0006E3DD512000000006F3DD5120000000035
:10E6C000C0000020CD0100200D4B00200C4B00208D
:10E6D000A5EB0803DBB2012B4AD001239AF80120F5
:10E6E0000AA8110902F00F0203FA01F1934084F81D
:10E6F0000B310C2384F80A1100F8083DFFF7D0FD18
:10E7000096E608F103093FE7A5EB0803DBB2012B0E
:10E710002ED0A3689AF8019098470122174B8DF8E4
:10E720001C20C3E900014FEA19130A3302FA03F36C
:10E73000C4F8183109F00F03C4F81C310F230AA8DC
:10E7400000F8083DFFF7ACFD07A8D7E7A5EB0803E5
:10E75000DBB2012B0CD09AF801300BB1022B07D1A0
:10E7600094F833209A423FF463AE84F833305FE686
:10E770004FF000097BE6C14608E700BFD00100204A
:10E7800030B585B003910446174B30B91B7803B3FD
:10E7900005B0BDE83040FFF79FBD00259DF90E1084
:10E7A0009DF80F201D70FFF78DFD90B10F48237A63
:10E7B00090F822502DB113F0010518BF012580F803
:10E7C00006511B0907D0009304F10C032046FFF704
:10E7D000EBFD05B030BD637F002BFAD1237F002B0A
:10E7E000F7D00093A36EF1E70D4B0020C00000208E
:10E7F00010B5044678B1836A012B0CD1C36A1BB9EA
:10E8000010210648F5F77AFCE36A587802288CBF95
:10E810000020012010BD0020FCE700BF04E5010836
:10E820002DE9F04F054689B018B10378033B012B61
:10E8300003D92221C148F5F761FC6B690BB11B7844
:10E840001BB12321BD48F5F759FC0027BC4C94F8B7
:10E85000FF3094F8FD800393D4F8003194F8FCB0B5
:10E86000029394F8FEA000F0AFF900F0B5F908AA01
:10E8700042F80C7DB3494046FDF7D6FD064620B967
:10E880002846FFF75FFC01260AE0059BA3B1FDF7D0
:10E890008DFD0599042907D92846FFF78BFC3E46D4
:10E8A000304609B0BDE8F08FA74841434FF47A7075
:10E8B000B1FBF0F0F4F714FAAB6894F820200133C0
:10E8C000102AAB602DD1012B09D1D4F8F0300133DF
:10E8D000C4F8F0309D4B5B699847A4F8E800B4F8A1
:10E8E000E8300133A4F8E830002707AB019306AB0A
:10E8F0000093314641F2707341F28832686994F8AE
:10E90000FF90069784F8FF70FFF71EFA0646A8B935
:10E910002846FFF717FC069800F07CFE84F8FF906D
:10E92000B1E7112A05D1636989489847A4F8E8003E
:10E93000DAE750218148F5F7E1FBD5E7069A84F83C
:10E94000FF9012B11378012B06D02846FFF7FAFB8F
:10E95000069800F05FFEA3E794F82030102B40F0FB
:10E96000A0801023002784F85030069BDA68626587
:10E9700003F15302002F00F0A3801121DFF8D4C16E
:10E9800084F8501003F1630E67461068516808322E
:10E9900003C77245BC46F7D1DFF8BCC103F12302BF
:10E9A00003F1330E674610685168083203C7724599
:10E9B000BC46F7D1DFF8A4C103F1330203F1430EE3
:10E9C000674610685168083203C77245BC46F7D1E4
:10E9D000DFF88CC103F1430203F1530E6746106860
:10E9E0005168083203C77245BC46F7D1544F9A6844
:10E9F000BA631A7CC2F3030287F8FF201A7CC2F3C1
:10EA0000021287F8FE20587CFFF7C0FC002206980F
:10EA100097F83110437C1230012B98BF87F80721FB
:10EA200011F0FD0F18BF87F83120C7E93D22C7F864
:10EA3000F02087F8322087F8332000F0E1F9FDF765
:10EA4000B5FC012384F83530FFF730FB8022074600
:10EA50006969183009F0FFF90023069AC7F8803079
:10EA6000C7F8982094F835207B723A753B709DF872
:10EA70000C202B78FA737B70029AE36B87F80CB04A
:10EA800087F80D8087F80EA03A61002B52D03946E6
:10EA9000686898476420F4F723F93846FFF716FBB7
:10EAA000FEE6112B07D192F82270002F3FF459AFE8
:10EAB00084F8503059E77D212048F5F71FFB54E7D3
:10EAC0001021DFF890C084F8501003F1630E674600
:10EAD00010685168083203C77245BC46F7D1DFF8A9
:10EAE00078C003F1230203F1330E674610685168C2
:10EAF000083203C77245BC46F7D1DFF860C003F1A6
:10EB0000230203F1330E674610685168083203C7C9
:10EB10007245BC46F7D1DFF848C003F1230203F188
:10EB2000330E674610685168083203C77245BC4609
:10EB3000F7D15BE73846FFF7E3FAB1E604E50108F1
:10EB4000C0000020F1E7000840420F0084F10108F6
:10EB50001801002098010020880100207801002081
:10EB600068010020437882781B02007843EA024360
:10EB700003430A20B3FBF0F07047000038B50446A9
:10EB800081B10D7884B1A36A012B0DD1E36A1BB961
:10EB90005D210648F5F7B2FAE36A5878431B5842FC
:10EBA000584138BDFF25EDE70020FAE794E501085C
:10EBB000044B93F8252083F8FF209A6AC3F80021BC
:10EBC000704700BFC0000020024B93F8242083F858
:10EBD000FD207047C0000020024B93F8232083F8EB
:10EBE000FC207047C0000020054B93F8242093F8C8
:10EBF000FD1091423ABF012083F8FD2000207047AC
:10EC0000C0000020064A92F8FC3092F82310994286
:10EC10003DBF03F1FF33012082F8FC300020704734
:10EC2000C000002010B5FFF7C3FF0120FDF784FDF1
:10EC30005023164C01212370002322461448637090
:10EC4000FDF71CFD18B932211248F5F757FA502389
:10EC50000121114A1148A370E170FDF70FFD18B9A9
:10EC600036210C48F5F74AFA5023237102230C4A47
:10EC700001210C486371FDF701FD28B9BDE8104082
:10EC80003A210448F5F73ABA10BD00BFB45200204B
:10EC9000043F0D0094E50108B6520020CC3F0D0062
:10ECA000B852002094400D00836A10B5012B044631
:10ECB00008D1C36A1BB94B210348F5F71FFAE36A71
:10ECC000587810BD0020FCE794E5010807B502A9BB
:10ECD00001F8010D0448FDF77DFB08B1FDF7A0FC2C
:10ECE00003B05DF804FB00BF7DEB00082DE9F041A7
:10ECF0004FF47A769046B1FBF6F6C8F30317052F6A
:10ED0000044630468CBF002701274FF00005FDF771
:10ED10004BFC18B10F2C8CBF0020012067F30005BD
:10ED200060F3410505F00303032B0CD12046FFF7E8
:10ED3000CDFF064B012103EB4402547003F814800D
:10ED40003046FDF79BFC2846BDE8F081B452002018
:10ED50000F282DE9F04105460F461FD8164B03EB4F
:10ED600040035C78231A5C425C414FF47A78B7FB2D
:10ED7000F8F0FDF719FC4FF0000360F3000364F3B3
:10ED8000410303F00303032B064609D04FF00000B4
:10ED900066F3000064F34100BDE8F0810024E4E77D
:10EDA0002846FFF793FF044A012102EB450208FBC6
:10EDB00007F0FDF763FCE9E7B4520020002373B5C8
:10EDC000044602AD0D4E05F8013D9DF807300F2BAE
:10EDD00001D902B070BD29463046FDF7FBFA18B1E3
:10EDE000E30708D5FDF702FC9DF8073064080133FE
:10EDF0008DF80730E9E7FDF7DFFBF5E77DEB00086D
:10EE000038B504460320FFF761FF0420FFF75EFFDB
:10EE10000520FFF75BFF0620FFF758FF0720FFF7ED
:10EE200055FF2046FFF79EFE0546FDF7BDFB48B1A6
:10EE30005023294A01219371032306325370284637
:10EE4000FDF71CFCE01CFFF78DFE0546FDF7ACFB53
:10EE500048B15023204A0121137204230832537011
:10EE60002846FDF70BFCA01DFFF77CFE0546FDF7CD
:10EE70009BFB48B15023184A0121937205230A32A3
:10EE800053702846FDF7FAFB04F10900FFF76AFE0C
:10EE90000546FDF789FB48B150230F4A0121137342
:10EEA00006230C3253702846FDF7E8FB04F10C00F2
:10EEB000FFF758FE0446FDF777FB58B15023064A8A
:10EEC000204693730723D3730121BDE838400E32E7
:10EED000FDF7D4BB38BD00BFB45200200738C0B224
:10EEE00005289ABF014B185C0820704747E50108C8
:10EEF00007289ABF014B185C002070474DE50108B8
:10EF0000052804D90628034818BF00207047024886
:10EF1000704700BF90D0030048E80100072810B5F3
:10EF2000044604D94FF49E710348F5F7E7F8034B04
:10EF300013F9240010BD00BF94E5010858E501084D
:10EF4000142810B5044613DD40F241111148F5F7BD
:10EF5000D5F8062C14DD082C14DD0A2C14DD0C2C3D
:10EF600014DD0E2C14DD152CB4BF0020082010BDBC
:10EF7000022803DD0428ECDC0620F8E70720F6E78A
:10EF80000520F4E70420F2E70320F0E70220EEE793
:10EF90000120ECE794E5010808B50F280DD8DFE85B
:10EFA00000F0181818081A1A1A0A0A0C0C0C0C0C83
:10EFB0000C0A732008BD0020FCE740F27B110748D3
:10EFC000F5F79CF8064B074A4FF4BE71034808F06A
:10EFD000EFFD3320EEE7DE20ECE700BF94E501080B
:10EFE00065B8010878E501082DE9F0468DB0924634
:10EFF00099462A4A149B074693420C4608D0284A51
:10F00000934203D0A6212748F5F778F8002600E0C0
:10F010000126254DEB6A98472046EB689847012F5B
:10F020004FF0000422D108230A22CDE90132AB6956
:10F0300031460B93CDE90877CDE90644CDE9044488
:10F04000039400943B464A4602200B9EB04721465B
:10F05000FF2004F0F5F9082004F0E8F93421392004
:10F060002B6C0B930DB0BDE8F04618474FF47A6354
:10F070000127CDE907430823CDE90173EB69CDE909
:10F0800005440B93CDE9034722465146CDF8009045
:10F09000334602200B9CA0473946D9E790D00300A5
:10F0A00048E80100D9E5010884F101082DE9F341A0
:10F0B0000446104615460E469846FFF721FF0746C0
:10F0C0002846FFF715FFC5B21DB9C5210948F5F758
:10F0D00015F864B94046FFF721FF024600972B461A
:10F0E00031462046FFF780FF02B0BDE8F0810022E4
:10F0F000F4E700BFD9E501080A68036853400360DC
:10F100004A684368534043608A6883685340836019
:10F11000CA68C3685340C36070470B6810B5146871
:10F120006340036054684B686340436094688B6835
:10F1300063408360CB68D2685340C36010BD000059
:10F14000A1F11003DBB2102B2DE9F0470C46154658
:10F1500008D84FF0010909FA03F303F0013323F053
:10F1600080732BB90023FF2085F8F030BDE8F087CD
:10F170000A460146284608F06EFE04F11C0E4FEACE
:10F180008E0E5FFA8EFE4FEA1E13013B85F8F030BB
:10F1900023462749B3FBF4F204FB1232E81812F0BD
:10F1A000FF0210F804AC10F803CC10F8027C10F841
:10F1B000016C32D111F80C804FEAD91289EA0808A3
:10F1C00011F807C08F5D11F80A604FEA420A5244F5
:10F1D000C24602EBC20282EA49025FFA82F91A1BB6
:10F1E000D2B215F802802A448AEA080A05F803A078
:10F1F00092F8018004338CEA080C80F801C092F880
:10F2000002C0DBB287EA0C078770D2789E4586EA97
:10F210000206C670BED80020A8E7182CDFD9102A35
:10F2200001BF11F80AA011F80CC0CF5D8E5DD6E7C2
:10F230001BE801082DE9F04F92F8F030A1B01A91C7
:10F240001892002B00F05D8101461CA8FFF765FFB6
:10F250004FF00108AC4CAD4DAD4E189B9DF875E0DC
:10F2600003EB081319939DF870309DF87AA0009372
:10F27000009A9DF87F90A05C9DF8742014F80A1005
:10F280000192019F9DF87920E75D02920697029F07
:10F290009DF87E20E75D03920797A25C9DF8787049
:10F2A000049208979DF873209DF87D70059214F8DC
:10F2B000093014F80EC0A25C09979DF872700A9785
:10F2C000E75D0B979DF877700C97E75D0D97089FAA
:10F2D000E75D0E97099FE75D0F979DF87C7010978B
:10F2E0009DF8717011979DF876701297E75D1397EE
:10F2F0009DF87B701497E75D1597109FE75D169753
:10F30000119FE75D1797189F97F8F07047453ED813
:10F310008DF870009DF818008DF872108DF874004B
:10F320009DF82C109DF838008DF87A108DF8780033
:10F330009DF810109DF858008DF876108DF87C001F
:10F340009DF84C109DF81C008DF87E108DF875000E
:10F350009DF854109DF83C008DF87F108DF87900D1
:10F360009DF834109DF85C008DF87B108DF87D00C1
:10F370008DF877201A98199A1CA98DF871C08DF80C
:10F380007330FFF7CAFE002021B0BDE8F08F81EA9C
:10F3900003071B97009F434015F807B01B9F80EAA7
:10F3A0000C008BEA070716F80EB081EA0C0187EA19
:10F3B0000B078DF8707015F80E707B4016F80A7008
:10F3C0007B408DF8713015F80A30584016F8093036
:10F3D0005840009B8DF8720016F803C0049B8CEA1D
:10F3E000010115F809C0534081EA0C018DF8731032
:10F3F00001991CA8695C4B400299715C4B408DF8E7
:10F400007430069B5A40029BEB5C5A40039BF35CB2
:10F410005A408DF87520DDE906325340039AAA5C04
:10F420005340059AB25C53408DF87630079A049B9E
:10F430005340019AB25C5340059AAA5C53408DF840
:10F4400077300D9A0B9B5340089AAA5C5340099A57
:10F45000B25C53408DF87830DDE90D325340099AA3
:10F46000AA5C53400A9AB25C53408DF87930DDE9CA
:10F470000E3253400A9AAA5C53400C9AB25C534035
:10F480008DF87A300B9B0F9A5340089AB25C534028
:10F490000C9AAA5C53408DF87B30159A139B53400D
:10F4A000109AAA5C5340119AB25C53408DF87C309C
:10F4B000DDE915325340119AAA5C5340129AB25CAE
:10F4C00053408DF87D30DDE916325340129AAA5C24
:10F4D0005340149AB25C53408DF87E30179A139BB8
:10F4E0005340109AB25C5340149AAA5C1999534045
:10F4F0008DF87F30FFF700FE08F101035FFA83F813
:10F50000ABE6FF2040E700BF1BE801081BE601084F
:10F510001BE701080068704782B0034660B16A4685
:10F5200059680068013B03C207221DF8021012F15E
:10F53000FF3203F8011FF8D202B070470FB404B0D5
:10F540007047000030B585B06D4685E80F00104C5F
:10F5500095E80F0084E80F0004F1100208A903C920
:10F5600082E803000BB90B4BE360A3680BB9094BAE
:10F57000A36063680BB1236833B9A3680648984752
:10F58000064B6360064B23600123237605B030BD34
:10F59000104C00203DF5000891E90108E97D0108C3
:10F5A000D97D01082DE9F041184D80462B7E0E468D
:10F5B0001BB973211648F4F7A1FDDE2E03D974217F
:10F5C0001348F4F79BFD2B6880209847044680B1D0
:10F5D0008022002108F063FCB8F1000F12D08EB138
:10F5E0002B6830469847074630B920466B689847E5
:10F5F0003C462046BDE8F0813246414608F02BFCEF
:10F600002677A76600236370F3E700BF104C002045
:10F6100044E9010870B50A4C0546237E1BB98F21C9
:10F620000848F4F76BFD55B1A86E636810B19847B0
:10F630000023AB6663682846BDE87040184770BD7C
:10F64000104C002044E901082DE9F0479C4B174677
:10F650001A7E92B005460E4698461AB9A7219948D7
:10F66000F4F74CFD032F01D80024D8E02A786B78FA
:10F6700043EA421333702B78022B02D0042B40F064
:10F680008D800023042F8DF82630EDD06B687370C9
:10F690006B681B0AB370EB88F370EB7933716B689E
:10F6A000CDF822309DF82630002B40F0C180052F88
:10F6B000DAD006242A7AC2F3400302F001019B014A
:10F6C00043EAC11343EA1213C2F3800243EA42132E
:10F6D000737195F808904FEA1919631C9F42C3DDB6
:10F6E0006A89DBB232556A890234120AF254D8F8B8
:10F6F00010301A886B899A4204D040F24711714841
:10F70000F4F7FCFCD8F81420D8F8103011781B68F6
:10F7100010290A930DD902930DF1220301930123BD
:10F72000297A009358320023090905F10C0000F0F2
:10F73000E5FCB9F1000F0BD004EB090A574593DB48
:10F7400030194A4605F10C0108F085FB5FFA8AF48E
:10F750002B7F002B77D0BC4286D26B7F04F101094E
:10F7600033556A7F5FFA89F9D8F81430002A68D1D6
:10F7700058330693AB6E06A907932B7F06EB09005F
:10F78000ADF8203000F0ACFB4844C4B2A7425AD2D6
:10F7900040F275114B48F4F7B1FC65E7032B01D03B
:10F7A000052B01D101236DE7002B3CD1082F7FF6FB
:10F7B0005BAFD8F81440701C224652F8083FC6F8D8
:10F7C000013053684360FFF7A7FE102F7FF64CAF60
:10F7D000224652F8103F06F10900C6F80930536876
:10F7E0004360FFF799FE122F7FF63EAFB4F89830D2
:10F7F00006A97374B4F8983005A81B0AB3741323D0
:10F800002834CDE90646ADF8203000F033FB162F42
:10F810007FF62AAF1724059BC6F813306B66204687
:10F8200012B0BDE8F087D8F80C30274898471BE79E
:10F8300040F23D112348F4F761FC4FF00009052424
:10F840004BE7883395E7E31C9F427FF70DAFD8F86D
:10F8500014301A78102A0DD1783306A905A8CDE9FD
:10F860000636ADF8204000F06CFA059B33510434A5
:10F87000E4B2D4E7112A1DD103F1780268330B9367
:10F880000DF122030F930A9B0BA91093B5F87A3060
:10F8900005A8ADF8443095F87C300C928DF84630D0
:10F8A00095F87D300D968DF84730ADF8384000F072
:10F8B00080FADAE74FF4CC710248F4F71FFCAEE7A8
:10F8C000104C002044E901081BE901082DE9F04F24
:10F8D0008F4DA3B02B7E06460F46904623B940F2CB
:10F8E000A5118C48F4F70AFC022F2CD92B68802034
:10F8F0009847044630B9EB6887489847204623B0BC
:10F90000BDE8F08F8022002108F0C9FA33785B0946
:10F9100023703278072B02F00302627003D1EB6888
:10F920007E4898470CE0B8F1000F00F0EF81012B02
:10F9300040F0C581AB687A48F3E74246794898477A
:10F940006B68204698470024D8E701F18802A0E1BF
:10F95000F3465068227A4FEADC1E6EF300024FEA4B
:10F960005C1E6EF382024FEA1C1E6EF3C3026CF340
:10F970000712227282B24A454FEA104C84BF0CF142
:10F98000010C1FFA8CFC09EB0C4906EB0800CDF8C2
:10F990003090FFF7BFFD0DF1880A68314AF8681D05
:10F9A0006066514607A800F0CCF9079B626E93424F
:10F9B00004D0EE685C495D48B047C1E72A6909F1A7
:10F9C0000101BBF1000F2CD05160227A04F10C032D
:10F9D000049313091A4606F108010498059308F0E8
:10F9E0003AFA6A69117810290CD90DF12A010191AE
:10F9F0000021CDF8089000915B46DDE90401583202
:10FA000000F07CFB237A1B0903F10C0297422DD9ED
:10FA100003F10D02974206D1002345482377EB6896
:10FA20006BE79160D1E70933A8EB0300617FC0B2B7
:10FA300020776A6961B958321E4408920996ADF878
:10FA400028002B689847A06620B9EB68394868E71A
:10FA50008832F1E7514600F043FA00283FF74EAFF5
:10FA6000EB68354898476B68A06E5AE70023237708
:10FA7000A36643E7212F01D101232AE1EB682F4838
:10FA80004FE79DF83F30043F09EB0700DB09FFF724
:10FA900041FD6E696066A3B30DF1580A0021302262
:10FAA000504608F0FCF9FF2332468DF8583052F8E2
:10FAB000083F0DF15900CDF8593053683836CDF86C
:10FAC0005D30FFF729FDB6F860303A468DF86130B9
:10FAD00049461B0A0DF163008DF8623008F0BBF94E
:10FAE000CDE9086A08F1070808A907A8ADF8288039
:10FAF00000F0C0F9636E079A9A4223D0EB68104871
:10FB00000FE72836CDE90869A8F10408ECE700BF43
:10FB1000104C002044E90108BEE90108D6E90108BB
:10FB200004EA010853EA010800C701088EEA010847
:10FB3000D3EA010807EB010839EB01085FEB010884
:10FB4000D1EB01089DF837609DF83630360446EA5F
:10FB500003269DF835300DF13B001E4366609DF88D
:10FB60003A709DF839303F0447EA03279DF8383052
:10FB70001F43A760FFF7CEFCE0609DF83F20237C89
:10FB8000D10961F3C713110961F3061362F303038B
:10FB900023749DF84030637494F8213003B322AB92
:10FBA00033F8472D9B786282237522AB33F8442DBE
:10FBB0009B78A4F81520E37522AB33F8412D9B7890
:10FBC0002283A37622AB33F83E2D9B78A4F81B202A
:10FBD000637722AB33F83B2D9B78E28384F82030A7
:10FBE0006D6994F9102005F1280C002AB5F89810D9
:10FBF00004F1230004F15303CDF858C016AA12DA19
:10FC000005F11807ADF868100092083504F14302B9
:10FC100004F13301CDE91776199500F0FCF90123C1
:10FC200084F822306AE6ADF864101946CDE917670A
:10FC300000F0B0F90023F3E7EB68394871E6701C77
:10FC4000FFF768FC804501466060EB687FF475AEA5
:10FC50004146344898470023052F6377A7F10408ED
:10FC600007D9737903F00F0308339845C4BFF35CD9
:10FC70006377F37996F8069096F805C049EA032968
:10FC8000637FA4F80A906969002B7FF45EAE01F1EE
:10FC900058024FF0010E0878CDE908266268102856
:10FCA000CDF82A20ADF828808DF82EE02A6902D9F7
:10FCB000002B7FF44DAE90684FF0000B4AE6032B0B
:10FCC000BDD0052BBBD0012BB6D1112F7FF4D2AE06
:10FCD000002384F821306B691FFA87F828330893D2
:10FCE000731C099308F1FF33ADF82830337808A965
:10FCF0000DF135008DF8343000F0D4F800280DF106
:10FD000034093FF7BEAEEB6807480AE6032B01D083
:10FD1000052BD8D1701CFFF7FDFB60609BE700BF8F
:10FD200006EC010823EA0108AEEB01080022FFF708
:10FD3000CDBD0B0A017043700B0C090E8370C170AE
:10FD4000704770B51025CEB00C462A4606460021F5
:10FD5000684608F0A4F849238DF80030A37BD4F856
:10FD60000A100DF106008DF80530FFF7E2FF21695A
:10FD70000DF10A00FFF7DDFF238908A88DF80F3089
:10FD800000F000FA216808A800F00CFA2A4669463B
:10FD900008A800F00DFA2289616808A800F008FAA6
:10FDA00008A90DEB050000F06EFA049B33604EB01D
:10FDB00070BD492370B500250C460646CEB08DF8BF
:10FDC00000300B8BCDE901558DF801301B0A8DF801
:10FDD00002308B7E03958DF80330CB7E0DF106004B
:10FDE0008DF804300B691968FFF7A3FF61690DF105
:10FDF0000A00FFF79EFFA38908A88DF80F308DF841
:10FE00000E5000F0BFF9216808A800F0CBF9694650
:10FE100008A8102200F0CCF9A289A16808A800F077
:10FE2000C7F908A904A800F02EFABDF8103008A8F8
:10FE300033808DF804508DF803508DF802508DF802
:10FE4000015000F09FF9616808A800F0ABF969461D
:10FE500008A8102200F0ACF9A289A16808A800F057
:10FE6000A7F908A904A800F00EFABDF810307380B5
:10FE70004EB070BD30B50C46CBB0054604A800F0BE
:10FE800081F9216804A800F08DF92289616804A82D
:10FE900000F08EF904A9684600F0F5F9009B2B608C
:10FEA0004BB030BD70B50C89BEB006460D46A4B14E
:10FEB00014F00F0411D101AA10212868FFF740F9AE
:10FEC0002889A04201DC3EB070BD68683119204429
:10FED00001AAFFF7AFF91034F2E74FF0FF30F2E775
:10FEE0002DE9F0430F89C7B081460D46002F4ED053
:10FEF000012410224FEA1718002117F00F0701A85C
:10FF000018BF08F1010807F0CAFFAB7BD5F80A104B
:10FF10000DF10A008DF809308DF80440FFF709FF54
:10FF200029690DF10E00FFF704FF6E68013E44459C
:10FF300003DD288947B0BDE8F08309AA10212868AD
:10FF40008DF81340FFF7FCF809AA05A901A8FFF7EF
:10FF500071F9444510DB002F14BF3B461023304697
:10FF60004A464B440DF1130C934207D80134A4B216
:10FF700009F110091036DAE71023F0E710F801EF65
:10FF80001CF8011F81EA0E0102F8011BECE74FF09B
:10FF9000FF30CFE770B5C2B0144606460D46F122D9
:10FFA000002105A807F07BFF0023CDE90333636838
:10FFB00010218DF805301A0A1B0C8DF80730A36844
:10FFC0008DF806208DF808301A0A1B0C8DF80A30BF
:10FFD000A3898DF809208DF80B301B0A8DF80C30A1
:10FFE000012305AA20688DF80430FFF7A9F805AAB7
:10FFF000314601A8FFF71EF9022305AA1021206847
:020000040801F1
:100000008DF80430FFF79CF805AA294601A8FFF7F0
:1000100011F942B070BD2DE9F0431025C3B04A9CE0
:1000200080460F4616460021F12205A8994607F0A2
:1000300036FF2A46002101A807F031FFA2682946B1
:100040008DF80520130AEA408DF80720E2688DF844
:100050000630D37920688DF8083093798DF809300F
:1000600053798DF80A3013798DF80B30D3788DF8E9
:100070000C3093788DF80D3053788DF80E3013785E
:1000800005AA8DF80F30238A8DF810301B0A8DF8E1
:10009000113001238DF80430FFF752F805AA4146CC
:1000A00001A8FFF7C7F8022305AA294660688DF862
:1000B0000430FFF745F805AA494601A8FFF7BAF84A
:1000C000032305AA294620688DF80430FFF738F885
:1000D00005AA394601A8FFF7ADF8042305AA294669
:1000E00020688DF80430FFF72BF805AA314601A8E7
:1000F000FFF7A0F843B0BDE8F0830000F0B50F298A
:10010000C7B004460D4616461F4604D94FF4A171E8
:100110001B48F3F7F3FF0123002F019318BF0223BD
:100120008DF808309DF830310DF10A0083F001039D
:100130008DF809304D9B1968FFF7FBFD4E990DF1C5
:100140000E00FFF7F6FD4FF4807309AA1021304628
:1001500005AEADF81230FEF7F3FF09AA314601A84B
:10016000FFF768F80023601EDAB2954201D847B065
:10017000F0BD10F8012FF15C01334A400270F3E743
:1001800040EC010810B5102204460021F13007F0C0
:1001900086FE00212046C4F81411F022BDE810406C
:1001A00007F07DBE0B46024610211846FEF7C8BF79
:1001B0002DE9FF470446D0F814010E46154604F217
:1001C000011920B3C0F110089045474628BF1746D3
:1001D00048443A4607F03FFED4F814313B440F2B15
:1001E000C4F814311ED9A8451CD204F1F1031946F4
:1001F00013F8012BD87B4B4582EA000203F8012C4F
:10020000F6D122460846FFF715F83E44ED1B0DF1E6
:10021000100A102D09D82A463146484607F01BFE21
:10022000C4F8145104B0BDE8F08704F1F002731E65
:1002300006F10F0013F8017F12F8011F834281EAD3
:1002400007011170F6D16A4604F1F103984617468A
:100250009446186859680833ACE803004B45624679
:10026000F6D1224639463846FEF7E4FF43463A4681
:1002700003CA524518605960174603F10803F6D1C6
:100280001036103DC5E7F0B50C4689B010220021AC
:100290000546684607F003FE224669466846FEF7B3
:1002A000C9FF9DF900306A46002B0DF10F0140DABD
:1002B000137812F8010F5B005BB243EAD01391424E
:1002C00002F8013CF4D19DF80F305B0083F0870306
:1002D0008DF80F30D4F81431102B39D1002304F2EB
:1002E000011211781DF8030001334140102B02F870
:1002F000011BF6D104F1F102134604F2011712F8C2
:10030000011BD07B974281EA000102F8011CF6D163
:1003100004AA9446164618685968083303C6BB42B7
:100320003246F7D1224629466046FEF783FF09B0E0
:10033000F0BD137812F8010F5B005BB243EAD013F3
:100340008A4202F8013CF4D19DF80F305B00BFE710
:100350009DF900206846002A28DA027810F8016F1B
:10036000520052B242EAD612814200F8012CF4D176
:100370009DF80F20520082F0870280218DF80F2017
:10038000E21882F80111002201330F2B1DD9C4F8A5
:100390001431002304F2011211781DF80300013317
:1003A0004140102B02F8011BF6D1A3E7027810F8A8
:1003B000016F520052B242EAD612814200F8012C7B
:1003C000F4D19DF80F205200D7E7E11881F8012100
:1003D000DAE70000002103E00A4B5B584350043188
:1003E00009480A4B42189A42F6D3094A02E0002310
:1003F00042F8043B074B9A42F9D300F00DF8F0F7AE
:100400007DFF70475CF90108000000208004002097
:10041000800400205C530020314B82B01A6842F403
:1004200080721A6099682F4A0A409A601A6822F00E
:10043000885222F001121A601A6822F480221A608F
:100440009A6822F47D029A600022DA6001921B68A9
:1004500013F4007318BF01230193019B012B37D1C3
:100460004FF48051204B1A68A3F5806322F00102FB
:10047000C3F80024D3F8002422F00202C3F80024B9
:10048000D3F8002422F00402C3F800245A6A42F090
:1004900080525A62154A11605168C906FCD49A68A4
:1004A0009A609A689A609A689A605A6822F46042E0
:1004B0005A605A6842F440425A609A6822F0030235
:1004C0009A609A689A60064A936813F00C0FFBD101
:1004D0004FF00062064B9A60064ADA6002B070473D
:1004E000003802400CC0FF88003C02400070004011
:1004F00000ED00E00003FA0570B5064688B02E480E
:1005000001F010FD2D4B1A680092009A91073CD51E
:1005100001214FF4007001F05FFF012001F052FD56
:10052000274A536843F400335360A2F537425368B7
:100530001B07FCD50024012502A801F02DFD02A90E
:100540001D488DF80D4006948DF81C508DF80C4018
:1005500001F0FCFC2A4606233146174801F03EFD17
:100560002946154801F024FD0221134801F0C8FD79
:10057000114801F0B7FD134D01940F4C02212046A4
:1005800001F0B8FD58B108B070BD1A6842F0010220
:100590001A60009A9207BBD41A680092F9E7019B8F
:1005A00001330193019BB3F5805FE7DB38212846D7
:1005B000F3F7A4FDE2E700BF002401400038024049
:1005C0000027014093EC010808B5002001F0FAFC77
:1005D0000021074801F0ECFC00214FF4007001F00D
:1005E000FBFE044A136823F00103136008BD00BF3B
:1005F000002401400038024013B5072301220146C0
:10060000114801F0EBFC02210F4801F079FD0E4882
:1006100001F068FD00230D4C019302210A4801F00E
:1006200069FD28B1084802B0BDE8104001F05FBD87
:10063000019B01330193019BB3F5805FEDDB4C21FE
:100640002046F3F75BFDE8E70024014093EC010846
:1006500070B506460825FFF74FFF00243046FFF728
:10066000CBFF013D0444F9D1FFF7AEFFC4F3CF0047
:1006700070BD00000000000008B51120FFF7E8FF82
:1006800006F078FE0146084806F080FF06F05AFAA8
:1006900003A3D3E9002306F0ADFA06F065FD08BD1B
:1006A0002FDD24068195F33F00F07F450F4A536A02
:1006B00043F0805353620E4B1A465968C906FCD466
:1006C0001B68022823F4C05306D143F4C0531360BF
:1006D0005368DB06FCD47047012802D143F48053F1
:1006E000F5E70028F3D143F40063F0E70038024057
:1006F0000070004010B50C4B5A68D206FCD41C6840
:1007000014F4C05F0BD114F480500AD114F40064C7
:1007100004D106482A21F3F7F1FC204610BD02203F
:10072000FCE70120FAE700BF00700040E1EC01089F
:1007300038B50546012001F0F3FC022D01BF154A32
:10074000136843F001031360134B1A6842F48032BC
:100750001A601A689203FCD542F690529A60996822
:100760009142FCD19A6842F002029A600A4B9C685E
:1007700014F00804FBD14FF480321A60074B084A8A
:1007800028461A60FFF792FF2046BDE8384001F086
:10079000BBBC00BF003C024000380240F801002012
:1007A00000093D0038B50546012001F0B9FC022DD5
:1007B00001BF144A136843F001031360124B1A6817
:1007C00042F480721A601A689205FCD55A6822F4C5
:1007D000604242F440425A6000229A600A4B9C6890
:1007E00014F00C04FBD14FF480721A60074B084AD6
:1007F00028461A60FFF75AFF2046BDE8384001F04E
:1008000083BC00BF003C024000380240F8010020D9
:10081000D0FE3F000C4B5A6B900513D45A6A42F03D
:1008200080525A62094A116841F480711160596B13
:1008300041F480715963596B8905FCD5136823F421
:1008400080731360704700BF0038024000700040A2
:10085000054B5A6B910706D45A6B42F001025A635A
:100860005A6B9207FCD5704700380240094B5A6A10
:1008700042F020025A629A6942F020029A619A6913
:1008800022F020029A610022A3F509331A801A850A
:100890005A6270470038024015210238002248434E
:1008A0000121064B1A85D86299825A621A821980F0
:1008B0001A8AD207FCD500221A8070470014004023
:1008C000002349F6FE7282B00193019B934201DD41
:1008D00002B07047019B01330193F6E7002340F615
:1008E000FE7282B00193019B934201DD02B070471A
:1008F000019B01330193F6E7002382B00193019B32
:10090000B3F5CC7F01DD02B07047019B0133F5E701
:10091000D0B1012801D1FFF7EFBF0C4B00211A68BD
:100920004FF47A73B2FBF3F2094B013A92B21A8593
:1009300001220138D8629A82596219821A801A8A71
:10094000D207FCD500221A80704700BFF8010020B2
:100950000014004000F1774303F57803B3F5804FAE
:100960002DE9F04106460C4617462DD202F1F73329
:1009700003F608030344B3F5804F25D2FFF7BAFE10
:10098000804610B10020FFF791FE01F0E1FB012548
:100990002744361BA7420AD101F0EAFBB8F1000F49
:1009A00002D04046FFF782FE2846BDE8F08141F6BE
:1009B000027001F0E5FB301914F8011B01F03CFC5A
:1009C000042818BF0025E5E70025EDE710B50C4623
:1009D00000F1774101F57801B1F5804F0DD202F1B8
:1009E000F73303F608030344B3F5804F05D20146FD
:1009F000204607F030FA012010BD0020FCE700007F
:100A000008B5114B984215D003F58063984213D076
:100A100003F58063984211D003F5806398420FD0AC
:100A200003F5006398420DD0084B094A1421094888
:100A300007F0BEF8002008BD0120FCE70220FAE71D
:100A40000320F8E70520F6E70000024078ED0108F2
:100A500032ED010891ED01080F2808B505D9094BC1
:100A6000094A3B21094807F0A3F8012303FA00F0E3
:100A7000C043074A51680140516013681840106034
:100A800008BD00BFE2ED01083CED010891ED010851
:100A9000000401400F292DE9F84F82460D46934688
:100AA0001F4605D95A4B5B4A54215B4807F080F832
:100AB0004FF0010909FA05F900F0B8F86FEA0903E7
:100AC000564E032D7268564C02EA03027260326879
:100AD00003EA0203534A3360136A43F001031362CB
:100AE0002ED80F22A3684FEA850802FA08F223EAFB
:100AF0000203A3605046FFF783FFA36800FA08F0E3
:100B00001843A0601BF0020F18BFB368464A1CBF11
:100B100043EA0903B3601BF0040F1EBFF36843EA06
:100B20000903F360336843EA090333603B01DBB236
:100B3000002D45D182F8063340231360BDE8F88FBD
:100B4000072D13D80F22A5F10408E3684FEA88089F
:100B500002FA08F223EA0203E3605046FFF750FF6F
:100B6000E36800FA08F01843E060CBE70B2D13D8D8
:100B70000F22A5F1080823694FEA880802FA08F253
:100B800023EA020323615046FFF73AFF236900FA84
:100B900008F018432061B5E70F22A5F10C0863693E
:100BA0004FEA880802FA08F223EA0203636150461A
:100BB000FFF726FF636900FA08F018436061A1E7B8
:100BC000012D03D182F807338023B6E7022D04D12B
:100BD00082F808334FF48073AFE7032D04D182F815
:100BE00009334FF40073A8E7042D04D182F80A33C7
:100BF0004FF48063A1E7092D04D882F817334FF42E
:100C000000039AE782F828334FF48073536095E726
:100C1000EEED010857ED010891ED010800040140D7
:100C2000000001400038024000E100E0144B98420F
:100C300005D1144AD36943F00103D3617047124BC5
:100C4000984204D10F4AD36943F00203F5E70F4BF2
:100C5000984204D10B4AD36943F00403EDE70C4BEF
:100C6000984204D1074AD36943F00803E5E7094BEA
:100C70009842E3D1034AD36943F02003DDE700BF84
:100C80000000024000380240000402400008024018
:100C9000000C0240001402400323490010B5846890
:100CA0008B4024EA030484600124022A04FA01F43C
:100CB00007D0032A0DD0012A07D18368234383601C
:100CC00003E083688A401A43826083681C4384601F
:100CD00010BD82681343F2E70F29F8B504460F46AA
:100CE00015461E4603D94B211948F3F707FA20464B
:100CF000FFF79CFF03237A009340DB4321681940F0
:100D000021600121D4F800C001FA02F04CEA000C85
:100D1000B940C4F800C009B266B1A688314389B2AF
:100D2000A180E168012D03EA0103E36006D0022DF2
:100D300008D0F8BDA68826EA0101F1E7E36803437D
:100D4000E360F6E7E36805FA02F21A43E260F0E7CF
:100D50003EEE01080F2970B505460C46164603D92C
:100D60006B210E48F3F7CAF92846FFF75FFF03230C
:100D700061008B40DB43EA68012E02EA0302EA606D
:100D800005D0022E03D02A6813402B6070BDEA689C
:100D900006FA01F11143E960F5E700BF3EEE0108F4
:100DA0000F2910B505D9074B074A8121074806F0DE
:100DB000FFFEFFF73BFF4B00032102689940114300
:100DC000016010BDE2ED0108FAED01083EEE0108F8
:100DD0000F2938B50446154605D987211B4B1C4AF7
:100DE0001C4806F0E5FE0F2A03D91B4B184A882140
:100DF000F6E7FFF71BFF07294FF00F0318D8006A2B
:100E00008A00934020EA03032362236A05FA02F270
:100E10001A4322620322236849008A4023EA02031C
:100E200023600223226803FA01F11143216038BDD7
:100E3000A1F10802406A9200934020EA0303636232
:100E4000636A95401D436562E4E700BFE2ED010877
:100E50000DEE01083EEE01082BEE0108012303FA16
:100E600001F189B201837047012303FA01F189B2CC
:100E700041837047012303FA01F189B20AB101836A
:100E8000704741837047008A084100F001007047B5
:100E90000F2938B505460C4603D9B4210548F3F7A8
:100EA0002DF928686400E04000F00300431E58421A
:100EB000584138BD3EEE0108808A084100F001002B
:100EC0007047000010B5084C23681BB90120F0F7EB
:100ED0008BFF206023682BB9BDE810403621034802
:100EE000F3F70CB910BD00BF2C4C00208DEE0108AB
:100EF00010B50B4C22681AB93C210A48F3F7FEF8EA
:100F0000206842F21071F1F7B7F801280CBF0124F4
:100F1000002403D040210348F3F7F0F8204610BD29
:100F20002C4C00208DEE010810B5074C22681AB930
:100F300051210648F3F7E2F8002320681A46BDE87D
:100F400010401946F0F7ACBE2C4C00208DEE010885
:100F500010B50446FFF7B6FFFFF7CAFF214610227F
:100F6000034801F025FF0446FFF7DEFF204610BDD1
:100F70000054004010B5FFF7A5FFFFF7B9FF01F0DF
:100F8000CFFE0446FFF7D0FF204610BD08B513463C
:100F90000A460146034801F003FB003018BF012058
:100FA00008BD00BF0054004008B513460A4601467C
:100FB000034801F0F5FB003018BF012008BD00BF59
:100FC0000054004008B513460A460146034801F0A4
:100FD000C3FC003018BF012008BD00BF0054004012
:100FE00008B513460A460146034801F045FD0030A6
:100FF00018BF012008BD00BF0054004008B51346CB
:101000000A460146034801F08FFD003018BF012059
:1010100008BD00BF005400400123064A83405169C7
:10102000194205D05361044B53F8203003B11847DF
:10103000704700BF00040140304C00200F2838B535
:1010400004460D4603D926210348F3F757F8034B0E
:1010500043F8245038BD00BFDBEE0108304C0020BF
:101060000020FFF7D9BF0120FFF7D6BF0220FFF70E
:10107000D3BF0320FFF7D0BF0420FFF7CDBF08B5D3
:101080000920FFF7C9FF0820FFF7C6FF0720FFF779
:10109000C3FF0620FFF7C0FFBDE808400520FFF7AB
:1010A000BBBF08B50F20FFF7B7FF0E20FFF7B4FF57
:1010B0000D20FFF7B1FF0C20FFF7AEFF0B20FFF76D
:1010C000ABFFBDE808400A20FFF7A6BFFEE7FEE73A
:1010D000FEE7FEE7FEE7FEE7FEE7FEE7FEE7FEE7E8
:1010E000FEE7FEE7FEE7FEE7FEE7FEE7FEE7FEE7D8
:1010F000FEE7FEE7FEE7FEE7FEE7FEE7FEE7FEE7C8
:10110000FEE7FEE7FEE7FEE7FEE7FEE7FEE7FEE7B7
:10111000FEE7FEE7FEE7FEE7FEE7FEE70A23B0FB99
:10112000F3F203FB120040EA0210C0B27047000065
:10113000CA22024B5A6253225A627047002800406A
:10114000014B1860704700BF704C00204FF4003214
:101150000F4B10B50F4C5A61E368DB0503D4302107
:101160000D48F2F7CBFFFFF7E3FF4FF40072A368DF
:1011700023F48853A360094BC3F88420FF236362E0
:10118000074B1B6813B1BDE81040184710BD00BFE6
:10119000000401400028004029EF010800E100E0C0
:1011A000704C00202DE9F04F9846374B85B01B78E6
:1011B000824691469DF838709DF83C602BB9334BC0
:1011C000334A8C21334806F0F3FC431E1E2B59D8BA
:1011D0000C2957D8A2F5FA63632B53D8B8F1170F2F
:1011E00050D83B2F4ED83B2E4CD802F13000C0B225
:1011F000FFF794FF83460846FFF790FF04465046EA
:10120000FFF78CFF40F400554046FFF787FF45EAA3
:101210000B4545EA042504463846FFF77FFF0002E8
:1012200040EA04443046FFF779FF20431A4CFFF7A9
:101230007FFFE36843F08003E360E3685B06FCD56F
:1012400065602060E36823F08003E360124BDA6896
:101250009206FCD5FF2204A85A6200F80C6D8DF8A6
:1012600007A08DF80810ADF809908DF806808DF86C
:101270000570FAF776FC094BC3E90001012005B0BF
:10128000BDE8F08F0020FAE7744C0020AAEF0108B7
:1012900077EF010829EF010800280040784C002072
:1012A00037B50578C4788378B0F8052001790195C1
:1012B000407800902046FFF775FF03B030BD000076
:1012C00038B52B4B04461B781BB9E4212948F2F7AB
:1012D00015FF294AD36823F02003D360D3689B0607
:1012E000FCD513685268C2F30741080900EB80007F
:1012F00001F00F0101EB4001C9B201F5FA61A4F858
:101300000510C2F30721C1F300108500284401F045
:101310000F0101EB4001D2B22171C2F3011101EBC7
:10132000810102F00F0202EB4102E270C3F30742B7
:10133000C2F3011101EB810102F00F0202EB410245
:10134000A270C3F30722C2F3021101EB810102F084
:101350000F0202EB4102DBB26270C3F3021202EB36
:10136000820203F00F0303EB4203237038BD00BF7A
:10137000744C002029EF0108002800401FB501A887
:10138000FFF79EFF01A8FAF7ECFB05B05DF804FB40
:1013900008B5FFF73FFA1B4A136843F480731360E4
:1013A000FFF7C6FE184A536B23F4403343F482031D
:1013B0005363164BDA6842F08002DA60DA6851064D
:1013C000FCD5FF221A611A6942F4FE021A619A687A
:1013D00022F040029A609A6822F44C529A60DA68CD
:1013E00022F08002DA60094BDA689206FCD5FF220F
:1013F0005A620122064B1A70FFF7C0FF054BC3E982
:10140000000108BD00700040003802400028004084
:10141000744C0020784C002008B5094B1B7823B988
:1014200040F21F110748F2F769FEFFF781FE064BF5
:101430009A6822F480729A60FF225A6208BD00BF47
:10144000744C002029EF01080028004008B5144B17
:101450001B7833B9134B144A40F22711134806F096
:10146000A7FBFFF765FE124BDA6822F48072DA60A0
:10147000104A916841F400319160116841F40031E3
:101480001160F0210C4A82F829134FF40071516069
:101490009A6842F488529A60FF225A6208BD00BFDF
:1014A000744C0020AAEF010883EF010829EF01081E
:1014B000002800400004014000E100E0F8B51E46AD
:1014C000194B17461B7833B9184B194A4FF4A571BD
:1014D000184806F06DFB184CFFF72AFEA56825F4A6
:1014E0008075A560E56825F48075E560FFF716FE58
:1014F00005460846FFF712FE000440EA056138463B
:10150000FFF70CFE05463046FFF708FE084340EAA9
:101510000520E368DB07FCD5FF23E0616362BDE8DB
:10152000F840FFF793BF00BF744C0020AAEF0108FA
:1015300098EF010829EF010800280040037842785D
:101540008178C078FFF7BABF38B50D460446F2F788
:10155000F1FA1F4A136823F001031360F2F70AFB44
:1015600025B11C4A536843F00603536072B6BFF3BB
:101570004F8FBFF36F8F184A0120136823F00303C6
:1015800043F4007343F00103136000F0D5FD134BE7
:101590001A6942F004021A6130BF1A6922F004028B
:1015A0001A610F4B0F4A1B6893420AD10220FFF7C2
:1015B000F9F8074A136843F00103136004B162B6F7
:1015C00038BD094A9342F4D10220FFF7B1F8F0E7A1
:1015D00010E000E0002004E00070004000ED00E0BA
:1015E000F8010020D0FE3F0000093D0062B67047C0
:1015F00000220E4B10B51A700D4A0E4C138820466F
:1016000023F040031B041B0C13800D210222FFF763
:10161000A1FB204602220E21FFF79CFB2046BDE8DD
:10162000104002220F21FFF795BB00BF804C002025
:10163000003800400004024038B50546274A2848D3
:10164000536A0C4643F4804353620D210522FFF791
:10165000BFFB05220E212248FFF7BAFB05220F210E
:101660001F48FFF7B5FBC5B101220D211C48FFF74C
:1016700013FB01220E211A48FFF70EFB01220F2156
:101680001748FFF709FB012C21D144F451740122C2
:10169000144B1C80144B1A7038BD2A460D2110487B
:1016A000FFF7FAFA2A460E210D48FFF7F5FA2A4607
:1016B0000F210B48FFF7F0FA012C05D0022C03D0C4
:1016C000032C14BF0024032444F45974DFE7022CD4
:1016D000DBD0032C0CBF03240024D6E700380240E3
:1016E0000004024000380040804C0020064B074AAE
:1016F000988111781A461889C00701D40029FAD1B7
:101700009089C0B2704700BF00380040804C002074
:10171000284A38B5136A054643F4805313620522FC
:1017200025480C461146FFF753FB052206212248A7
:10173000FFF74EFB052207211F48FFF749FBC5B104
:10174000022205211C48FFF7A7FA022206211A48A7
:10175000FFF7A2FA022207211748FFF79DFA012C92
:1017600021D144F451740122144B1C80144B1A7083
:1017700038BD2A4605211048FFF78EFA2A46062171
:101780000D48FFF789FA2A4607210B48FFF784FA2C
:10179000012C05D0022C03D0032C14BF00240324F9
:1017A00044F45974DFE7022CDBD0032C0CBF032474
:1017B0000024D6E70038024000000240003001401B
:1017C000814C002000220E4B10B51A700D4A0E4CB1
:1017D0001388204623F040031B041B0C13800521B3
:1017E0000222FFF7B7FA204602220621FFF7B2FADB
:1017F0002046BDE8104002220721FFF7ABBA00BF28
:10180000814C00200030014000000240064B074A96
:10181000988111781A461889C00701D40029FAD195
:101820009089C0B2704700BF00300140814C002059
:10183000054AD36823F4E0631B041B0C43F0BF6329
:1018400043F40033D360704700ED00E02022002114
:10185000114B10B5C3F88420104B114C1A6A204666
:1018600042F480421A625A6942F480425A615A69CB
:1018700022F480425A610B4A91811A6A092122F4AA
:1018800080421A620222FFF765FA2046BDE8104046
:1018900002220A21FFF75EBA00E100E000380240B0
:1018A000000002400038014008B5064B02461860AF
:1018B00000B1012240F22551034800F02CFE012026
:1018C00008BD00BF844C00200038014010B50B4C0F
:1018D00040F22551204600F03CFE48B1204600F081
:1018E00016FE074BC0B21B6833B1BDE81040184765
:1018F000A388044ADBB2137010BD00BF003801405A
:10190000844C0020D452002010B5044680210848A1
:1019100000F019FE0028F9D02146054800F0F3FD3B
:10192000034C4021204600F00EFE0028F9D010BDE7
:101930000038014010B5441E14F8010F00B910BD65
:10194000FFF7E2FFF8E7000008B5024800F0DFFD0E
:10195000C0B208BD003801402DE9F043884601219E
:1019600089B08146084614461D4600F029FD012134
:101970004FF4804000F030FD4FF4C0670223012295
:10198000002602A93F488DF80C308DF80D308DF8F7
:101990000F2002978DF80E6000F074FC07220921D9
:1019A000384800F0B1FC07220A21364800F0ACFCB0
:1019B000B8F1450FCDF810903CD14FF48063ADF8ED
:1019C0001830072C42D10023ADF81430052D4ED12C
:1019D0004FF48053ADF816300023ADF81C300C23C3
:1019E00004A92948ADF81A3000F032FD274B1A68D7
:1019F00002B1012240F22551234800F08CFD012163
:101A0000214800F075FDFFF79FFF25238DF8043076
:101A10009DF840308DF8053000238DF80630012305
:101A20008DF80730FFF704FF01A800F05FFA09B056
:101A3000BDE8F083B8F14F0F02D1ADF81870C0E7E0
:101A4000072CADF818600DD1592107E0082C02D100
:101A50004FF48053B8E7092CB8D154210C48F2F761
:101A60004DFBB3E7082CAED0092CAFD1F0E70F2D1A
:101A700002D14FF44053ADE7022D0CBF4FF4005399
:101A80000023A7E70000024000380140844C0020FA
:101A9000B3EF01080E2307B5082200934E2101235E
:101AA000FFF75AFF03B05DF804FB0000402200215D
:101AB0000D4B0E48C3F884200D4B5A6A42F4003295
:101AC0005A629A6942F400329A619A6922F40032A9
:101AD0009A61084A91815A6A032122F400325A62BB
:101AE0000222FFF737B900BF00E100E0000002402A
:101AF000003802400044004008B5024800F007FDED
:101B0000C0B208BD004400402DE9F04F4FF000097D
:101B10001F46262389B09DF848808A4614468DF8D2
:101B2000043083469DF84C509DF850608DF8058038
:101B30008DF806908DF80790FFF77AFE01A800F067
:101B4000D5F90121084600F03BFC01214FF400309B
:101B500000F04EFCB5B10823029302238DF80E90DD
:101B60008DF80C304FF00309012302A956488DF877
:101B70000F308DF80D9000F085FB07224946524842
:101B800000F0C2FBBEB10423029301238DF80F3095
:101B900000234FF002098DF80E30032302A94A48B2
:101BA0008DF80C908DF80D3000F06CFB0722494643
:101BB000454800F0A9FBBAF1450FCDF810B043D16C
:101BC0004FF48063072CADF818304BD10023ADF8EB
:101BD0001430052F57D14FF480530024ADF8163040
:101BE000ADF81C40002E59D1ADF81A6075B1BDF8A2
:101BF0001A3043F00403ADF81A30344B1A6802B1BE
